:020000040000FA
:080000000002040000000000F2
:020000040000FA
:10040000AF0121000E7F22000E01880000000000D5
:100410000C000700C0FF26000100200011000700AB
:10042000000020000000E000020032000000020096
:1004300000000000B8710200000000000040DA0077
:100440000000FE004440A900409A21000000E000A6
:100450000300320000002000A00188004440A800F2
:100460000000060091018800800078000000EB0089
:1004700015003700E280400032A0B4009101BA00BC
:10048000E280400032A0B4009102BA00E280400055
:1004900032A0B4000002EB00472BDE00F507B200EB
:1004A000602CE10004003A000059EB008301E900F0
:1004B000FDFF3E00040037006128E100010032002A
:1004C0000082EB00040007001101BA000200E00006
:1004D000E8FF3A00000006003159BA008301E90044
:1004E0000C0032002159BA008301E90008003200F3
:1004F0000400E00003003A00E280400032A0B400B3
:10050000F5FF370011D9BA008301E900FAFF3A007C
:100510008100E800E180400032A0B4000000060045
:1005200006600400000000000C60040000000000F1
:10053000B0600400000000009A60040000000000A9
:100540000E600400000000002660040000000000AF
:100550006A60040000000000DC600400000000008D
:10056000F060040000000000F660040000000000DD
:100570001E6104000000000056610400000000003D
:100580009A61040000000000B26104000000000055
:10059000B861040000000000CC610400000000000D
:1005A0001462040000000000AE7C040000000000A3
:1005B000B47C040000000000EC7C0400000000009B
:1005C0002048040000000000284B04000000000048
:1005D000464B0400000000007648040000000000C4
:1005E000AA48040000000000DE48040000000000EB
:1005F000FA48040000000000E04A04000000000087
:100600004E4C0400000000002C48040000000000D4
:100610002E480400000000004848040000000000CC
:100620003048040000000000D04A04000000000030
:10063000744C040000000000644C04000000000042
:10064000F84B040000000000244C040000000000EF
:10065000C04A040000000000924B040000000000AB
:10066000684B040000000000164904000000000070
:10067000844C040000000000524904000000000007
:100680007E49040000000000B249040000000000A0
:100690005C4A040000000000744A040000000000EE
:1006A0006048040000000000C84B04000000000087
:1006B000B44C040000000000764F0400000000006D
:1006C000A64F040000000000E84F040000000000F6
:1006D000EA4F040000000000F64F04000000000094
:1006E0008E4F0400000000000250040000000000D3
:1006F00044500400000000006450040000000000AA
:10070000A650040000000000C650040000000000D5
:10071000025104000000000022510400000000000B
:100720003C510400000000006A5104000000000079
:10073000A251040000000000C451040000000000A9
:10074000F4510400000000002052040000000000EA
:100750004C52040000000000785204000000000029
:10076000A252040000000000BE520400000000007D
:10077000DC51040000000000C4520400000000002E
:10078000F0520400000000001C53040000000000B0
:1007900048530400000000007253040000000000F1
:1007A000E24F040000000000E44F040000000000DD
:1007B000E64F040000000000C253040000000000E7
:1007C000C453040000000000DC53040000000000DB
:1007D0000040DA000000FE001004B1000300350004
:1007E0009001B10001003C00100005000000050070
:1007F000800078001104B100030035009101B100C0
:1008000001003C000050A000000006001004B100F0
:10081000070035009001B100040034007000B10001
:10082000030035009001B10001003C0010000500FC
:10083000000005006900E100040035006D00E100E2
:10084000030034000002B100010032000000050086
:10085000100005002002E20004003D002342AB002E
:10086000020032002302AB00FEFF32000040DA003B
:10087000FEFF37000A00FA0080017800E20F500006
:1008800028003E00B0788000E10F500008003200E0
:10089000802320000000E000050032000423200037
:1008A0002523200046232000800178000400370023
:1008B000042220002522200046222000832220003E
:1008C000144090000004E000040035008009EB00B3
:1008D000144090000074A000104298001540900051
:1008E0000028A30003003A00154090000024A00057
:1008F000904298008001EB000700370015409000FF
:100900000008A300FDFF320063C078000000FB0078
:10091000000B78008301E800828F5100F7FF3A0056
:100920000800370030002000B0BF9F00C3BF9F0009
:10093000D1BF9F00E2BF9F006A80570000C0DA006D
:100940006FB99700020078000080FA0000000600EE
:100950000A00FA00881F7800800178000000E0009B
:1009600029003A00B0788000E10F50000800320002
:10097000802320000000E000050032000423200056
:100980002523200067232000800178000400370021
:10099000042220002522200067222000832220003C
:1009A000144090000004E000040035008009EB00D2
:1009B000144090000074A000104298000002EB0068
:1009C0000C003700130A20001544780061406400D1
:1009D00002003A008301E900FBFF3A000402E8004C
:1009E0009541780061C06100050032001700780071
:1009F0008058780004035100820F5200F1FF3A0042
:100A0000060051000800370020002000A0BF9F0012
:100A1000B3BF9F00C1BF9F00D2BF9F006C80570033
:100A200000C0DA005FB897004F0478000080FA0039
:100A3000000006000A00FA0011002000B1BF9F006C
:100A4000C0BF9F006A80570000C0DA004FB897000F
:100A50000080FA00000006000A00FA0051002000A1
:100A6000B1BF9F00C0BF9F006A80570000C0DA007E
:100A70005FB897000080FA0000000600889FBE0063
:100A800080047800C07880000000E00003003A0095
:100A9000100007000000E0000A003500C078800068
:100AA0000900E00002003A00000478000600370068
:100AB0000004780009004000060007000000E00084
:100AC00001003D000084EB00080078004F04BE00E8
:100AD00000000600800078000000E00004003A00FA
:100AE000A0F12000C07888000101780006003700DE
:100AF0000081EB00A0012100808F500002003E0029
:100B0000C17888000001EB000200780000000600B8
:100B1000020AB900001BB9000200B80081004200BF
:100B200081004300000006006022B8000602200099
:100B30000000D0008180D2000482D2008582D200E1
:100B40000000A0000202520083825A00030031001C
:100B50000202420083824A000000A1000603E9006D
:100B6000F3FF3A000000060004002000580237009E
:100B7000889FBE008A9FBE008C1F78006F0207000E
:100B80007602330003866C006450E10024003200DA
:100B90006420E100270032006150E10022003200B1
:100BA0006120E100210032008B854200EB07B1009B
:100BB0000134B800003AB8000804420089844A00B1
:100BC000013AB8000030B8008880400009014A00AE
:100BD0000400330000004000818048000201490009
:100BE0008B05E900C909DD008301700001003200B6
:100BF00013002000C814DE004814DD004709DE00A1
:100C00001200B200C808DE0008847000630207000A
:100C100001F0A1000CF0A70001F0A000580237007D
:100C20006120E1005A0232000801BE000200BE004D
:100C3000F7FF37006150E100FCFF3A005402370033
:100C40000001BE007B0207000470A70003F0A100B2
:100C500003F8A30013003A006509B1001000320048
:100C6000090035006928E100020035000100280074
:100C70000000050000004000818048008502E90076
:100C8000FCFF3A0000000600F88F42000500350026
:100C90008100D1000080D3008502E800FCFF3A000B
:100CA000000006008000EB0000000500889FBE00E9
:100CB0008A9FBE00010578000100E00004003500B5
:100CC00008003C000000E000200032000500370072
:100CD00060001000E080180002003B0001F02C00D2
:100CE0001A0037000004BE006011B8006B09200034
:100CF0000982CF00020039000882CF000441B00011
:100D0000694252000E00320008003B0082817100EF
:100D1000610164008904D1000884D3008B05E800D8
:100D20000442E800F9FF3A000500370008044400D7
:100D300089844C008B05E9000442E900FBFF3A007E
:100D4000160207000AF0A70001F0A0004F05BE0040
:100D50004F04BE000000060003F0A200889FBE0002
:100D60008A9FBE008C1F7800F4010700FB0133004E
:100D70006450E1004F0032006420E1005200320074
:100D800003826C0007003B000905D0000306D00079
:100D9000820F54000C065D00020039000200320090
:100DA00089017800030678008582550004003D0023
:100DB0000003FD008103FD008502EA008B854200EF
:100DC000840F720002003B0060001000E0801800F9
:100DD0006011B8000005EB007A28E1000A00390034
:100DE00006007800C75DDD00F707B2008780750058
:100DF0002D003700828171000A01780061056000D2
:100E00008180D1000080D3008502E900F9FF3B001A
:100E1000060440008784480002003B006004140080
:100E2000E0841C000988A300070032008A81710059
:100E300082817100610164008904D1000884D300BB
:100E40008B05E800170037000978A30013003A006B
:100E50000B00E000130034008B05E9000804440097
:100E600089844C000A4474000978A3000D003A00FC
:100E70000B00E000070034008B05E9000804440083
:100E800089844C0001003A000B0020000978A3007F
:100E9000F7FF32000001EB00020037008281710091
:100EA0000A017800BD0107000CF0A70001F0A000C6
:100EB000B30137006420E10002003A00838F6C0028
:100EC000B30133000801BE000200BE00AC013700D0
:100ED000889FBE008A9FBE008C1F78009701070084
:100EE0009E01330003866C006450E1002E00320046
:100EF0006420E100330032006150E1002F00320035
:100F00006120E1003100320085855500EB07B0001B
:100F100009002000080420000500370008044400F0
:100F200089844C000A0031000603430087834B008C
:100F30000001530081815B00F8FF33000203BE0013
:100F40000800A0000804440089844C00F6FF390022
:100F5000C639DD0083017300010032001300200058
:100F60008904D1000884D3000998A3000500320049
:100F70000800A7000300A0008904D1000884D30062
:100F80008B05E8008904D1000884D3000001EB0040
:100F90000281D2008101070001F0A1000CF0A7003E
:100FA00001F0A000760137006420E10078013200F2
:100FB0000801BE000200BE00F7FF37006120E1001B
:100FC000730132006000B800F3FF3700000020001A
:100FD00001F82700F0FF37000001BE00950107006F
:100FE0000470A70003F0A1006509B10016003200EB
:100FF0000D0035006828E10006003500F0FF2F00E5
:10100000F1FF27000300E00013003B00010028006F
:101010000000050000004000818048008502E900D2
:10102000FCFF3A0008003700F88F420002003C0045
:101030008000EB00000005008100D1000080D3009B
:101040008502E800FCFF3A000300E00002003B00DC
:1010500060001000E080180000000600B2FE0700EB
:101060000400BE0000000600881F7800000478001D
:101070005001BE004000BE000400400085804800D2
:101080000601490087814900009CBE000294BE0011
:101090000400E1000588E1000690E1000798E10006
:1010A00002003100680044001008E8004F04780096
:1010B00000000600F4874700889FBE008A9FBE009C
:1010C0008C9FBE008E1F78000205BE000004BE008B
:1010D000D4B79F00E5B79F00F6B79F0087BF9F007A
:1010E0000000EB00C0B79F00B0B79F00A0B79F0003
:1010F00090B79F0080B79F000D042000BFB09700FD
:101100004FB09700000140000000E0000F003D00DC
:101110004F08DE0000007100C0B79F009E0007006E
:1011200001003D0012002000A100070001003D0069
:1011300012002000A6000700B1000700B60007005B
:101140000F004000C8FF0700220037004F08DE00F4
:1011500000067100CCB79F008F00070001003D0022
:10116000120020009200070001003D001200200044
:1011700097000700A20007000FB297009FB29700E8
:101180002FB39700BFB39700A900070000005200DB
:1011900081805A0002015B0083815B0080B79F0061
:1011A00091B79F00A2B79F00B3B79F000007EB0065
:1011B0009F0007000020E10001A8E10002B0E1006B
:1011C00003B8E100010031001E0020000E005600AF
:1011D000C0B79F004FB297000400E0000700350041
:1011E00010002000010020006011B8000804700009
:1011F000898470000A0571008B8571008D06E900F5
:10120000BEFF3A000400E00003003D00820007003A
:101210000F00400094FF07004FA897000000E00077
:1012200004003A000FB497009FB497002FB59700C1
:10123000BFB59700940007004F0778004F06BE0027
:101240004F05BE004F04BE004F01B1000000060074
:10125000881F780018002000881F780095FF07007D
:101260008F87E9004F04780000000600801FEB0024
:1012700090FF07008F87E90000000600889FBE00EE
:101280008A9FBE008C1F78006E00070007003D009B
:1012900073000700E00F5B00E08F5B0007003D007C
:1012A000320007000006EB0004003700340007009E
:1012B00002003D002A0007001C0020007200070009
:1012C000E3FF07000203BE000002BE000C00E000C6
:1012D00001003200220007000400BE000601BE002B
:1012E0004F0678004F05BE004F04BE000000060008
:1012F000889FBE008A9FBE008C1F780051000700A7
:1013000005003D0056000700E00F5B00E08F5B002A
:1013100006003D00040037001900070003003D00EF
:101320006000B8006011B800100007005600070008
:10133000CEFF07000203BE000002BE000C00E0006A
:1013400001003200060007000400BE000601BE00D6
:101350004F0678004F05BE004F04BE000000060097
:101360006000B8006011B8000000370004025000AF
:101370008582580006035900878359000000060043
:101380000006EB00E00F5200E08F5A00E00F5B0018
:10139000E08F5B00000006000180400090B79F00D6
:1013A0000001EB008FB097000100E0000000060094
:1013B0000200700090B79F000180400080B79F003E
:1013C0000001EB00FFA897000100E000000006000C
:1013D0000200700080B79F00018040006FAA970054
:1013E000CF20DE0001007000F0AF9F000402420039
:1013F000250007004F18DE00000272000000060002
:10140000E4AF9F000804440089844C000A054D00A5
:101410008B854D00000006003FB29700CFB29700C9
:101420005FB39700EFB3970000FE2F0000000600A7
:101430003FB09700CFB097005FB19700EFB1970032
:10144000000006000205BE000004BE00E00F5000D0
:10145000E08F5800E00F5900E08F590000000600AF
:101460006000B8006011B80008045000898458007A
:101470000A0559008B8559001C002000E00F52001E
:10148000E08F5A00000006000800BE000A01BE00FE
:1014900000000600839F68000100E00002003D009C
:1014A00060001000E08018000300E00002003D0032
:1014B00060011100E08119009BFD07004F00E00072
:1014C00002003B0060001000E080180000000600F1
:1014D000889FBE008A9FBE00841F78001700070007
:1014E0004F00780011003300F0FF2F00838F6C0055
:1014F00006003B00040565000A00A700080037004D
:1015000009F0A6001000200008003700820F5400E8
:10151000838F5C00030039001000200001003E00B2
:101520000000200009F0A7000000EA004F05BE00FF
:101530004F04BE000000E000000006000004BE00F2
:101540003C0007000003BE000405BE000200BE0010
:1015500038000700844F7500000006000200BE003E
:101560006450E100050036006420E100020036000E
:101570000968A30001003A000800BE000160A00055
:101580004F0678004F05BE004F04BE000000060065
:10159000F0FF2F00F1FF2700F9FF37008100200046
:1015A000618055000B003D000B00200061FE2F0004
:1015B0000100E1001D0034008281710061016400BE
:1015C0008904D1000884D3000000E800FAFF3A0043
:1015D00071002000610064000300700002006000E0
:1015E0000900320061044400E0844C000988A50031
:1015F000050032008B05E8006808E10002003A00AF
:101600008904D1000884D300F20F20000258E100C1
:1016100005003D00C75DDD00F907B2008980750057
:1016200008007800000006000BF827008B00780007
:1016300000000500C70ADE00F107B200F50FB20096
:1016400008003200E1CF4200020032000170A00029
:1016500024000500810F700001003200040805001D
:1016600044000500810F700002003A0014000500DC
:101670008502E9000000400081C04800FCFF3B00FB
:101680000170A000240005008001EB00020037007B
:10169000817178008301E800828F5100FCFF3A00DD
:1016A000000006000C00FA00889FBE0000047800CD
:1016B000CFB09700F0FF2700D0BF9F008004EB0061
:1016C00099BF9F0088BF9F00A8BF9F00200C2000EB
:1016D000B0BF9F0078815700708057009C000700C2
:1016E0000FB89700094878000FB897000804500019
:1016F000080078004F04BE000080FA0000000600D9
:101700008001780000017800010037000201E80044
:101710001204E000FDFF3A003140780000597800E3
:101720000004E000FCFF3A0003007800000006001F
:10173000810178000002EB000B003700E4407800E4
:101740000104E000030032000402E80093CF5000DF
:10175000040032008180FB001380FB0000805000F9
:10176000000006008301E800820F5200F3FF3A00F8
:10177000000005000C00FA00A0BF9F00C0BF9F0042
:101780005D000700B0BF9F00F0BF9F00100C20005D
:10179000D0BF9F0074815700EFB097006C80570056
:1017A0004C0307000080FA000000060000037800E8
:1017B00080027800020278008001EB000800370008
:1017C0000402E90063C07800805A78008301E800D1
:1017D0000004E00002003A008000EB000600370041
:1017E000828F5100F6FF3A00FBFF37000040EB000C
:1017F00080F07A008100E800848F5000FBFF3A00FF
:1018000006007800000006000000FA00CFB897003C
:10181000688157004E0007000080FA0000000600B3
:10182000810178000000E9000081EB00E50F500025
:1018300004003E0080004000A0EF2000608178009E
:1018400003B0780002007800000006000001780074
:101850000000E900E50F50000F003E00800040004E
:10186000A0EF2000E08078000100E00002003A00D4
:101870001000200038040700E18F4000060032000D
:101880000000EB00E18F50000400320002007800FD
:1018900001000100000005000080EB0000000600D0
:1018A00010002000E9FF0700100020002A040700B4
:1018B0008002780080017800010037008301E80091
:1018C0001304E000FDFF3A000002EB00820F52001B
:1018D0000600320064C07800805978000402E800F5
:1018E0000004E00002003200F8FF37008049EB00FE
:1018F0000500780000000600800078003004E00059
:10190000FEFF3A00010050000000E9000000060060
:10191000800178000001780031407800005978009B
:101920000004E000FCFF3A0003007800000006001D
:1019300010417800814F5100040032000000E8009F
:101940000204E000FAFF3A000000EB00000006008D
:10195000FE874700889FBE008A9FBE008C9FBE0006
:101960008E1F7800F0B79F000107780082BF9F00AC
:101970000000EB00A0B79F009F0237008006EB003D
:1019800050C2B30080CF5000090032000100FB00BC
:10199000FFB09700F4030700E10F40009602320009
:1019A000AFB097008100E800A1B79F009202370016
:1019B0009E407800D0C2B30080CF50000C003200AF
:1019C00007003C006D40500080CF50000A003200FC
:1019D0006B40400080CF50000E003A0008003700F6
:1019E00000C3B30080CF50000A003A000600370061
:1019F0000D30A000050037000D00A00003003700E7
:101A00000D10A000010037000D20A0000E07E80017
:101A1000E7FF37000D18A300010032000D00A10000
:101A20000D38A300010032000D20A1000100FB00D1
:101A300002FD2F0002004000E90F50000E003E00A2
:101A40000002EB00C4B79F0082017800CFB297007C
:101A50006A28B9001E01FB0000014100030141009A
:101A6000C2B79F005E00FB0003004000E90F50007A
:101A70000B003E00F5FF37000006EB00CCB79F00DF
:101A8000A0C2B30080CF500005003A000FB8970005
:101A9000C000780080BF9F00C1B79F000E07E8001C
:101AA0000001EB00B2B79F00E0C2B3009E4F1000F0
:101AB00018003A000DE0A0008E00E80064405000DD
:101AC000914F100002003200010778000C0037002F
:101AD0000FBA9700C402780084BF9F00B5B79F007B
:101AE0000E87E8000B0037003FB697006A60B90028
:101AF0000000410003004000B0B79F000E07E8005F
:101B00001E01FB0003FD2F0003004100E90F500000
:101B1000F5FF3600BE407800E1D79F00C0C6B30095
:101B200080CF5000220032000F003C00694050007E
:101B300080CF50007700320004003C000104E00038
:101B4000310232006B4050000F00370040C6B30036
:101B500080CF5000930032006540400080CF50009D
:101B60008B003A008F00370030C7B30080CF5000A1
:101B70001A00320007003C006440500080CF500043
:101B8000110032000040E80080CF500080003A0091
:101B90000F00370050C7B30080CF500080003200E4
:101BA0006340400080CF500079003A0009003700C0
:101BB000000028000D48A30001003A0000012000A9
:101BC00080867600D3FF37000D60A00075003700D7
:101BD0000D50A0000D70A000720037008FB8970064
:101BE0004100780081BF9F00000478000000E00001
:101BF00001003A00A8EA20008004EB000100370051
:101C00008104E80089007800088044001004E000A6
:101C1000FBFF3A003FB197000200E00003003200F2
:101C2000890F510001003100820478000002EB00AE
:101C3000E4AF9F00CFB29700898F520002003600B8
:101C400009805200E0AF9F004368DE00E1066000BB
:101C50001B003A000D06780009003700FFB097001E
:101C60000002200040030700E10F400003003200A3
:101C70002FB097000000E800A0B79F000C06E80016
:101C8000EFA89700810F5600F4FF3A000081EB00A7
:101C9000E2AF9F000A003700880078003100FB00A7
:101CA00001047800FFB097002F030700E10F400008
:101CB000030032002FB297000402E800A4B79F008F
:101CC0000900E90080047800E10F4000F2FF3A00CB
:101CD0000006EB000D00E0000A003A00C6013700E4
:101CE000FFB09700000220001F030700E10F400033
:101CF00003003200AFB297008502E800A5B79F004D
:101D00000C06E8006FA89700800F5600F4FF3A0019
:101D1000B90137008FB897004100780081BF9F005C
:101D2000CF80DE0001017800820178000205BE004C
:101D30000004BE000203BE000002BE004822DE0016
:101D4000482EDD0004027600E4D79F000D48A30072
:101D50000A0032000404E00008003200E14F4200B3
:101D60000600320071FD2F00018047000448780012
:101D7000184098002900200002003700F0D79F008B
:101D80001900200072FD2F0002844700A1FF3700D8
:101D900064FD2F0004844700190020009DFF3700D8
:101DA0000D0CB3000D007800000CB20028003A00C2
:101DB0000D00E00005003D008FBA97004505BE000C
:101DC0004504BE0085BF9F00140037000D48A300E6
:101DD0000B0032000FBE97004C00BE008CBF9F006E
:101DE0004F89DE00CF91DE000002BE0002037800C2
:101DF000820378000605BE000404BE000700370019
:101E00008FB897004100780081BF9F0000047800E0
:101E1000CFC4DE00090578008A057800E00F540081
:101E2000E08F5C00E00F5D00E08F5D001F003D0073
:101E30003D00B3006000B8006011B8000804500015
:101E4000898458000A0559008B855900170037000E
:101E50000D00E00005003D000FB997004205BE00EF
:101E60004204BE0082BF9F00100037000D48A3004F
:101E7000070032000FBA97004400BE0084BF9F00E5
:101E80006011B8000205BE000004BE000700370064
:101E90008FBA97004500780085BF9F000004780046
:101EA000090020000A0020000B0020003FB6970028
:101EB0000C00E00007003A00E00F5400E08F5C00E7
:101EC000E00F5D00E08F5D0002003A00100020008E
:101ED000B0B79F008D007800010CB200E1B79F0001
:101EE00000042000808F50003000320003003C00CE
:101EF0000100E00008003200400037000008200028
:101F00006FB19700800F510014003200000C2000C8
:101F1000800F510039003A0014C0B300A5E0200042
:101F20000B0037000400FB004300DD00050040000B
:101F30005001BE004000BE000040E10001C8E100C9
:101F400002D0E10003D8E1002B0039000442E80090
:101F5000F44F5200F3FF3A00270037000001200041
:101F6000010020006011B80014C0B3000040E1007F
:101F700001C8E10002D0E10003D8E1001E003900F1
:101F8000450020000000D0008180D2000281D200F4
:101F90008381D2008502E900FAFF3A000442E8009A
:101FA000F04F5200F1FF3A0013003700800020008C
:101FB000010020006011B80014C0B3000040E1002F
:101FC00001C8E10002D0E10003D8E1000A003900B5
:101FD0003C0020000000D0008180D2000281D200AD
:101FE0008381D2000C06E900FAFF3A000442E800BF
:101FF000F54F5200F1FF3A00E4D79F00EFD0970071
:102000000100FB003FB19700820F500002003D002D
:10201000E2D79F00040037003FB29700800F5200C4
:1020200001003D00B0B79F00CFB297000500E0006F
:102030000400320063806600020032008502E9007D
:10204000C5B79F000DE8A3000B0032004FB6970004
:102050003FB09700800F560003003C008000EB006B
:10206000C1B79F00040037004FB197003FB29700FF
:1020700004015100C2B79F00EFD297000500FB009A
:102080000006EB00DCAF9F00CFB09700808F5000C0
:102090000200340000805000D0AF9F000D28A30044
:1020A00037003200E18066000D18A3000C003200FA
:1020B000D00220000100E00001003A000080E900A9
:1020C000FFB0970028020700E10F40000E00320029
:1020D0002FB197000201E800A2B79F000A00370065
:1020E0000100E00008003200FFB09700000220006D
:1020F0001D020700E10F4000030032002FB29700DD
:102100000402E800A4B79F00DFAA97000500E000E2
:102110000F0032000006EB00FFB097000003200024
:1021200011020700E10F4000030032002FB09700BA
:102130000000E800A0B79F000C06E800DFA89700A9
:10214000810F5600F4FF3A000001EB00D2AF9F0070
:102150003FB29700C320DD0020E0200080804000D7
:1021600091B79F004220DD006400500080B79F00BF
:102170006320B900F0AF9F00630650008400370071
:10218000DFAA97000500E0001100320068806600B9
:102190000F003A0000067800FFB097000002200010
:1021A000F1010700E10F4000030032002FB097005B
:1021B0000000E800A0B79F000C06E800DFA8970029
:1021C000810F5600F4FF3A000001EB00D2AF9F00F0
:1021D000E18066000D18A3000C003200D002200040
:1021E0000100E00001003A000080E900FFB0970024
:1021F000DD010700E10F4000D5FF32002FB297004C
:102200000402E800A4B79F00D1FF37000100E000FE
:10221000CFFF3200FFB0970000022000D20107007C
:10222000E10F4000CAFF3200AFB297008502E8001C
:10223000A5B79F00C6FF370000042000EFB097004D
:10224000808F50003100320003003C000100E000AC
:10225000080032003E003700000820006FB19700F0
:10226000800F510011003200000C2000800F51003F
:1022700037003A001FB097003002BE002003BE00B6
:102280000800BE000A01BE00F1FB0700A400200008
:10229000050020006033B800F4FB070004C3B3005E
:1022A00004424000E4D79F002900370015EB2000CE
:1022B000D5B79F000D58A30002003A0020EC200083
:1022C000D0B79F0014002000050020006033B80044
:1022D0008FB097008100E900050033000402D000B0
:1022E0008582D2000683D2008783D200F9FF3700AF
:1022F0000800BE000A01BE00D5FB07006F006000A9
:102300005FB1970062407800100037001400200091
:10231000050020006033B8000C0078000000E900E0
:10232000050033000402D0008582D2000683D2006B
:102330008783D200F9FF37000800BE000A01BE0003
:10234000C3FB0700674060000043B000E0D79F0078
:10235000EFD097000100FB00FFB09700820107005B
:10236000E10F4000030032002FB197000201E800A6
:10237000A2B79F001FB297006802520094B79F0057
:102380008FB29700E482520085B79F006306560023
:10239000D0FF2F003FB197000090B9007FAA9700AF
:1023A0000000420063005000800F5600A2FF3A0078
:1023B0000D38A30010003200DFAA97000500E000EE
:1023C0000D0034000006EB00FFB097000002200073
:1023D00065010700E10F4000030032002FB09700B5
:1023E0000000E800A0B79F000C06E800DFA89700F7
:1023F000810F5600F4FF3A00BE407800E1D79F00FD
:102400000104E0005DFD3A002FB097004F0778000F
:102410004F06BE004F05BE004F04BE00EF01B100E5
:1024200000000600889FBE00000478008144780008
:1024300000FD2F0000004400E90F500002003E00A4
:10244000000178000D00370008007800E2F807006E
:102450000000E0000300320008007800E4F8070004
:102460000004780008007800E8F807000000E000A9
:102470000700320090FA2F00000144000980FB00A1
:10248000800F510002003D000280FB000100370078
:10249000F00F20004F04BE0000000600881F7800E7
:1024A000607880007701070000047800E1F80700F9
:1024B0000000E000FAFF3A00E10F440003003200A0
:1024C0006178800008007800A20107004F047800BE
:1024D00000000600EC874700889FBE008A9FBE0070
:1024E0008C9FBE008E1F780081BF9F00020778007E
:1024F000607888008046EB00040137008884FB0088
:1025000009007800CBF80700800078000000E000A8
:1025100002003200E1FF0700FC00370050C2B300A8
:10252000804F5400F0003A000FBD970020C0B30068
:10253000C0EF9F00D1EF9F0081EF9F0003003700A5
:1025400040C0B300C0EF9F000FBD97000FB99700C8
:10255000B240780082BF9F008184FB0090C6B30028
:1025600080CF50003500320017003E00664050001A
:1025700080CF5000620032000C003E0077405000D7
:1025800080CF50002800320006003E000104E00029
:102590009B003200A0C2B30080CF50006E003A0012
:1025A0001D00370080C5B3001600370040C6B300D9
:1025B00080CF5000210032006440400080CF5000A6
:1025C00065003A001200370030C7B30080CF5000DA
:1025D0001E00320007003E006740500080CF5000D0
:1025E000110032006340400080CF50005A003A0092
:1025F0001400370050C7B30080CF50000F003200E6
:102600006340400080CF500053003A00650037001F
:1026100020C0B300CBFF3700DFE897008140E8001F
:10262000D1EF9F00C8FF37004FE9970080C0B3008B
:10263000E24F5100C3FF3A00C1FF3700ACC0B30006
:10264000590037008CC0B3005700370093FF0700D4
:10265000DFE897000104E00002003A004E01780034
:10266000D2B79F0060788000060107000004780060
:10267000E10F4000A20032008FEC970012003700FB
:102680000A85E8008ABF9F00160037008FB89700C0
:102690001100FB00800F5400F9FF32005FE9970042
:1026A0000204E00003003A005FB097000858780089
:1026B000D0B79F008944E9000A00320060788000AA
:1026C000F0000700000478000800E800E10F500067
:1026D000040036000800780056F807000000E0000B
:1026E000EAFF3200DFE897000104E00087003A00CB
:1026F0008D46E8005FB197000149780083003700FC
:102700005FE897000004E00003003A008D46E8000F
:10271000CE007800D1B79F0060788000D900070014
:10272000E10F4000760032005FE997000204E0000C
:1027300003003A00DFB0970080587800D1B79F00BF
:102740000FE997000241E90082EF9F004240A90093
:102750006E003400F0FF37000180FB0008FD2F0001
:1027600008004000E90F50005F003E000A007800BA
:102770001501070080EF9F008800780003003700F4
:102780000FB897000000E80080BF9F000FB99700C6
:102790001200FB0001004000E90F5000F8FF360076
:1027A00069FF37000CC1B3003CFF07006078800070
:1027B000B4000700000578000040EB00E0EF9F0048
:1027C000D0022000800F550005003A00607880009C
:1027D000AC0007000005780011C0B300E1EF9F00D6
:1027E0008C4078000A0078000EFF0700E14F40009F
:1027F0000A003A00617880000A007800D5000700DE
:102800000D04E0004B003A0060788000300090003A
:102810000048A30043003200480037008FED9700C6
:102820006044B8000C81FB00030020000800BE00DB
:10283000B7F807000004BE008C4078000A0078005A
:10284000F8FE07000080FB000100200008044000A3
:10285000898448008B45E9000700320060788000D9
:1028600088000700000578008C407800EDFE070026
:10287000E14F4000EBFF3A008C4078000A007800FE
:10288000E8FE0700E14F400003003A006178800055
:102890000A007800AF0007006FE997000204E0002B
:1028A0000200320060041400E0841C005FE897001E
:1028B0000004E00015003A008D46E800CFE89700DC
:1028C000E4CF500003003A004E0078000888BE00B4
:1028D0000E0037000E81E900020778001200780030
:1028E000080878000900370060788000650007005C
:1028F000808F540005003200E10F40000B003A00C9
:102900000D04E0000D0032000A0037008FB8970078
:102910003144780081BF9F000804E000F7FE3A00D0
:10292000040037000000EB000500370061788000EC
:10293000880007000D80FB00010037000080EB00DD
:102940004F0778004F06BE004F05BE004F04BE0083
:10295000CF00B1000000060000047800BE000700B0
:1029600008007800BBF70700889FBE0000017800D0
:1029700001047800B10090000118A3003D0032006E
:102980000198A30003003A00180090000000E00046
:1029900038003A000190A0003104980082047800C9
:1029A000F90FB200180090000000E00002003A00A9
:1029B00028009000000C7800EA8F540006003A00CE
:1029C000380090000078A30003003A0088007800E7
:1029D000D0002000E4FF070098009000580090000D
:1029E000808F50000B0032000100E80010049800B6
:1029F0001800780009587800000C780011C0B30066
:102A0000A0F0200001487800EA8F54000600320050
:102A10001900370088007800094078009C00070002
:102A20008004780014003700380090000088A3006C
:102A30001100320018019000A8009000480090009A
:102A40008CF7070098009000810F500004003200BE
:102A5000380090000003B300300498008084EB003D
:102A60000000EB001004980028009000000C780093
:102A7000010037008084EB00090078004F04BE009D
:102A800000000600881F780000047800B000900065
:102A90000148A30007003A000108A3000500320026
:102AA0000198A30008003200100090000000E00030
:102AB00005003200380090000040A000300498006B
:102AC0008080EB00200037000190A10031049800C5
:102AD000180090000000E000060034000000E9004B
:102AE0001004980018007800B080FB00000C7800FB
:102AF00006003700380090000068A300EDFF3A00A0
:102B000008007800A50007008000780038009000D9
:102B10000078A3000C003A00FA8F500008003A0039
:102B2000280090000000E000E2FF32001800900052
:102B30000000E80010049800180CE900DDFF3700E1
:102B4000ED8F5000E2FF3200010078004F04780062
:102B50000000060080017800E10F400017003200FD
:102B6000310090000008A300140032000098A30078
:102B700012003A00210290000400E0000F00320031
:102B80001101900051009000800F51000B003200A5
:102B900011007800840F500002003A008008E8001D
:102BA000020037000200E800900098001100E900E0
:102BB0008008780003487800010037008081EB002E
:102BC00003007800000006000001780000C2B30096
:102BD000010037000201E8009240780080CF5000E9
:102BE000FCFF3200E9CF5000FAFF3200D0C2B30040
:102BF00080CF500003003A000201E80014C0B30087
:102C0000050037000042EB00B0C2B30080CF500097
:102C100001003A000201E8008000EB0005FD2F00F2
:102C2000040037006A08B9000080410085004000B8
:102C30000201E8009201FB0005804100E90F50000D
:102C4000F8FF36000404E000010032008100EA00D1
:102C50000100780000000600881F7800707880006E
:102C60000000E000010032000000010068ED2000DB
:102C700008007800970007006C044400A0EF2000D3
:102C8000800F5400FAFF3A004F047800000006005D
:102C90000200FA00889FBE00A0FF9F000104780098
:102CA000B1009000810478000904B20002003200F3
:102CB0000000FB00360037000118A30005003A00B1
:102CC0000103B30031049800190498000080EB0060
:102CD0002F003700580090000000E00006003A0086
:102CE0004800900012002000E6805700E1F607003F
:102CF0001904980024003700280090000000E0002C
:102D000008003A0060F0200020049800000C7800D1
:102D10002000200050049800100498000130A0000A
:102D20003104980018019000A8009000480090001D
:102D3000D0F6070028009000000C78000080EB001F
:102D40001004980018007800AFF897000158780038
:102D5000000C78002FF89700EA4F50000A003A0064
:102D6000380090000088A30007003200180190008E
:102D7000A800900048009000BEF6070019049800D3
:102D8000A8009000010C7800AFF897000100FB004C
:102D90004F04BE000080FA00000006000200FA00A6
:102DA000889FBE008A1F7800000478000000EB00B6
:102DB00010049800380090008080EB000008A30009
:102DC0003F003200A0F020001004E00010003200AC
:102DD00069ED2000CAED20001A0078006C0545005E
:102DE0002010B20021102000810F500002003A0094
:102DF000090078006F000700EC844400A0EF200079
:102E0000808F5400F4FF3A00A0F020000048EB004F
:102E100048009000580190000200E0000D003A00C8
:102E20001204980012002000E8805700C8F607003E
:102E3000E10F500003003A000FF897008080FB007C
:102E40001F003700380090000040A00030049800B8
:102E500012003700A8009000BDF60700100498008B
:102E60000000E00003003200E10F40000D003A00D6
:102E700003003700380090000040A0000200370037
:102E8000380090000003B30030049800A8009000C0
:102E9000010C78000000EB00100498008080EB002B
:102EA00007003700A8009000010C78000000E9003E
:102EB0001004980001007800B080FB00000C78003E
:102EC000010078004F0578004F04BE000080FA0032
:102ED00000000600889FBE008A1F7800000478006A
:102EE0003000900063006000240032000800780089
:102EF000300007003805900080EF2F0000006500CB
:102F000030049800280090000000E0000400320027
:102F1000E804650002003A005F00070029049800F9
:102F200048009000C3F60700E10F40001300320094
:102F3000B80090000102B20010003A000AC8A300D5
:102F400018003200907880000000E0001500320088
:102F50000001780081047800012A200012289000E6
:102F6000880F5000070032004205B0004905B0004C
:102F7000818F54000B003200F8FF37000080EB0017
:102F80000900370002007800B3F60700907880004F
:102F9000090040008000EB00112898000100780033
:102FA000010037000000EB004F0578004F04BE0021
:102FB00000000600881F78000004780030009000B0
:102FC0000008A30007003200800078000120B20052
:102FD00004003A0011049800A8009000010C780049
:102FE000170037000018A300190032000098A30052
:102FF00017003200A80090000100E0001400320029
:10300000180190000200E00011003200480090001A
:1030100018F6070098009000810F5000030032005E
:10302000380090000003B300300498000000EB006B
:103030001004980028009000000C780038009000E0
:103040000058A300020032000080EB0001003700AE
:103050000000EB004F04780000000600817880003B
:103060000100E00003003200110078008078880041
:10307000030037002000200080F607008000780061
:10308000E18F400002003A00906E2600A078880090
:1030900001007800000006008178800001087800B7
:0830A0008078880000000600A2
:020000040000FA
:0200000401F009
:04000C00FBFF0000F6
:020000040000FA
:0200000401F009
:04001000FDFF0000F0
:020000040000FA
:0200000401F009
:040014007FFF00006A
:020000040000FA
:10000800E8030000E8030000AC710000B2710000D2
:10001800E8030000E8030000E8030000E80300002C
:10002800E80300000A660000E8030000E677000025
:10003800E8030000E8030000E8030000E80300000C
:10004800E8030000E8030000E80300000A76000067
:10005800E8030000E8030000E8030000E8030000EC
:10006800E8030000E8030000E8030000E8030000DC
:10007800E8030000E8030000E8030000E8030000CC
:10008800E8030000E8030000E8030000F668000049
:10009800AC690000E8030000E8030000E803000082
:1000A800E8030000E8030000E8030000E80300009C
:1000B800E8030000E8030000E8030000E80300008C
:1000C800E8030000E8030000E8030000E80300007C
:1000D800E8030000E8030000E8030000E80300006C
:1000E800E8030000E8030000E8030000E80300005C
:1000F800E8030000E8030000E8030000E80300004C
:10010800E8030000E8030000E8030000E80300003B
:10011800E8030000E8030000E8030000E80300002B
:10012800E8030000E8030000E8030000E80300001B
:10013800E8030000E8030000E8030000E80300000B
:10014800E8030000E8030000E8030000E8030000FB
:10015800E8030000E8030000E8030000E8030000EB
:10016800E8030000E8030000E8030000E8030000DB
:10017800E8030000E8030000E8030000E8030000CB
:10018800E8030000E8030000E8030000E8030000BB
:10019800E8030000E8030000E8030000E8030000AB
:1001A800E8030000E8030000E8030000E80300009B
:1001B800E8030000E8030000E8030000E80300008B
:1001C800E8030000E8030000E8030000E80300007B
:1001D800E8030000E8030000E8030000E80300006B
:1001E800E8030000E8030000E8030000E80300005B
:0801F800E8030000E803000029
:020000040000FA
:10020800E8030000E8030000AC710000B2710000D0
:10021800E8030000E8030000E8030000E80300002A
:10022800E80300000A660000E8030000E677000023
:10023800E8030000E8030000E8030000E80300000A
:10024800E8030000E8030000E80300000A76000065
:10025800E8030000E8030000E8030000E8030000EA
:10026800E8030000E8030000E8030000E8030000DA
:10027800E8030000E8030000E8030000E8030000CA
:10028800E8030000E8030000E8030000F668000047
:10029800AC690000E8030000E8030000E803000080
:1002A800E8030000E8030000E8030000E80300009A
:1002B800E8030000E8030000E8030000E80300008A
:1002C800E8030000E8030000E8030000E80300007A
:1002D800E8030000E8030000E8030000E80300006A
:1002E800E8030000E8030000E8030000E80300005A
:1002F800E8030000E8030000E8030000E80300004A
:10030800E8030000E8030000E8030000E803000039
:10031800E8030000E8030000E8030000E803000029
:10032800E8030000E8030000E8030000E803000019
:10033800E8030000E8030000E8030000E803000009
:10034800E8030000E8030000E8030000E8030000F9
:10035800E8030000E8030000E8030000E8030000E9
:10036800E8030000E8030000E8030000E8030000D9
:10037800E8030000E8030000E8030000E8030000C9
:10038800E8030000E8030000E8030000E8030000B9
:10039800E8030000E8030000E8030000E8030000A9
:1003A800E8030000E8030000E8030000E803000099
:1003B800E8030000E8030000E8030000E803000089
:1003C800E8030000E8030000E8030000E803000079
:1003D800E8030000E8030000E8030000E803000069
:1003E800E8030000E8030000E8030000E803000059
:0803F800E8030000E803000027
:020000040000FA
:1030A800705F000061700000705F0000636F0000D7
:1030B8006E66000069670000006F00006E65000022
:1030C8006C7900006E7800002F73000072630000B6
:1030D8002F480000756200002E63000000250000E4
:1030E800733A0000256900002025000073200000C5
:1030F8002D2D000020610000737300006572000030
:10310800746900006F6E00002066000061690000AD
:103118006C650000640A0000000000000000000068
:103128000000000000000000000000000000000097
:103138000000000000000000000000000000000087
:103148000000000000000000000000000000000077
:103158000000000000000000000000000000000067
:103168000000000000000000000000000000000057
:103178000000000000000000000000000000000047
:103188000000000000000000000000000000000037
:103198000000000000000000000000000000000027
:1031A8000000000000000000000000000000000017
:1031B8000000000000000000000000000000000007
:1031C80000000000000000000000000000000000F7
:1031D80000000000000000000000000000000000E7
:1031E80000000000000000000000000000000000D7
:1031F80000000000000000000000000000000000C7
:1032080000000000000000000000000000000000B6
:1032180000000000000000000000000000000000A6
:103228000000000000000000000000000000000096
:103238000000000000000000000000000000000086
:103248000000000000000000000000000000000076
:103258000000000000000000000000000000000066
:103268000000000000000000000000000000000056
:103278000000000000000000000000000000000046
:103288000000000000000000000000000000000036
:103298000000000000000000000000000000000026
:1032A80000000000000000000048000075620000F7
:1032B8002046000056650000722000003D200000F6
:1032C800257500002E250000752E000025750000CC
:1032D800005300006C65000065700000696E000016
:1032E800672000003D200000257500000057000001
:1032F8006972000065640000204900005020000049
:103308003D200000256400002E250000642E0000EA
:10331800256400002E2500006400000044480000D9
:1033280043500000697300004F6E0000203D00000C
:1033380020250000750000005746000020410000CD
:103348007463000068640000203D00002025000030
:103358007500000057460000204300006F6E000013
:103368006E200000203D00002025000075000000B0
:1033780057460000204600005665000072200000F5
:10338800203D000020250000642E00002564000078
:103398002E2500006400000057460000204600006B
:1033A800562000004F4B0000203D00002025000063
:1033B80075000000574600002053000053490000E4
:1033C80044200000203D000020250000730000007C
:1033D800574600002049000050200000202000002F
:1033E800203D000020250000642E00002564000018
:1033F8002E250000642E0000256400000057000000
:103408004620000053650000634D00006420000062
:103418003D20000025630000005700004620000002
:1034280057650000704B0000492000003D20000057
:1034380025640000004500004E4400000000000024
:103448000000000000000000000000000000000074
:103458000000000000000000000000000000000064
:103468000000000000000000000000000000000054
:103478000000000000000000000000000000000044
:103488000000000000000000000000000000000034
:103498000000000000000000000000000000000024
:1034A8000000000000000000000000000000000014
:1034B8000000000000000000000000000000000004
:1034C80000000000000000000000000000000000F4
:1034D80000000000000000000000000000000000E4
:1034E80000000000000000000000000000000000D4
:1034F80000000000000000000000000000000000C4
:1035080000000000000000000000000000000000B3
:1035180000000000000000000000000000000000A3
:103528000000000000000000000000000000000093
:103538000000000000000000000000000000000083
:103548000000000000000000000000000000000073
:103558000000000000000000000000000000000063
:103568000000000000000000000000000000000053
:103578000000000000000000000000000000000043
:103588000000000000000000000000000000000033
:103598000000000000000000000000000000000023
:1035A8000000000000000000000000000000000013
:1035B8000000000000000000000000000000000003
:1035C80000000000000000000000000000460000AD
:1035D800697200006D7700006172000065200000CC
:1035E8003D200000257500002E250000752E0000E6
:1035F80025750000004C00004544000042720000A0
:1036080069740000652000003D2000002575000059
:1036180000480000616E00006443000074720000FE
:103628006C2000003D2000003000000057690000B9
:1036380046690000204D00006F640000203D000036
:10364800202500006400000057690000466900005A
:10365800436F00006E6E0000203D00002025000032
:1036680064000000576900004669000046560000E3
:103678004F6B0000203D0000202500006400000082
:103688005769000046690000465600006572000050
:10369800203D000020250000752E00002575000043
:1036A8002E250000750000005769000046690000DB
:1036B8005353000049440000203D0000202500002D
:1036C800730000005769000046690000416400006B
:1036D80064720000203D000020250000642E0000D8
:1036E800256400002E250000642E000025640000DB
:1036F8000057000069460000695300006563000038
:103708004D2000003D200000256300000057000008
:103718006946000069530000656300004B20000003
:103728003D2000002573000000000000000000009C
:103738000000000000000000000000000000000081
:103748000000000000000000000000000000000071
:103758000000000000000000000000000000000061
:103768000000000000000000000000000000000051
:103778000000000000000000000000000000000041
:103788000000000000000000000000000000000031
:103798000000000000000000000000000000000021
:1037A8000000000000000000000000000000000011
:1037B8000000000000000000000000000000000001
:1037C80000000000000000000000000000000000F1
:1037D80000000000000000000000000000000000E1
:1037E80000000000000000000000000000000000D1
:1037F80000000000000000000000000000000000C1
:1038080000000000000000000000000000000000B0
:1038180000000000000000000000000000000000A0
:103828000000000000000000000000000000000090
:103838000000000000000000000000000000000080
:103848000000000000000000000000000000000070
:103858000000000000000000000000000000000060
:103868000000000000000000000000000000000050
:103878000000000000000000000000000000000040
:103888000000000000000000000000000000000030
:103898000000000000000000000000000000000020
:1038A8000000000000000000000000000000000010
:1038B80000000000000000000053000063610000E9
:1038C8006E20000020490000442000003D20000038
:1038D800256400000053000043200000496E0000EA
:1038E80064650000782000003D2000002564000089
:1038F800004E000065740000436F0000756E000004
:10390800742000003D2000002564000000530000E2
:10391800636100006E53000053490000442000001A
:103928003D2000002573000000530000656300007F
:10393800204D00006F640000652000003D2000005D
:1039480025640000004E000065740000205400004B
:1039580079700000652000003D200000256400000B
:103968000053000069670000202000005374000025
:10397800722000003D20000025640000004C00007B
:103988006F610000644400006F6E00006520000055
:103998003D20000025640000000000000000000039
:1039A800000000000000000000000000000000000F
:1039B80000000000000000000000000000000000FF
:1039C80000000000000000000000000000000000EF
:1039D80000000000000000000000000000000000DF
:1039E80000000000000000000000000000000000CF
:1039F80000000000000000000000000000000000BF
:103A080000000000000000000000000000000000AE
:103A1800000000000000000000000000000000009E
:103A2800000000000000000000000000000000008E
:103A3800000000000000000000000000000000007E
:103A4800000000000000000000000000000000006E
:103A5800000000000000000000000000000000005E
:103A6800000000000000000000000000000000004E
:103A7800000000000000000000000000000000003E
:103A8800000000000000000000000000000000002E
:103A9800000000000000000000000000000000001E
:103AA800000000000000000000000000000000000E
:103AB80000000000000000000000000000000000FE
:103AC80000000000000000000000000000000000EE
:103AD80000000000000000000000000000000000DE
:103AE80000000000000000000000000000000000CE
:103AF80000000000000000000000000000000000BE
:103B080000000000000000000000000000000000AD
:103B1800000000000000000000000000000000009D
:103B2800000000000000000000000000000000008D
:103B3800000000000000000000000000000000007D
:103B4800000000000000000000000000000000006D
:103B58000043000075720000722E0000204900002A
:103B6800502000003D200000256400002E250000A4
:103B7800642E0000256400002E250000640000006B
:103B880043750000722000004D610000736B000057
:103B9800203D000020250000642E00002564000060
:103BA8002E250000642E0000256400000047000058
:103BB8006174000065770000617900002020000032
:103BC8003D200000256400002E250000642E000022
:103BD800256400002E2500006400000050720000DB
:103BE800692E0000204400004E530000203D0000D4
:103BF80020250000642E0000256400002E2500000A
:103C0800642E000025640000005300006563000076
:103C18002E200000444E0000532000003D200000EC
:103C2800256400002E250000642E00002564000095
:103C38002E2500006400000044650000662E000088
:103C48002049000050200000203D000020250000F1
:103C5800642E0000256400002E250000642E00005C
:103C68002564000000440000656600002E4D000039
:103C7800617300006B2000003D20000025640000F7
:103C88002E250000642E0000256400002E2500006B
:103C98006400000044480000435000002020000059
:103CA8004F6E0000203D0000202500006400000049
:103CB8004E65000074420000494F00005320000088
:103CC800203D000020250000730000004D41000049
:103CD800432000004164000064720000203D0000A1
:103CE8002025000073000000000000000000000014
:103CF80000000000000000000000000000000000BC
:103D080000000000000000000000000000000000AB
:103D1800000000000000000000000000000000009B
:103D2800000000000000000000000000000000008B
:103D3800000000000000000000000000000000007B
:103D4800000000000000000000000000000000006B
:103D5800000000000000000000000000000000005B
:103D6800000000000000000000000000000000004B
:103D7800000000000000000000000000000000003B
:103D8800000000000000000000000000000000002B
:103D9800000000000000000000000000000000001B
:103DA800000000000000000000000000000000000B
:103DB80000000000000000000000000000000000FB
:103DC80000000000000000000000000000000000EB
:103DD80000000000000000000000000000000000DB
:103DE80000000000000000000000000000000000CB
:103DF80000000000000000000000000000000000BB
:103E080000000000000000000000000000000000AA
:103E1800000000000000000000000000000000009A
:103E2800000000000000000000000000000000008A
:103E3800000000000000000000000000000000007A
:103E4800000000000000000000000000000000006A
:103E5800000000000000000000000000000000005A
:103E6800000000000000000000000000000000004A
:103E7800000000000000000000000000000000003A
:103E8800000000000000000000000000000000002A
:103E9800000000000000000000000000000000001A
:103EA8005749000046490000204900005020000002
:103EB800494E0000464F0000004300006F6E0000AE
:103EC80066690000672000004D2000003D200000CA
:103ED8002564000000000000000000000000000051
:103EE80000000000000000000000000000000000CA
:103EF80000000000000000000000000000000000BA
:103F080000000000000000000000000000000000A9
:103F18000000000000000000000000000000000099
:103F28000000000000000000000000000000000089
:103F38000000000000000000000000000000000079
:103F48000000000000000000000000000000000069
:103F58000000000000000000000000000000000059
:103F68000000000000000000000000000000000049
:103F78000000000000000000000000000000000039
:103F88000000000000000000000000000000000029
:103F98000000000000000000000000000000000019
:103FA8000000000000000000000000000000000009
:103FB80000000000000000000000000000000000F9
:103FC80000000000000000000000000000000000E9
:103FD80000000000000000000000000000000000D9
:103FE80000000000000000000000000000000000C9
:103FF80000000000000000000000000000000000B9
:1040080000000000000000000000000000000000A8
:104018000000000000000000000000000000000098
:104028000000000000000000000000000000000088
:104038000000000000000000000000000000000078
:104048000000000000000000000000000000000068
:104058000000000000000000000000000000000058
:1040680000000000004E00006577000020480000B6
:104078007562000020490000502000003D2000002B
:10408800256400002E250000642E00002564000031
:104098002E250000640000004E6500007720000017
:1040A80048750000622000004D610000736B00003D
:1040B800203D000020250000642E0000256400003B
:1040C8002E250000642E000025640000004E00002C
:1040D8006577000020480000756200002047000056
:1040E800572000003D200000256400002E25000018
:1040F800642E0000256400002E25000064000000E6
:104108004E6500007720000048750000622000001E
:104118004448000043500000203D000020250000D6
:10412800640000004E650000772000005769000019
:104138004669000020490000502000003D20000092
:10414800256400002E250000642E00002564000070
:104158002E250000640000004E6500007720000056
:104168005769000046690000204D00006173000097
:104178006B2000003D200000256400002E25000073
:10418800642E0000256400002E2500006400000055
:104198004E6500007720000057690000466900005E
:1041A80020470000572000003D2000002564000043
:1041B8002E250000642E0000256400002E25000036
:1041C800640000004E650000772000005769000079
:1041D80046690000204400004843000050200000C9
:1041E8003D200000256400000000000000000000E1
:1041F80000000000000000000000000000000000B7
:1042080000000000000000000000000000000000A6
:104218000000000000000000000000000000000096
:104228000000000000000000000000000000000086
:104238000000000000000000000000000000000076
:104248000000000000000000000000000000000066
:104258000000000000000000000000000000000056
:104268000000000000000000000000000000000046
:104278000000000000000000000000000000000036
:104288000000000000000000000000000000000026
:104298000000000000000000000000000000000016
:1042A8000000000000000000000000000000000006
:1042B80000000000000000000000000000000000F6
:1042C80000000000000000000000000000000000E6
:1042D80000000000000000000000000000000000D6
:1042E80000000000000000000000000000000000C6
:1042F80000000000000000000000000000000000B6
:1043080000000000000000000000000000000000A5
:104318000000000000000000000000000000000095
:104328000000000000000000000000000000000085
:104338000000000000000000000000000000000075
:104348000000000000000000000000000000000065
:104358000000000000000000000000000000000055
:104368000000000000000000000000000000000045
:104378000000000000000000004C0000534900004D
:10438800004200006F6100007264000020490000D4
:10439800442000003D20000025730000004D00006F
:1043A800616900006E20000046570000562000009A
:1043B8003D200000257500002E250000752E000008
:1043C80025750000004F00006E6500004C79000064
:1043D8006E780000202000003D20000025750000B8
:1043E8002E250000752E00002575000000570000DE
:1043F800694600006920000046570000562000006A
:104408003D200000257500002E250000752E0000B7
:104418002575000000480000616E0000642000005F
:1044280046570000562000003D200000257500007A
:104438002E250000752E000025750000005700008D
:10444800656200002046000057560000202000004A
:104458003D200000257500002E250000752E000067
:1044680025750000004100006C70000061630000C9
:1044780061200000562000003D2000002575000046
:104488002E250000752E0000257500000042000052
:104498006F61000072640000205600005220000086
:1044A8003D2000002575000000000000000000000D
:1044B80000000000000000000000000000000000F4
:1044C80000000000000000000000000000000000E4
:1044D80000000000000000000000000000000000D4
:1044E80000000000000000000000000000000000C4
:1044F80000000000000000000000000000000000B4
:1045080000000000000000000000000000000000A3
:104518000000000000000000000000000000000093
:104528000000000000000000000000000000000083
:104538000000000000000000000000000000000073
:104548000000000000000000000000000000000063
:104558000000000000000000000000000000000053
:104568000000000000000000000000000000000043
:104578000000000000000000000000000000000033
:104588000000000000000000000000000000000023
:104598000000000000000000000000000000000013
:1045A8000000000000000000000000000000000003
:1045B80000000000000000000000000000000000F3
:1045C80000000000000000000000000000000000E3
:1045D80000000000000000000000000000000000D3
:1045E80000000000000000000000000000000000C3
:1045F80000000000000000000000000000000000B3
:1046080000000000000000000000000000000000A2
:104618000000000000000000000000000000000092
:104628000000000000000000000000000000000082
:104638000000000000000000000000000000000072
:1046480000000000000000000000000053540000BB
:104658004154000055530000257500000054000027
:10466800656D00007028000043290000202000002C
:104678003D20000025730000004E0000500000009F
:104688004375000072720000205000006F73000034
:10469800203D0000202500006C750000005400003B
:1046A8006172000067200000506F00007320000056
:1046B8003D200000256C00007500000049730000D3
:1046C8004D6F0000766900006E670000203D000015
:1046D800202500007500000049730000486F0000A5
:1046E8006D6900006E670000203D00002025000075
:1046F8007500000049730000486F00006D650000F8
:1047080064200000203D0000202500007500000006
:1047180046460000446500007465000063740000AC
:10472800203D00002025000075000000546D0000A9
:1047380070500000726F000062650000203D0000AC
:104748002025000075000000526500006D6F000014
:1047580074650000494F0000203D0000202500003E
:1047680075000000486E00006420000043740000DB
:104778006C720000203D000020250000750000003C
:104788005265000076650000727300006520000025
:10479800203D00002025000075000000454E000067
:1047A80044000000000000000000000000000000BD
:1047B80000000000000000000000000000000000F1
:1047C80000000000000000000000000000000000E1
:1047D80000000000000000000000000000000000D1
:1047E80000000000000000000000000000000000C1
:1047F80000000000000000000000000000000000B1
:1048080000000000000000000000000000000000A0
:104818000000000000000000000000000000000090
:104828000000000000000000000000000000000080
:104838000000000000000000000000000000000070
:104848000000000000000000000000000000000060
:104858000000000000000000000000000000000050
:104868000000000000000000000000000000000040
:104878000000000000000000000000000000000030
:104888000000000000000000000000000000000020
:104898000000000000000000000000000000000010
:1048A8000000000000000000000000000000000000
:1048B80000000000000000000000000000000000F0
:1048C80000000000000000000000000000000000E0
:1048D80000000000000000000000000000000000D0
:1048E80000000000000000000000000000000000C0
:1048F80000000000000000000000000000000000B0
:10490800000000000000000000000000000000009F
:10491800000000000000000000000000000000008F
:10492800000000000000000000000000000000007F
:1049380000000000434F00004E46000049470000B9
:1049480025750000004E0000696300006B6E0000D2
:10495800616D0000652000003D2000002573000007
:10496800004D000061780000205000006F730000C7
:10497800202000003D200000256C0000750000008C
:104988004465000076200000547900007020000083
:10499800203D000020250000632500006300000082
:1049A800544300006F6D0000702000004F4E00005F
:1049B800203D000020250000317500000054000053
:1049C800656D0000704300006F2000002563000043
:1049D800203D000020250000640000005443000032
:1049E800204D00006F64000065200000203D00009D
:1049F8002025000063000000424C00004320000016
:104A0800456E000020200000203D00002025000009
:104A180075000000424C0000432000005374000061
:104A280070730000203D0000202500007500000084
:104A38004C45000044200000427200007420000031
:104A4800203D0000202500007500000054430000B0
:104A5800405300007461000072740000203D0000A3
:104A68002025000075000000484F00006E5300002C
:104A78007461000072740000203D000020250000D1
:104A880075000000000000000000000000000000A9
:104A9800000000000000000000000000000000000E
:104AA80000000000000000000000000000000000FE
:104AB80000000000000000000000000000000000EE
:104AC80000000000000000000000000000000000DE
:104AD80000000000000000000000000000000000CE
:104AE80000000000000000000000000000000000BE
:104AF80000000000000000000000000000000000AE
:104B0800000000000000000000000000000000009D
:104B1800000000000000000000000000000000008D
:104B2800000000000000000000000000000000007D
:104B3800000000000000000000000000000000006D
:104B4800000000000000000000000000000000005D
:104B5800000000000000000000000000000000004D
:104B6800000000000000000000000000000000003D
:104B7800000000000000000000000000000000002D
:104B8800000000000000000000000000000000001D
:104B9800000000000000000000000000000000000D
:104BA80000000000000000000000000000000000FD
:104BB80000000000000000000000000000000000ED
:104BC80000000000000000000000000000000000DD
:104BD80000000000000000000000000000000000CD
:104BE80000000000000000000000000000000000BD
:104BF80000000000000000000000000000000000AD
:104C0800000000000000000000000000000000009C
:104C180000000000544500004D50000020430000F3
:104C28004F4D00005025000075000000544300005F
:104C38006F6D0000702000004F4E0000203D000006
:104C48002025000075000000546500006D7000000C
:104C5800496E000020250000632000003D20000070
:104C6800256C0000640000005374000065700000AB
:104C7800536900007A650000203D000020250000EF
:104C880064000000000000000000000000000000B8
:104C9800000000000000000000000000000000000C
:104CA80000000000000000000000000000000000FC
:104CB80000000000000000000000000000000000EC
:104CC80000000000000000000000000000000000DC
:104CD80000000000000000000000000000000000CC
:104CE80000000000000000000000000000000000BC
:104CF80000000000000000000000000000000000AC
:104D0800000000000000000000000000000000009B
:104D1800000000000000000000000000000000008B
:104D2800000000000000000000000000000000007B
:104D3800000000000000000000000000000000006B
:104D4800000000000000000000000000000000005B
:104D5800000000000000000000000000000000004B
:104D6800000000000000000000000000000000003B
:104D7800000000000000000000000000000000002B
:104D8800000000000000000000000000000000001B
:104D9800000000000000000000000000000000000B
:104DA80000000000000000000000000000000000FB
:104DB80000000000000000000000000000000000EB
:104DC80000000000000000000000000000000000DB
:104DD80000000000000000000000000000000000CB
:104DE80000000000000000000000000000000000BB
:104DF80000000000000000000000000000000000AB
:104E0800000000000000000000000000000000009A
:104E1800000000007B22000064650000767300003B
:104E2800223A00005B200000225A00005A220000AB
:104E38002C200000224F0000412200002C200000FE
:104E4800224F0000422200005D7D00000044000067
:104E5800657600006963000065730000203D00006E
:104E68002025000073000000256C00007800000079
:104E7800000000000000000000000000000000002A
:104E8800000000000000000000000000000000001A
:104E9800000000000000000000000000000000000A
:104EA80000000000000000000000000000000000FA
:104EB80000000000000000000000000000000000EA
:104EC80000000000000000000000000000000000DA
:104ED80000000000000000000000000000000000CA
:104EE80000000000000000000000000000000000BA
:104EF80000000000000000000000000000000000AA
:104F08000000000000000000000000000000000099
:104F18000000000000000000000000000000000089
:104F28000000000000000000000000000000000079
:104F38000000000000000000000000000000000069
:104F48000000000000000000000000000000000059
:104F58000000000000000000000000000000000049
:104F68000000000000000000000000000000000039
:104F78000000000000000000000000000000000029
:104F88000000000000000000000000000000000019
:104F98000000000000000000000000000000000009
:104FA80000000000000000000000000000000000F9
:104FB80000000000000000000000000000000000E9
:104FC80000000000000000000000000000000000D9
:104FD80000000000000000000000000000000000C9
:104FE80000000000000000000000000000000000B9
:104FF80000000000000000000000000000000000A9
:105008004E690000636B00006E6100006D65000072
:10501800203D0000202500007300000044650000CA
:105028007620000054790000702000003D20000028
:105038002563000025630000004600006972000037
:105048006D77000061720000652000003D200000BF
:1050580025750000005300007465000070530000BF
:10506800697A0000652000003D20000025750000D9
:10507800004D000061780000205000006F730000B0
:10508800203D0000202500006C750000004C000049
:105098006F6300006B2000003D20000025750000B4
:1050A8000043000068650000636B0000203D0000BD
:1050B8002025000075000000454E00004400000057
:1050C80000000000000000000000000000000000D8
:1050D80000000000000000000000000000000000C8
:1050E80000000000000000000000000000000000B8
:1050F80000000000000000000000000000000000A8
:105108000000000000000000000000000000000097
:105118000000000000000000000000000000000087
:105128000000000000000000000000000000000077
:105138000000000000000000000000000000000067
:105148000000000000000000000000000000000057
:105158000000000000000000000000000000000047
:105168000000000000000000000000000000000037
:105178000000000000000000000000000000000027
:105188000000000000000000000000000000000017
:105198000000000000000000000000000000000007
:1051A80000000000000000000000000000000000F7
:1051B80000000000000000000000000000000000E7
:1051C80000000000000000000000000000000000D7
:1051D80000000000000000000000000000000000C7
:1051E80000000000000000000000000000000000B7
:1051F80000000000000000000000000000000000A7
:105208000000000000000000000000000000000096
:105218000000000000000000000000000000000086
:105228000000000000000000000000000000000076
:105238000000000000000000000000000000000066
:105248000000000000000000000000000000000056
:105258005365000072690000616C0000203D000089
:10526800202500006C7500000044000061740000F7
:10527800652000003D200000256C00006C750000D2
:105288000056000065720000736900006F6E000030
:10529800203D000020250000750000004620000089
:1052A8005665000072730000696F00006E200000F0
:1052B8003D2000002575000000460000696C0000D4
:1052C800652000003D20000025730000000000005C
:1052D80000000000000000000000000000000000C6
:1052E80000000000000000000000000000000000B6
:1052F80000000000000000000000000000000000A6
:105308000000000000000000000000000000000095
:105578000025000030320000580000007B220000A7
:10558800756900006E74000036340000223A00008D
:10559800202500006C7500002C22000073740000A8
:1055A800726900006E670000223A000020000000C7
:1055B8002573000022250000732200007D000000F2
:1055C80054680000652000007265000063650000F3
:1055D8006976000065640000206300006F6D0000BC
:1055E8006D6100006E6400002069000073200000F7
:1055F800666F0000726D0000617400007465000041
:1056080064200000696E0000636F00007272000081
:1056180065630000746C000079000000556E00009E
:10562800616300006365000070740000616200003F
:105638006C6500002050000061720000616D000080
:105648006574000065720000205200006563000068
:10565800656900007665000064200000496E00005E
:10566800204300006F6D00006D6100006E64000053
:10567800005200006563000065690000766500005F
:1056880064200000436F00006D6D0000616E000033
:10569800642000005761000073200000546F000070
:1056A8006F2000004C6F00006E670000005500007E
:1056B8006E6B00006E6F0000776E000020430000E4
:1056C8006F6D00006D6100006E64000020520000E4
:1056D80065630000656900007665000064000000ED
:1056E800436100006E6E00006F74000020450000EA
:1056F80078650000637500007465000020430000B1
:105708006F6D00006D6100006E640000205700009E
:10571800686900006C6500002044000065760000A0
:10572800696300006520000049730000204D0000F7
:105738006F760000696E000067000000436100009A
:105748006E6E00006F740000204500007865000050
:105758006375000074650000204300006F6D000051
:105768006D6100006E640000202D000020440000E0
:105778006576000069630000652000004973000039
:10578800204E00006F740000204800006F6D00007C
:105798006564000000430000616E00006E6F000049
:1057A80074200000457800006563000075740000EF
:1057B80065200000436F00006D6D0000616E000001
:1057C8006420000057680000696C00006520000034
:1057D8004465000076690000636500002049000008
:1057E80073200000536C00006565000070690000BC
:1057F8006E67000000430000616E00006E6F0000DD
:10580800742000004578000065630000757400008E
:1058180065200000436F00006D6D0000616E0000A0
:105828006420000057690000746800006F7500006C
:1058380074200000546500006D70000020500000C6
:10584800726F00006265000020410000747400005F
:105858006163000068650000642E000000430000DA
:105868006F6D00006D7500006E69000063610000D7
:10587800746900006F6E000020700000726F0000F5
:10588800626C0000656D00002077000069740000FC
:1058980068200000576900002D46000069200000BC
:1058A800426F000061720000640000004361000064
:1058B8006E6E00006F7400002050000075730000C9
:1058C800682000005365000074740000696E0000D1
:1058D800677300002E2000004E650000636500001D
:1058E80073730000617200007920000053650000A6
:1058F80074740000696E00006773000020410000A6
:1059080072650000204D0000697300007369000093
:105918006E670000004400006576000069630000BF
:1059280065200000547900007065000020490000DF
:10593800732000005365000074200000496E0000C9
:10594800636F00007272000065630000746C0000F1
:1059580079000000496E0000636F00006D70000060
:1059680061740000696200006C6500002046000058
:10597800697200006D770000617200006520000008
:105988005665000072730000696F00006E00000029
:105998005468000065200000636F00006D6D000012
:1059A800616E000064200000697300002069000037
:1059B8006E760000616C00006964000020620000DF
:1059C80065630000617500007365000020740000C5
:1059D80068650000206400006576000069630000C7
:1059E8006520000069730000206800006F6D0000EA
:1059F800696E000067000000546800006520000020
:105A0800636F00006D6D0000616E0000642000008F
:105A18007265000063650000697600006564000037
:105A28002077000061730000206600006F7200009C
:105A3800206100006E200000696E000076610000A1
:105A48006C69000064200000746100007267000047
:105A5800657400002064000065760000696300003A
:105A6800650000005468000065200000466F0000D3
:105A7800637500007365000072200000646F000009
:105A880065730000206E00006F740000206800003D
:105A980061760000652000003132000056200000C9
:105AA800706F00007765000072000000457200000A
:105AB800726F0000722000007465000078740000A6
:105AC800206E00006F74000020640000656600000E
:105AD800696E0000656400000000000030000000EE
:105AE8006F6E0000656C0000796E0000782F000072
:105AF80073720000632F0000436C000069650000AA
:105B08006E7400002E63000000250000733A000048
:105B18002569000020250000732000002D2D0000BD
:105B28002061000073730000657200007469000052
:105B38006F6E000020660000616900006C6500005F
:105B4800640A00000021000000000000007000004E
:105B58005F6300006C690000656E0000742D000032
:105B68003E770000726900007465000000000000C4
:105B7800000000000000000000000000000000001D
:105B8800000000000000000000000000000000000D
:105B980000000000000000000000000000000000FD
:105BA80000000000000000000000000000000000ED
:105BB80000000000000000000000000000000000DD
:105BC80000000000000000000000000000000000CD
:105BD80000000000000000000000000000000000BD
:105BE80000000000000000000000000000000000AD
:105BF800000000000000000000000000000000009D
:105C0800000000000000000000000000000000008C
:105C1800000000000000000000000000000000007C
:105C2800000000000000000000000000000000006C
:105C3800000000000000000000000000000000005C
:105C4800000000000000000000000000000000004C
:105C5800000000000000000000000000000000003C
:105C6800000000000000000000000000000000002C
:105C7800000000000000000000000000000000001C
:105C8800000000000000000000000000000000000C
:105C980000000000000000000000000000000000FC
:105CA80000000000000000000000000000000000EC
:105CB80000000000000000000000000000000000DC
:105CC80000000000000000000000000000000000CC
:105CD80000000000000000000000000000000000BC
:105CE8000000000000000000000000000045000067
:105CF800523D0000256400002000000025730000CC
:105D08000A00000000000000000000000000000081
:105D1800000000000000000000000000000000007B
:105D2800000000000000000000000000000000006B
:105D3800000000000000000000000000000000005B
:105D4800000000000000000000000000000000004B
:105D5800000000000000000000000000000000003B
:105D6800000000000000000000000000000000002B
:105D7800000000000000000000000000000000001B
:105D8800000000000000000000000000000000000B
:105D980000000000000000000000000000000000FB
:105DA80000000000000000000000000000000000EB
:105DB80000000000000000000000000000000000DB
:105DC80000000000000000000000000000000000CB
:105DD80000000000000000000000000000000000BB
:105DE80000000000000000000000000000000000AB
:105DF800000000000000000000000000000000009B
:105E0800000000000000000000000000000000008A
:105E1800000000000000000000000000000000007A
:105E2800000000000000000000000000000000006A
:105E3800000000000000000000000000000000005A
:105E4800000000000000000000000000000000004A
:105E5800000000000000000000000000000000003A
:105E6800000000000000000000000000000000002A
:105E7800000000000000000000000000000000001A
:105E8800000000004745000054430000464700005A
:105E980000530000434C000042000000474500004A
:105EA80054440000424700000052000045420000F0
:105EB8004F4F0000540000005245000053450000B9
:105EC80054000000474500005448000055420000B7
:105ED800494E0000464F0000005300005753000091
:105EE8005300000053570000534D000000530000BA
:105EF800575300004B00000053570000574900005B
:105F0800005300005750000053000000574900009C
:105F1800464900004445000046410000554C000039
:105F28005453000000570000494600004952000041
:105F38004553000045540000005700004946000042
:105F480049530000434100004E000000474500004F
:105F5800544E000045540000004C00004F41000022
:105F6800444E00004554000000470000455400001E
:105F780048490000500000005345000054530000F9
:105F880049500000005300004554000048530000E9
:105F98004D000000534500005448000053470000DE
:105FA800005300004554000048530000440000001E
:105FB80053410000564500004950000000530000BE
:105FC80049500000525300005400000047450000AB
:105FD8005457000049500000005300004554000089
:105FE8005749000050000000534500005457000076
:105FF800534D000000530000455400005753000063
:106008004700000053450000545700005344000067
:1060180000530000415600004557000046000000AC
:106028004745000054480000435300000053000057
:106038004554000048530000530000005345000039
:106048005448000043560000005300004554000027
:106058005743000056000000474500005456000012
:1060680045520000004200004F4F0000544C000011
:106078004F41000044000000257500000053000057
:106088004554000000530000544F000052450000E2
:106098000044000045460000415500004C540000F3
:1060A8005300000053430000414E00000000000070
:1060B800484500004C4C00004F000000484F0000CD
:1060C8004D45000000430000454E000054450000C7
:1060D800520000004D310000490000004D31000021
:1060E8004F0000004D4F0000520000004D490000D5
:1060F800520000004D41000000450000524D0000D4
:10610800005300004C4500004550000000570000B7
:10611800414B000045000000474500005453000073
:10612800544100005455000053000000474500004A
:10613800544300004F4E000046490000470000004D
:10614800534300004454000000530000435400002F
:106158004300000053430000544D0000005300006A
:10616800435400004500000053430000545300000E
:1061780000530000434E00004E000000534300004F
:106188004253000000530000434200004500000055
:1061980053430000435000000052000045530000E4
:1061A80045540000005200004556000045520000CA
:1061B8005345000000530000455400004D410000C5
:1061C8005800000053450000544900004E54000098
:1061D80000470000455400005443000049000000F7
:1061E8005345000054460000535300000048000087
:1061F800414C000054000000534500005448000082
:106208004F5300000047000045540000444500007B
:1062180056000000484100004C540000454400006E
:10622800004D0000002500006C75000000530000C0
:1062380045540000002500006C6400000048000080
:106248000025000075000000535400004F50000066
:10625800504500004400000047450000544300003A
:106268004647000000470000455400005345000021
:106278005200000053430000445400000053000043
:10628800434E00004E0000005245000056450000F5
:10629800525300004500000053450000544D0000D3
:1062A80041580000005300004554000046530000C8
:1062B80053000000534100005645000053450000BC
:1062C80054000000524500005345000054000000EF
:1062D800555300004553000045540000005300008A
:1062E800455400005345000052000000534500008B
:1062F800544400004154000000530000455400007D
:10630800464900004C000000474500005446000084
:10631800494C00004500000053410000564500006C
:10632800464900004C450000005300004554000059
:10633800534900004700000047450000545300003F
:1063480049470000005300004554000000250000A4
:106358006C750000005300004156000045440000E1
:106368000000000000000000000000000000000025
:106378000000000000000000000000000000000015
:106388000000000000000000000000000000000005
:1063980000000000000000000000000000000000F5
:1063A80000000000000000000000000000000000E5
:1063B80000000000000000000000000000000000D5
:1063C80000000000000000000000000000000000C5
:1063D80000000000000000000000000000000000B5
:0863E800000000000A000000A3
:020000040000FA
:1063F000881F7800000478000040EB0070FC9800D3
:106400006000B8001004980021049800300498003F
:1064100041049800485090000004A100E8040700DF
:10642000485090000064A100000507000074A1001E
:10643000FE0407000044A1004054980010C0B300BF
:1064400000DC980010C4B30020CC98000000EB00E2
:106450007034980008007800387C020000000000CA
:10646000080078009A7C0200000000004F047800C9
:10647000000006000400FA00881F7800000478007D
:10648000E0C4B300005C9800F0C6B300105C980054
:1064900002C2B300225C980040C4B300305C980094
:1064A00051C6B300415C980060C7B300505C9800CF
:1064B0006D405000605C980066405000705C980031
:1064C000016498001264980028F8910020649800F4
:1064D0008042EB003564980045649800556498004C
:1064E0006564980075649800056C980058109000D9
:1064F0000080A10050149800A0C5B300605498001B
:106500007054980010C0B300106C9800254C98008F
:1065100045DC98000002EB006414980074149800A5
:10652000041C9800141C9800241C98006011B800EA
:10653000321C9800431C9800521C9800631C980061
:10654000721C9800032498001224980023249800B9
:10655000322498004324980010C4B30020CC980043
:10656000800220000084980068489100E1CFB300C9
:1065700001406000604C9900684891000044A1000F
:10658000604C9900123498002334980074349800B9
:10659000485090000140600089040700A1B9200024
:1065A000914078008180FB009BCBBF004800DD005C
:1065B0000100700041152B00810F500025003A00AA
:1065C00096CBBF000080FB0071B92000914078009D
:1065D000C808DD0080807000A0AA2A00808F5000CB
:1065E0001C003A0078004400E1B920000F000900C7
:1065F000315878000001B100D4BF9F00C5FF9F0053
:10660000AFCBBF00A0FF9F00B0CBBF00B0FF9F008B
:10661000668057008E740200000000000004E00055
:106620000500320076004400AFF89700014878007A
:10663000BFF897001140980051BB200091407800AE
:106640008180FB00B6CBBF004800DD000100700078
:10665000703498004F0478000080FA0000000600B3
:106660000000FA00889FBE0080047800A865020040
:1066700000000000090078007EFF070011C0B30091
:1066800009007800BC7402000000000009007800D6
:1066900057FF0700694891000038A30003003A0043
:1066A000495090000024A000C0549800CF0FB000C3
:1066B00040F02F0000844700470407006C6402008C
:1066C00000000000880778003E640200000000001F
:1066D0004F04BE000080FA0000000600881F78000A
:1066E000000478000009B0006066020000000000AD
:1066F00010708000E10F50000A00320003003900E2
:10670000E20F50000C003200022EEF00080078006B
:10671000127E0200000000001000200010708800AF
:1067200009003700080078000F0007002000200053
:106730001070880004003700080078006A6C0200BE
:1067400000000000022EEF0008007800447C0200E8
:10675000000000000800780046540200000000001D
:106760004F04780000000600881F780000047800BD
:1067700010889000E20F5000060032004850900050
:106780000054A100405498000000EB0060A4980061
:1067900028003700485090000054A0002304070050
:1067A0000018A30023003A0068A09000E10F5000F9
:1067B00015003200E20F500018003200E8A89000E7
:1067C000E0232000808F500006003E000800780083
:1067D0004E580200000000001000200060A4980045
:1067E00014003700502D2000808F5000110036001B
:1067F000080078006A580200000000002000200015
:1068000060A498000B003700E8A89000E023200067
:10681000808F50000700360004003700E8A8900081
:10682000502D2000808F500002003E000000EB0041
:1068300060A498004F047800000006000002BE002B
:106840000000E00004003D00D0C2B30080487800A2
:106850000402EA0002003700B0C2B30080487800AA
:1068600042062000110009000202D80001C3B30053
:1068700081414000934298000280B900000052001C
:10688000A2002000801F7800110009000200D8003B
:10689000000178004F00780001C3B30001424100BD
:1068A000A4429800E4C2B300B44298006A11B9004F
:1068B0000200500001404000C04298000040EB0040
:1068C000D042980000000600D000FA00889FBE0069
:1068D0008A1F78000005780020262A00C7000900DA
:1068E000305F78008E0CB1006604570040F02F0036
:1068F0008004440029F891000000FB00801F78000C
:10690000A1322A00811F78000E007800520B02008D
:1069100000000000B50307000200010008589600BF
:10692000E48757000048A3000B003200880C2000C9
:106930000E044400A0252A0007000900305C7800FE
:106940008800B1001900780088007800BBFF0700BC
:10695000881F78000200370010342A00801F78005A
:1069600031332A00811F78000E007800520B02009C
:1069700000000000E48757009C03070002000100AC
:106980002E5096000018A300020032006000B800EC
:10699000020037000E0097009E009700809FBE0007
:1069A00041342A00811F78000E007800520B02004B
:1069B00000000000E68757008C030700020001007A
:1069C0006604570049F02F008904440058009700DE
:1069D000E8009700809FBE0031352A00811F7800B3
:1069E0000E007800520B0200000000007F03070039
:1069F0000200010008589600E11F600020362A00BE
:106A0000801F78000E007800520B0200000000008A
:106A10007603070002000100085896000000D1002C
:106A2000E11F600001372A00811F78000E00780006
:106A3000520B0200000000006C030700020001007E
:106A4000085896004200DE00E11F6000E0372A008F
:106A5000801F78000E007800520B0200000000003A
:106A60006203070002000100801FEB00C1382A000A
:106A7000811F78000E007800520B02000000000019
:106A80005A03070002000100085896004400DE0087
:106A9000E11F6000A0392A00801F78000E007800F6
:106AA000520B02000000000050030700020001002A
:106AB000085896004500DE00E11F6000813A2A0078
:106AC000811F78000E007800520B020000000000C9
:106AD0004603070002000100085896004300DE004C
:106AE000E11F6000603B2A00801F78000E007800E4
:106AF000520B020000000000E0FD2F0080874700DD
:106B00003A03070002000100694891004400DE00DA
:106B1000E11F6000413C2A00811F78000E007800D0
:106B2000520B0200000000003003070002000100C9
:106B300041030700203D2A0002000100E4875700BE
:106B40004F0578004F04BE000080FA0000000600E8
:106B5000C800FA00889FBE008A9FBE00000578002A
:106B600000F32F000F004000613D2A00C70009001C
:106B700031587800800CB100E604500048F02F0036
:106B80000884440028F891000000FB00801F780072
:106B9000E0492A00801F7800C0F22F000F0040005B
:106BA000520B02000000000023030700C0F22F0078
:106BB0000F00400002000100F81F4400714A2A0043
:106BC000811F780080F22F000F004000520B02005E
:106BD000000000001803070080F22F000F004000A3
:106BE000020001007828900088309000809FBE004D
:106BF000514B2A00811F780020F22F000F00400027
:106C0000520B0200000000000B03070020F22F00CF
:106C10000F00400002000100395896000000FB0000
:106C2000801F7800295896000000FB00801F780024
:106C3000424C2A00821F7800C0F12F000F00400054
:106C4000520B020000000000FB020700C0F12F0001
:106C50000F0040000200010048D890000000FB0037
:106C6000801F7800404D2A00801F780080F12F009F
:106C70000F004000520B020000000000EE0207006F
:106C800080F12F000F00400002000100C802B00098
:106C900019042000F88757006B042000B81F780003
:106CA000891F7800314E2A00811F7800A0F22F0042
:106CB0000F004000520B020000000000DE0207003F
:106CC000A0F22F000F004000020001008904E8003C
:106CD000E68757008B8F5400F0FF3A00E0EF2F005B
:106CE00002F32F000F0141000004410028C890006A
:106CF0000000FB00801F7800204F2A00801F7800D2
:106D0000C0F22F000F004000520B020000000000F4
:106D1000C9020700C0F22F000F004000020001006E
:106D200068489100E11F600001502A00811F78002F
:106D300080F22F000F004000520B02000000000004
:106D4000BD02070080F22F000F004000020001008A
:106D500008819000821F7800E0502A00801F780090
:106D600040F22F000F004000520B02000000000014
:106D7000B102070040F22F000F00400002000100A6
:106D8000F07D0200000000000080FB00801F780002
:106D9000C1512A00811F780000F22F000F0040002F
:106DA000520B020000000000A302070000F22F00B7
:106DB0000F00400002000100581090004800DE0063
:106DC000E11F6000A2522A00821F7800C0F12F004C
:106DD0000F004000520B0200000000009602070066
:106DE000C0F12F000F004000020001001868900061
:106DF0000080FB00801F780080532A00801F7800ED
:106E000080F12F000F004000520B02000000000034
:106E10008902070080F12F000F00400002000100EE
:106E200085020700203D2A0002000100F887570074
:106E30004F05BE004F04BE000080FA0000000600AF
:106E4000CA00FA00889FBE008A9FBE008C9FBE00C9
:106E500080067800E0EF2F00A1F22F008F80400025
:106E600000864000010478007C309000001C78000F
:106E70005C1590004855DE0061456500ACCD900082
:106E8000CCDC90002CF8910061542A00C700090066
:106E9000315C7800880CB1000000FB00801F780096
:106EA000E0602A00801F780008007800520B020082
:106EB0000000000050020700020001008904FB00EE
:106EC000891F7800A1612A00811F780008007800DE
:106ED000520B020000000000470207000200010000
:106EE0008B05FB008B1F7800204F2A00801F780045
:106EF00008007800520B0200000000003E0207006C
:106F000002000100E11F6500A1522A00811F7800E4
:106F100008007800520B0200000000003602070053
:106F200002000100CC02B00018042000F0875700D6
:106F3000C0F22F00808447006A042000BC1F780044
:106F4000881F7800314E2A00811F780009007800E0
:106F5000520B0200000000003A020700090078000E
:106F6000020001000804E800E68757008A0F540079
:106F7000F2FF3A0040F32F00A1F22F008F80400073
:106F800080844000180420000185E8006B04200084
:106F9000B91F7800B91F7800881F780080622A0026
:106FA000801F78000A007800520B020000000000E9
:106FB000240207000A007800020001000804E8002B
:106FC000E88757008B0F5400F1FF3A00DF1097005D
:106FD000811F780080632A00801F78000A007800F3
:106FE000520B020000000000160207000A007800A1
:106FF0000200010013020700203D2A0002000100E8
:10700000E48757004F06BE004F05BE004F04BE0088
:107010000080FA0000000600C800FA00881F78000F
:107020000004780060F32F000F00400061642A0024
:10703000C700090031587800800CB10000017800C9
:1070400000252500F16424000099BE0090C42400AE
:10705000513425000099BE000049EB001801900052
:1070600011C0B30060F32F000F00400002000100C8
:10707000E0702A00801F7800B1722A00811F78001A
:1070800020F32F000F004000520B02000000000010
:107090001801900011C0B30020F32F000F00400032
:1070A000020001001801900011C0B300203D2A0029
:1070B00002000100E48757004F0478000080FA00C6
:1070C000000006000000FA00889FBE008A1F7800BA
:1070D0000005780081047800020478000101200096
:1070E00002007800847D0200000000000004E0003F
:1070F00005003A0011002000090078003E6B0200F4
:10710000000000001000370078004500880078007B
:10711000880C020000000000CF0FB00040F02F00EC
:10712000008447007D0009003A1C7800C80FB100B8
:10713000CA0FB1006C6402000000000088077800EC
:107140003E640200000000004F0578004F04BE00BE
:107150000080FA00000006000000FA00881F780096
:107160000002780081017800A601070005003600C2
:1071700011002000030078003E6B020000000000B8
:107180000D00370021CA9800CF0FB00040F02F004B
:10719000008447007D000900341C7800C80FB1004E
:1071A000C40FB1006C640200000000008807780082
:1071B0003E640200000000004F0478000080FA00E6
:1071C000000006000000FA00881F780080037800A5
:1071D00081017800820278008A0107000B003E00DE
:1071E0000100FB00F1FB2F000103400092409000E2
:1071F000B0C2B30080CF5000090032000084EB0021
:1072000000C0E80080CF50000600320011002000CE
:10721000030078003E6B02000000000025003700EC
:1072200018002000354190000201FB0040062000BC
:107230000091B900254090000000FB0004FD2F00E4
:1072400004004000843E20000480B9000001410099
:10725000454090000000FB006A00B90000014100B9
:10726000554090000000FB000001410000B32E00DB
:107270000001410006024300C402B00002C0B90090
:1072800000B27B00CF0FB00040F02F000084470019
:107290007D000900371C7800C80FB100C70FB1008E
:1072A0006C64020000000000880778003E64020061
:1072B000000000004F0478000080FA000000060083
:1072C0000000FA00889FBE00800478000102780068
:1072D00092417800F0CBB30000C04100F94F50005C
:1072E00005003E008200E800F0CBB30011404000F2
:1072F000F94F500005003600A1002000040078007E
:107300003E6B0200000000002A003700E3549800A2
:1073100091407800F15498000900780034FC07008F
:107320008040EB0009007800187E02000000000099
:10733000694891000038A3000D00320079289000C0
:10734000893090008100D1000080D300E0049800D3
:10735000F1049800090078009A7C02000000000007
:1073600009007800A658020000000000080037005D
:107370006000B80090049800A1049800B004980040
:10738000C1049800495090000024A000C054980007
:10739000CF0FB00040F02F00008447000E0107001F
:1073A0006C64020000000000880778003E64020060
:1073B000000000004F04BE000080FA00000006003C
:1073C000881F780001047800405090000018A30046
:1073D00006003200C1002000080078003E6B020069
:1073E000000000008000EB000A003700E07D020092
:1073F00000000000110020000004E00005003A0039
:10740000E1002000080078003E6B02000000000050
:107410008000EB00010078004F04780000000600B7
:10742000881F780000017800010478004050900027
:107430000018A30006003200C100200008007800F8
:107440003E6B0200000000008000EB0013003700DC
:10745000425090000028A30006003A00510020008E
:10746000080078003E6B0200000000008000EB0086
:107470000A003700E07D020000000000110020003B
:107480000004E00005003A00E10020000800780058
:107490003E6B0200000000008000EB00010078005D
:1074A0004F047800000006000000FA00881F7800F2
:1074B0008180FB008100EA00CF08DE006049910076
:1074C0000204A1000141710062489900CF0FB00091
:1074D00041F02F0001844700CF0007006C640200D8
:1074E00000000000880778003E64020000000000F1
:1074F0004F0478000080FA00000006000000FA0047
:10750000881F780002809800CF0FB00041F02F0054
:1075100001844700C00007006C6402000000000006
:10752000880778003E640200000000004F047800E5
:107530000080FA00000006000000FA00881F7800B2
:107540008180FB008100EA00CF08DE00116898000E
:10755000CF0FB00041F02F0001844700AE000700BC
:107560006C64020000000000880778003E6402009E
:10757000000000004F0478000080FA0000000600C0
:107580000000FA00881F780080017800010278006E
:10759000405090000048A30005003A007100200010
:1075A000040078003E6B0200000000000D00370070
:1075B000C2D99800CF0FB00040F02F0000844700E0
:1075C0007D000900331C7800C80FB100C30FB10063
:1075D0006C64020000000000880778003E6402002E
:1075E000000000004F0478000080FA000000060050
:1075F0000000FA00881F7800E1806000C808DD0004
:10760000501190000280A1000101710052109800F9
:10761000CF0FB00041F02F00018447007E0007002B
:107620006C64020000000000880778003E640200DD
:10763000000000004F0478000080FA0000000600FF
:10764000889FBE008A1F780000057800010278003C
:107650000204BE00604891000038A30005003A0013
:107660007A2890008A309000820F5000838F580053
:107670000500310011002000040078003E6B02007C
:10768000000000000D0037002AF89100186A02007F
:10769000000000001805980029059800380598009A
:1076A000490598000A007800786502000000000093
:1076B0002AF89100266A0200000000004F057800B9
:1076C0004F04BE00000006000000FA00889FBE00C4
:1076D00080047800604891000068A3000700320031
:1076E00092349800A334980019309000A93090008B
:1076F000F02C9800813498000800370011C0B300C6
:1077000009007800187E020000000000792890002F
:107710008930900090349800A1349800CF0FB000C9
:1077200040F02F00008447002B0007006C6402002B
:1077300000000000880778003E640200000000009E
:107740004F04BE000080FA00000006000000FA00AE
:10775000889FBE0080047800024478007029900061
:107760008031900010029000A002900004015100AE
:1077700085815900B2FF070061406400C400DD004C
:10778000694891000044A10001407000E04C99005C
:10779000CF0FB00040F02F00008447000E0007001C
:1077A0006C64020000000000880778003E6402005C
:1077B000000000004F04BE000080FA000000060038
:1077C0001A0007000014A100180007000024A100FF
:1077D00040549800000006007D000900391C780024
:1077E000C80FB100C90FB100000006001200070069
:1077F0000E00780000000600120007000800780064
:107800000000060092407800F0CBB30000C04000BA
:10781000E44F5000000006007D000900301C780095
:10782000C80FB100C00FB10000000600405498001E
:1078300048509000000006001A01900011C0B300EB
:10784000000006001D01900011C0B30000000600FA
:10785000000178000040EB000051980010519800A2
:10786000205198000100E0000D003A0040852900F9
:10787000801F780080012000801F7800108629007A
:10788000801F780030872900801F7800E0EE2000FC
:10789000040C020000000000500C02000000000078
:1078A0000109780001007800507A02000000000011
:1078B00000000600B1C4B300614898000000060053
:1078C00000000600C800FA00889FBE008A9FBE0024
:1078D0000004780010892900EE04070090E42400D9
:1078E00061F42400CE040700020001002000200003
:1078F000801F78008004EB00891F78003000200092
:10790000801F780090952900801F78000E00780075
:10791000520B020000000000C30407000200010037
:10792000891F7800D0962900801F78000E0078000B
:10793000520B020000000000BB040700020001001F
:10794000E60457004AE62F000A8544009A007800B2
:10795000314090000080FB00801F780021409000A3
:107960000080FB00801F7800114090000080FB0029
:10797000801F78001180FB00801F7800B0972900DD
:10798000801F78000E007800520B020000000000FB
:10799000A5040700020001001A007800406890006A
:1079A0004600DE00E11F600020992900801F78005A
:1079B0000E007800520B0200000000009A0407003D
:1079C000020001004AE892000080FB00801F78005E
:1079D000009A2900801F78000E007800520B0200E8
:1079E0000000000090040700020001004AF8900027
:1079F0000080FB00801F7800E09A2900801F78003B
:107A00000E007800520B020000000000EBFD2F007A
:107A10008B874700840407000200010069F094008E
:107A20000080FB00801F780059F094000080FB006C
:107A3000801F780049F094000080FB00801F7800D0
:107A4000C09B2900801F78000E007800520B0200B6
:107A50000000000074040700020001005AE89200D0
:107A60000080FB00801F7800009D2900801F7800A7
:107A70000E007800520B0200000000006A040700AC
:107A800002000100F81F4500E09D2900801F7800DA
:107A90000E007800520B0200000000006204070094
:107AA0000200010039F894000080FB00801F78007C
:107AB00029F894000080FB00801F780019F89400DA
:107AC0000080FB00801F780009F894000080FB0014
:107AD000801F7800C09E2900801F78000E0078006B
:107AE000520B0200000000004F04070002000100DA
:107AF0001A7890000080FB00801F780030A02900D9
:107B0000801F78000E007800520B02000000000079
:107B100045040700020001000E0178007065240092
:107B2000013225000099BE0050362600B19427008E
:107B30000099BE0000D22300010220000089BE008F
:107B400039040700020001003AF890000080FB00B1
:107B5000801F780010A12900801F78000E00780097
:107B6000520B0200000000008B8747002E04070024
:107B700002000100180190003F040700020001000C
:107B80004F05BE004F04BE000080FA000000060052
:107B9000C800FA00889FBE008A1F780000057800A0
:107BA00030A229003704070020002000801F780041
:107BB000801FEB0030002000801F7800B0AE29004D
:107BC000801F78000E007800520B020000000000B9
:107BD00024040700020001006604570049E62F0054
:107BE0008904440028F094000080FB00801F780086
:107BF000F0AF2900801F78000E007800520B0200C1
:107C0000000000001704070002000100D0B02900A6
:107C1000070407000200010099007800314090003D
:107C20000080FB00801F7800214090000080FB0056
:107C3000801F7800114090000080FB00801F7800BA
:107C40001180FB00801F7800B0972900801F78000A
:107C50000E007800520B0200000000000104070033
:107C60000200010049E892000080FB00801F7800BC
:107C7000A0B12900801F78000E007800520B02008E
:107C800000000000F70307000200010049F890001F
:107C90000080FB00801F780080B22900801F7800E0
:107CA0000E007800520B020000000000ED030700F8
:107CB0000200010059E892000080FB00801F78005C
:107CC00060B32900801F78000E007800520B02007C
:107CD00000000000E0FD2F0080874700E10307005F
:107CE0000200010068F094000080FB0001FD2F00FD
:107CF000811F400058F094000080FB00811F40006D
:107D000048F094000080FB00811F400040B429002F
:107D1000801F78000E007800520B02000000000067
:107D2000D003070002000100F89F440080B529003D
:107D3000801F78000E007800520B02000000000047
:107D4000C80307000200010038F894000080FB001F
:107D5000801F780028F894000080FB00801F7800C6
:107D600018F894000080FB00801F780008F8940049
:107D70000080FB00801F780060B62900801F78001B
:107D80000E007800520B020000000000B50307004F
:107D90000200010099789000F68757000104E00086
:107DA0000C00320020C4B300E8CF50000A003200BB
:107DB00030C4B300E7CF50000700320040C4B30026
:107DC000E1CF50000400320050C4B300E2CF5000B5
:107DD0000100320010C4B3000000FB00801F7800D7
:107DE000D0B72900801F78000E007800520B0200E7
:107DF000000000009B0307000200010080E92F0043
:107E0000801F4700B0B82900801F78000E0078005E
:107E1000520B020000000000920307000200010064
:107E20008703070002000100E88757004F0578002C
:107E30004F04BE000080FA0000000600C800FA00EF
:107E4000889FBE008004780090B92900870307004E
:107E50003035240011E424000099BE000092240073
:107E6000E16424000099BE00F004200000097800BD
:107E70007503070002000100E0E52F000004470041
:107E8000085092000080FB00801F780010C6290077
:107E9000801F78000E007800520B020000000000E6
:107EA0006903070002000100285092000080FB00D7
:107EB000801F7800F0C62900801F78000E0078002F
:107EC000520B0200000000005F03070002000100E7
:107ED000185092000080FB00801F7800D0C7290056
:107EE000801F78000E007800520B02000000000096
:107EF000550307000200010030112000801F4400DC
:107F0000B0C82900801F78000E007800520B0200D4
:107F1000000000004C0307000200010038709200CE
:107F20000080FB00801F780090C92900801F780026
:107F30000E007800520B0200000000004203070010
:107F400002000100487092000080FB00801F780052
:107F500070CA2900801F78000E007800520B0200C2
:107F60000000000038030700020001005870920072
:107F70000080FB00801F780050CB2900801F780014
:107F80000E007800520B0200000000002E030700D4
:107F90000200010028E892000080FB00801F7800AA
:107FA00030CC2900801F78000E007800520B0200B0
:107FB0000000000000FE2F0080874700220307001A
:107FC00002000100190190002B03070002000100CC
:107FD0004F04BE000080FA0000000600DC00FA003A
:107FE000889FBE008A1F7800000578007E2C9600CE
:107FF00050CE290027030700900425000192240099
:108000000099BE00E0642400F10420000089BE0055
:108010001403070002000100384090000080FB00BC
:10802000801F7800284090000080FB00801F7800AF
:10803000184090000080FB00801F78001880FB0033
:10804000801F7800D0DA2900801F78000E007800A9
:10805000520B0200000000000203070002000100B2
:10806000784090000080FB00801F780068409000FE
:108070000080FB00801F7800584090000080FB00CB
:10808000801F7800484090000080FB00801F78002F
:1080900040DC2900801F78000E007800520B02009F
:1080A00000000000EF0207000200010038489000C5
:1080B0000080FB00801F7800284890000080FB00B3
:1080C000801F7800184890000080FB00801F780017
:1080D000084890000080FB00801F7800B0DD290078
:1080E000801F78000E007800520B02000000000094
:1080F000DC02070002000100784890000080FB00CD
:10810000801F7800684890000080FB00801F780086
:10811000584890000080FB00801F7800484890007D
:108120000080FB00801F780020DF2900801F78007E
:108130000E007800520B02000000000080FD2F00AE
:1081400080874700C70207000200010038509000F6
:108150000080FB00801F7800285090000080FB000A
:10816000801F7800185090000080FB00801F78006E
:10817000085090000080FB00801F780090E02900EC
:10818000801F78000E007800520B020000000000F3
:10819000B402070002000100785090000080FB004C
:1081A000801F7800685090000080FB00801F7800DE
:1081B000585090000080FB00801F780048509000CD
:1081C0000080FB00801F780000E22900801F7800FB
:1081D0000E007800520B020000000000A102070010
:1081E00002000100385890000080FB00801F7800DA
:1081F000285890000080FB00801F780018589000DD
:108200000080FB00801F7800085890000080FB0071
:10821000801F780070E32900801F78000E0078002E
:10822000520B0200000000008E0207000200010055
:10823000486890004600DE00E11F6000E0E429008D
:10824000801F78000E007800520B02000000000032
:10825000E0FD2F0080874700820207000200010036
:10826000FC1F4400C0E52900801F78000E00780044
:10827000520B0200000000007A0207000200010019
:10828000890C20008E84440010CD290013000900C1
:10829000B05C78004901B100D00220000800400025
:1082A0001080FB00E8689000C808DD008080700046
:1082B000786890000080FB00087190004811DD0094
:1082C00000017100187090000080FB00A871900000
:1082D000C819DD0080817100090078002C020700B8
:1082E000891F7800A0E62900801F78000E00780022
:1082F000520B0200000000005A02070002000100B9
:108300004F02070002000100E88757004F05780080
:108310004F04BE000080FA0000000600DC00FA00F6
:10832000889FBE008A1F780000057800C0E82900F9
:108330005402070040F529003D0207000200010039
:10834000E0E52F0000044700187892000080FB0051
:10835000801F7800087892000080FB00801F780062
:10836000787092000080FB00801F78006870920097
:108370000080FB00801F7800D0DA2900801F780081
:108380000E007800520B02000000000035020700CA
:1083900002000100587892000080FB00801F7800E6
:1083A000487892000080FB00801F780038789200A7
:1083B0000080FB00801F7800287892000080FB007E
:1083C000801F780040DC2900801F78000E007800B4
:1083D000520B020000000000220207000200010010
:1083E00018C092000080FB00801F780008C0920037
:1083F0000080FB00801F7800787892000080FB00EE
:10840000801F7800687892000080FB00801F780051
:10841000B0DD2900801F78000E007800520B0200AA
:10842000000000000F0207000200010058C0920087
:108430000080FB00801F780048C092000080FB0095
:10844000801F780038C092000080FB00801F7800F9
:1084500028C092000080FB00801F780020DF2900E8
:10846000801F78000E007800520B02000000000010
:1084700080FD2F0080874700FA01070002000100FD
:1084800018C892000080FB00801F780008C8920086
:108490000080FB00801F780078C092000080FB0005
:1084A000801F780068C092000080FB00801F780069
:1084B00090E02900801F78000E007800520B020027
:1084C00000000000E70107000200010058C8920008
:1084D0000080FB00801F780048C892000080FB00ED
:1084E000801F780038C892000080FB00801F780051
:1084F00028C892000080FB00801F780000E229005D
:10850000801F78000E007800520B0200000000006F
:10851000D40107000200010018D092000080FB0087
:10852000801F780008D092000080FB00801F780038
:1085300078C892000080FB00801F780068C8920015
:108540000080FB00801F780070E32900801F780006
:108550000E007800520B020000000000C10107006D
:1085600002000100183091004600DE00E11F6000AB
:10857000E0E42900801F78000E007800520B020012
:1085800000000000E0FD2F0080874700B5010700D4
:1085900002000100183091004700DE00E11F60007A
:1085A00010F62900801F78000E007800520B0200A0
:1085B00000000000AB0107000200010020152000B0
:1085C000801F4400C0E52900801F78000E0078005D
:1085D000520B020000000000A2010700020001008F
:1085E000890C20008E84440080E7290013000900D4
:1085F000B05C78004901B10030162000080040004E
:108600001080FB00C8E09200C808DD008080700088
:1086100058E092000080FB0068E192004811DD0004
:108620000001710078E092000080FB0088E9920070
:10863000C819DD008081710009007800540107002D
:10864000891F7800A0E62900801F78000E007800BE
:10865000520B02000000000082010700020001002E
:108660007701070002000100EC8757004F057800F2
:108670004F04BE000080FA0000000600E400FA008B
:10868000889FBE008A9FBE008C1F780080057800FE
:10869000E0E52F0080044700295E9300F0F62900F2
:1086A000780107008A0C20000E054500680D2000A7
:1086B0000E04440008007800467A02000000000022
:1086C00006000900381D7800EA00B100E800B1009A
:1086D0003EC891000080FB00801F78002EC89100EA
:1086E0000080FB00801F78001EC891000080FB0006
:1086F000801F78001A80FB00801F780070032A001A
:10870000801F78000E007800520B0200000000006D
:108710004F010700020001007EC891000080FB00AD
:10872000801F78006EC891000080FB00801F7800D9
:108730005EC891000080FB00801F78004EC8910049
:108740000080FB00801F780000052A00801F780051
:108750000E007800520B0200000000003C010700F0
:10876000020001003ED091000080FB00801F7800D5
:108770002ED091000080FB00801F78001ED0910059
:108780000080FB00801F78000ED091000080FB006D
:10879000801F7800B0062A00801F78000E00780045
:1087A000520B020000000000290107000200010036
:1087B0004ED091000080FB00801F780040082A0006
:1087C000801F78000E007800520B020000000000AD
:1087D000E8FD2F00888747001D0107000200010007
:1087E000195093000080FB00801F7800095093000F
:1087F0000080FB00801F7800794893000080FB0018
:10880000801F7800694893000080FB00801F78007B
:1088100060092A00801F78000E007800520B0200C9
:10882000000000000A0107000200010059509300F7
:108830000080FB00801F7800495093000080FB00FF
:10884000801F7800395093000080FB00801F780063
:10885000295093000080FB00801F7800000B2A0045
:10886000801F78000E007800520B0200000000000C
:10887000F700070002000100195893000080FB0078
:10888000801F7800095893000080FB00801F78004B
:10889000795093000080FB00801F7800695093009E
:1088A0000080FB00801F7800C00C2A00801F780029
:1088B0000E007800520B020000000000E4000700E8
:1088C000020001000C86FB008C1F7800600E2A005D
:1088D000801F78000E007800520B0200000000009C
:1088E00088874700DA000700020001001B019000A2
:1088F000E1000700020001004F0678004F05BE00AE
:108900004F04BE000080FA0000000600CE00FA000E
:10891000889FBE008A9FBE008C9FBE000004780026
:1089200066005700D0E8940031CF9900E0E8940049
:1089300021CF9900F0E8940011CF990090E89400BD
:1089400001CF9900A0E8940041CF9900B0EE9400C7
:1089500040F69400D0F5940060F59400900F2A0042
:10896000C200070060552400213525000099BE0093
:1089700090F42400E1342500A90007000200010062
:10898000111C2A00811F7800501C2A00801F7800CB
:108990000E007800520B020000000000A200070049
:1089A0000200010021002000811F78008004EB00FC
:1089B000891F780030002000801F7800311D2A00B8
:1089C000811F78000E007800520B020000000000AA
:1089D000950007000200010060002000801F780061
:1089E000891F7800891F7800711E2A00811F780076
:1089F0000E007800520B0200000000008A00070001
:108A0000020001000A85FB008A1F78008B85FB00AD
:108A10008B1F78000C86FB008C1F7800B01F2A008B
:108A2000801F78000E007800520B0200000000004A
:108A30007D000700020001008D06FB008D1F7800FD
:108A4000CEC891000100FB00801F78008EC8910005
:108A50000100FB00801F7800F0202A00801F7800B2
:108A60000E007800520B020000000000C0FD2F0035
:108A7000808747006C000700020001009EC891003B
:108A80000100FB00801F7800AEC891000100FB00D0
:108A9000801F7800BEC891000100FB00801F780095
:108AA00030222A00801F78000E007800520B02004E
:108AB000000000005C00070002000100891F780030
:108AC000891F7800891F780071232A00811F780090
:108AD0000E007800520B0200000000005200070058
:108AE0000200010030002000801F7800B1242A001D
:108AF000811F78000E007800520B02000000000079
:108B00004900070002000100180190005A00070008
:108B100002000100F48757004F06BE004F05BE005B
:108B20004F04BE000080FA00000006000000FA00BA
:108B3000889FBE008144780061489800CF19B0003A
:108B400041E62F0001844700CD000900301C780069
:108B5000C819B100C019B100626402000000000031
:108B6000880778003E640200000000000940780099
:108B7000F67D0200000000004F04BE000080FA00F5
:108B800000000600B06502000000000000000600C2
:108B90000600FA00889FBE008A9FBE008C9FBE0020
:108BA00000057800F1B79F0082BF9F0093BF9F0030
:108BB0008004EB008905780072865700ADC3B300CE
:108BC000040037000B00E000020032008D747D00CD
:108BD0008904E8003C44780008407800527602009E
:108BE0000000000000F57C00084078006676020076
:108BF0000000000089004500904098008984E8004A
:108C00008B05E800E68F5500EEFF3A004F06BE00E8
:108C10004F05BE004F04BE000080FA0000000600B1
:108C20000099BE000049EB00180190000A003700CF
:108C30000C000900305F7800DE00B1000900370049
:108C40001A0190000C003700190190000200370053
:108C50001B0190000000370011C0B3000E00780027
:108C6000000006001A019000FBFF37000500070016
:108C70000E0178000000060011C0B300F0A1290029
:108C800000000600C7000900305F78008E0CB100BC
:108C900000000600F5FF0700805425002104220093
:108CA0000099BE0000000600881F7800650440009F
:108CB0005200200088007800C0052B00980B0200AD
:108CC00000000000018224000000E000D900320012
:108CD0005A03070020062B00980B0200000000003A
:108CE00081B224000000E000D200320056030700E9
:108CF00070062B00980B02000000000061B42400F5
:108D00000000E000CB00320052030700E0062B0019
:108D1000980B020000000000618724000000E000C2
:108D2000C40032004B03070020072B00980B020001
:108D300000000000A18A24000000E000BD00320015
:108D40004403070060072B00980B0200000000009E
:108D5000E18D24000000E000B60032003D03070072
:108D6000A0072B00980B020000000000A18F240038
:108D70000000E000AF0032002200200088007800F0
:108D8000E0072B00980B02000000000001AE240059
:108D90000000E000A70032002E03070010082B009F
:108DA000980B020000000000E1C424000000E00075
:108DB000A0003200520020008800780050082B00EC
:108DC000980B020000000000C18224000000E000B7
:108DD0009800320019030700B0082B00980B02001E
:108DE00000000000E18224000000E0009100320059
:108DF000920020008800780000092B00980B0200E8
:108E000000000000818424000000E000890032009E
:108E10009200200088007800A0092B00980B020027
:108E200000000000018324000000E0008100320007
:108E300002030700400A2B00980B0200000000000C
:108E400001AD24000000E0007A003200FB020700C0
:108E5000900A2B00980B02000000000041C724007C
:108E60000000E00073003200F4020700E00A2B006B
:108E7000980B02000000000041C624000000E00042
:108E80006C003200ED020700300B2B00980B020043
:108E90000000000081BF24000000E00065003200F7
:108EA000E6020700800B2B00980B02000000000078
:108EB00041C224000000E0005E003200DF02070033
:108EC000D00B2B00980B02000000000001AC240026
:108ED0000000E00057003200D8020700200C2B00F1
:108EE000980B02000000000021B924000000E000FF
:108EF00050003200D1020700700C2B00980B0200CA
:108F00000000000081B624000000E00049003200AB
:108F1000CA020700C00C2B00980B020000000000E2
:108F2000619124000000E000420032005200200065
:108F300088007800100D2B00980B02000000000044
:108F400041C824000000E0003A0032007200200016
:108F500088007800700D2B00980B020000000000C4
:108F6000219524000000E00032003200B602070024
:108F7000F00D2B00980B020000000000E197240088
:108F80000000E0002B003200AF020700600E2B0053
:108F9000980B020000000000219B24000000E0006C
:108FA00024003200A8020700D00E2B00980B02000C
:108FB00000000000C1A524000000E0001D003200F8
:108FC000A1020700400F2B00980B020000000000D8
:108FD00041A724000000E0001600320097020700BD
:108FE000B00F2B00980B0200000000000186240047
:108FF0000000E0000F0032009302070000102B0079
:10900000980B02000000000081BC24000000E0007A
:10901000080032008C02070070102B00980B020031
:109020000000000041CB24000000E00001003200FD
:109030008000EB00010078004F047800000006007B
:10904000780141009001900011C0B3000200780047
:1090500003000100000006000000060000000600FA
:109060000000FA00881F7800CF0FB00041F02F00F9
:10907000018447007A020700A835020000000000C2
:10908000880778004F0478000080FA00000006008E
:109090000000FA00881F7800CF0FB00041F02F00C9
:1090A000018447006E0207006434020000000000E3
:1090B000880778004F0478000080FA00000006005E
:1090C000881F7800000478000200780044580200ED
:1090D000000000001801900011C0B300E0102B0048
:1090E000020001004F04780000000600889FBE00C7
:1090F0008A9FBE005F02070061055000E0855800AE
:109100006002070004003600630207003E6B0200A5
:10911000000000000C003700890078000200780091
:10912000103A0200000000000004E00006003200D7
:109130000A01BE0008007800885802000000000004
:1091400058020700020001004F05BE004F04BE0098
:1091500000000600889FBE008A9FBE0045020700EF
:1091600061054000E0854800460207000400360023
:10917000490207003E6B0200000000000C003700AF
:109180008900780002007800103A02000000000018
:109190000004E000060032000A01BE00080078006A
:1091A00088580200000000003E0207000200010093
:1091B0004F05BE004F04BE0000000600889FBE00A1
:1091C0003C020700103A0200000000000004E0002A
:1091D000060032000103200008007800CE5802008B
:1091E000000000002F020700020001004F04BE0033
:1091F00000000600889FBE002E020700103A020001
:10920000000000000004E00006003200110320000E
:1092100008007800CE58020000000000210207007C
:10922000020001004F04BE00000006000400FA0026
:10923000889FBE00D8010700648040008E1F780020
:1092400071112B00811F7800BA0B02000000000092
:10925000E4875700E10F500006003A00792890009B
:10926000893090001E01BE00820F5000838F58008D
:1092700004003100130207003E6B020000000000F2
:109280000500370012020700203B0200000000002A
:10929000D3010700020001004F04BE000080FA0065
:1092A000000006000200FA00889FBE00CE01070001
:1092B00067804000E6805700B87D02000000000093
:1092C0000000E00007003A002FF9970000020700B5
:1092D000A63B020000000000C101070002000100DF
:1092E00003003700F70107003E6B0200000000009A
:1092F0004F04BE000080FA00000006000400FA00DF
:10930000889FBE00A4010700668040008E1F780081
:1093100071112B00811F7800BA0B020000000000C1
:10932000E4875700E10F500002003A00B301070044
:1093300004003600E30107003E6B0200000000005D
:1093400005003700E2010700643B02000000000056
:10935000A3010700020001004F04BE000080FA00D4
:10936000000006000400FA00889FBE008A9FBE002D
:109370008004780082057800890107006685400036
:10938000F0CBB3001A404000E44F50000D003E0007
:109390007144900000C3B300804F54000D003200B0
:1093A00065405000804F54000A0032006640400083
:1093B000804F54000700320064405000804F54003A
:1093C00004003200B40107003E6B02000000000000
:1093D00035003700678040008E1F7800F1112B00A8
:1093E000811F7800BA0B020000000000E4875700DC
:1093F000E10F500007003A008001070005003C0023
:1094000010DC2B0001FF2F00800F5100818F5900CD
:1094100003003D00A00107003E6B020000000000B9
:10942000D0C2B300804F54000300320064404000BB
:10943000804F540007003A001E0078000081EB00C6
:109440000201B800008051009E0090008101500090
:10945000028FBE001A80FB004200DD0021F32F00C6
:10946000010040000B0040001E01BE000288BE004B
:10947000CF0FB00040F02F00008447007D000900AE
:109480003B1C7800C80FB100CB0FB1006C64020028
:1094900000000000880778003E6402000000000021
:1094A0005C010700020001004F05BE004F04BE0032
:1094B0000080FA00000006000000FA00881F780013
:1094C000CF0FB00041F02F00018447006401070076
:1094D0002037020000000000880778004F04780061
:1094E0000080FA00000006000400FA00889FBE0019
:1094F0008A1F7800000578008204780028010700A0
:10950000668040008E1F780071112B00811F78004B
:10951000BA0B020000000000E4875700E10F500082
:1095200005003200110020000A0078003E6B0200A6
:10953000000000000E0037001E007800F034980094
:10954000CF0FB00040F02F00008447003301070028
:109550006C64020000000000880778003E6402008E
:10956000000000001A019000100107000200010035
:109570004F0578004F04BE000080FA00000006008E
:10958000881F78000C01070062380200000000000C
:1095900013010700020001004F04780000000600DC
:1095A000881F7800040107006039020000000000F5
:1095B0000B010700020001004F04780000000600C4
:1095C0000400FA00889FBE0019010700F40007009C
:1095D0000180E8008E1F780071112B00811F780038
:1095E000BA0B020000000000E4875700E10F5000B2
:1095F00005003A007828900088309000BE0F500097
:10960000AE8F580004003100230107003E6B0200BA
:10961000000000000B0037000800BE00103A0200F6
:10962000000000000004E000060032001E01BE0041
:1096300008007800885802000000000019010700A7
:10964000020001004F04BE000080FA000000060086
:10965000889FBE0017010700E039020000000000EB
:109660000004E0000700320008007800A65802005D
:10967000000000001901900011C0B30030122B004F
:10968000020001004F04BE0000000600889FBE00DB
:1096900008010700103A0200000000000004E0008A
:1096A0000900320078299000883190008301D100B0
:1096B0000281D300080078008858020000000000F2
:1096C000F8000700020001004F04BE000000060081
:1096D0000200FA00889FBE00BC000700E680570029
:1096E000B87D0200000000000000E00007003A0022
:1096F000AFF8970008007800543A0200000000001C
:10970000C40007000200010003003700E200070068
:109710003E6B0200000000004F04BE000080FA0013
:10972000000006000200FA00889FBE0000047800D6
:1097300082047800000FEB00648040008E1F7800E8
:1097400051122B00811F7800BA0B020000000000AC
:10975000E4875700E10F500006003200D9000700EF
:109760003E6B0200000000009D00070002000100A7
:10977000040037001E017800D50007007E3A020081
:10978000000000004F04BE000080FA000000060048
:109790000200FA00889FBE00A50007000040EB0011
:1097A000A0FF9F0066804000E6805700B87D020061
:1097B000000000000000E00007003A00AFF897004A
:1097C000080078009C3A02000000000091000700A9
:1097D0000200010003003700AF0007003E6B0200EB
:1097E000000000004F04BE000080FA0000000600E8
:1097F0000200FA00889FBE007B00070064804000E2
:10980000E6805700B87D0200000000000000E00084
:1098100007003A002FF99700AD000700C03A020098
:10982000000000006E000700020001000300370086
:10983000A40007003E6B0200000000004F04BE00C1
:109840000080FA00000006000200FA00889FBE00B7
:109850005E000700E6805700B87D020000000000AF
:109860000000E00007003A00AFF897000800780019
:10987000F83A020000000000660007000200010044
:1098800003003700840007003E6B02000000000068
:109890004F04BE000080FA0000000600881F780018
:1098A0000004780002007800FE580200000000006A
:1098B0001801900011C0B30080122B0002000100BB
:1098C0004F04780000000600881F78003A00070067
:1098D000AC38020000000000410007000200010057
:1098E0004F04780000000600881F7800320007004F
:1098F000E238020000000000390007000200010009
:109900004F047800000006000000FA00889FBE00A7
:109910008A1F780000057800820478000200780031
:109920003033020000000000CF0FB00040F02F00E5
:1099300000844700390007006C640200000000004A
:10994000880778003E640200000000001A019000C1
:1099500016000700020001004F0578004F04BE000A
:109960000080FA00000006000000FA00881F78005E
:10997000CF0FB00041F02F000184470038000700EE
:109980000C38020000000000880778004F047800BF
:109990000080FA00000006000004780082047800CD
:1099A000000FEB003E1778000000060011C0B30066
:1099B000B0112B00000006000004780002007800BF
:1099C000648140008800780000000600180007004D
:1099D0000040EB00E0F79F006480400000000600BC
:1099E00018019000F1FF370000047800820478002D
:1099F0000040EB00E0F79F00000006001E01BE00E3
:109A0000F0232400F1002000800F5100818F5900C5
:109A10000000060019019000E4FF37007D000900F6
:109A2000391C7800C80FB100C90FB1000000060052
:109A30008004780002047800000006004200200044
:109A4000880078000000060062002000880078008E
:109A500000000600320020008800780000000600A8
:109A60007D000900321C7800C80FB100C20FB100A0
:109A700000000600EEFF070012009000A200900018
:109A8000000006007228900082309000800F550080
:109A9000818F5D00000006001100200009007800A1
:109AA000000006001901900011C0B30050112B00F6
:109AB00000000600DEFF070080007800020078004A
:109AC00000000600110020000800780000000600D9
:109AD0008800780009007800000006000000EB0014
:109AE00000000600881F7800650440004A03070054
:109AF00060F42A00980B02000000000061F72400C7
:109B00000000E000F600320046030700D0F42A000F
:109B1000980B02000000000061FA24000000E00041
:109B2000EF0032003C03070020F52A00980B0200EA
:109B30000000000081FE24000000E000E800320088
:109B40003503070090F52A00980B02000000000082
:109B5000A1FE24000000E000E100320052002000DD
:109B60008800780000F62A00980B02000000000030
:109B700061FF24000000E000D9003200A2002000B4
:109B80008800780060F62A00980B020000000000B0
:109B9000E1F824000000E000D100320021030700BA
:109BA00010F72A00980B0200000000002100250099
:109BB0000000E000CA0032001A03070060F72A0024
:109BC000980B020000000000410425000000E000A6
:109BD000C300320013030700B0F72A00980B0200FD
:109BE00000000000410625000000E000BC0032003B
:109BF0000C03070000F82A00980B02000000000088
:109C0000610A25000000E000B500320005030700EE
:109C100050F82A00980B020000000000610C25009B
:109C20000000E000AE003200C20020008800780092
:109C3000A0F82A00980B0200000000002110250067
:109C40000000E000A60032009200200088007800AA
:109C500070F92A00980B0200000000002112250074
:109C60000000E0009E0032008200200088007800A2
:109C700010FA2A00980B020000000000C113250012
:109C80000000E00096003200E3020700A0FA2A007C
:109C9000980B020000000000A11625000000E00063
:109CA0008F003200720020008800780010FB2A002C
:109CB000980B020000000000211A25000000E000BF
:109CC00087003200D402070090FB2A00980B0200A4
:109CD00000000000411C25000000E0008000320070
:109CE000CD02070000FC2A00980B020000000000D3
:109CF000411F25000000E00079003200C602070085
:109D000070FC2A00980B02000000000001222500D0
:109D10000000E00072003200BF020700E0FC2A00F1
:109D2000980B020000000000C12425000000E000A4
:109D30006B003200B802070050FD2A00980B0200A9
:109D400000000000812725000000E00064003200D0
:109D5000B1020700C0FD2A00980B020000000000BD
:109D6000212A25000000E0005D003200AA02070061
:109D700030FE2A00980B020000000000E12B2500B5
:109D80000000E00056003200A3020700A0FE2A00F7
:109D9000980B020000000000C11D25000000E0003B
:109DA0004F0032009C02070010FF2A00980B0200AF
:109DB00000000000412C25000000E00048003200B7
:109DC0009502070080FF2A00980B020000000000A7
:109DD000012F25000000E000410032008E02070044
:109DE000F0FF2A00980B020000000000C13125009E
:109DF0000000E0003A0032008702070060002B00FC
:109E0000980B020000000000813425000000E000F3
:109E10003300320080020700D0002B00980B0200B4
:109E200000000000213725000000E0002C00320077
:109E30007902070040012B00980B0200000000008F
:109E400021FE24000000E00025003200720207001D
:109E5000B0012B00980B02000000000041FE24001E
:109E60000000E0001E0032006B02070020022B0001
:109E7000980B02000000000061FE24000000E000DA
:109E8000170032006402070090022B00980B0200BA
:109E900000000000213C25000000E000100032001E
:109EA0005D02070000032B00980B02000000000079
:109EB000413C25000000E000090032007200200053
:109EC0008800780070032B00980B0200000000004F
:109ED000C13D25000000E000010032008000EB00E1
:109EE000010078004F047800000006000000FA002E
:109EF000881F7800CF19B00041E62F000184470089
:109F00004B020700C83D02000000000088077800EF
:109F10004F0478000080FA00000006000000FA00FC
:109F2000881F7800CF19B00041E62F000184470058
:109F30003F020700623C0200000000008807780032
:109F40004F0478000080FA00000006000200FA00CA
:109F5000889FBE000004780082047800000FEB00A8
:109F6000648040008E1F780001042B00811F780060
:109F7000BA0B020000000000E4875700E10F500018
:109F800004003A009E00780040062000808F5000B8
:109F9000040036002B0207003E6B020000000000A8
:109FA0000500370009007800964502000000000017
:109FB00004020700020001004F04BE000080FA0006
:109FC0000000060000000600000006000000060079
:109FD0000000060010019000FB01070002000100D4
:109FE000D87D020000000000000006001001900073
:109FF000F501070002000100D87D0200000000000A
:10A0000000000600889FBE008A9FBE000005780001
:10A01000810478000E0207001400340064804400BC
:10A020007C0C02000000000001022000810F5000A3
:10A030000E003E00880920000B044400E480440028
:10A0400008007800880C020000000000080078007A
:10A050007C0C020000000000807D99001A01900035
:10A06000D9010700020001000400370011002000A0
:10A070000A0078003E6B0200000000004F05BE00A1
:10A080004F04BE000000060080017800C14090002F
:10A09000F0CBB30000C04000E44F500005003E008C
:10A0A0001179990013019000C70107000200010017
:10A0B0000400370011002000030078003E6B02000E
:10A0C0000000000000000600889FBE008A9FBE00BE
:10A0D0000005780081017800DD01070014003400DC
:10A0E000E4844100090078007C0C020000000000BC
:10A0F00001042000810F50000D003E00A80B20003D
:10A100000B0444000800BE00880C020000000000A0
:10A11000080078007C0C020000000000A0FD9900FF
:10A120001A019000A8010700020001000400370096
:10A13000110020000A0078003E6B020000000000C1
:10A140004F05BE004F04BE000000060080017800ED
:10A15000C1409000F0CCB30000C04000E34F50007D
:10A1600005003E0031F999001301900096010700A7
:10A1700002000100040037001100200003007800F5
:10A180003E6B02000000000000000600B70107005F
:10A1900017003200027891000004E000090032004C
:10A1A000927891000104E0000600320010C4B30070
:10A1B00080CF50000800320022F891000004E00037
:10A1C00005003A0091002000030078003E6B020079
:10A1D000000000000A003700E00F200002004000ED
:10A1E00071042B007B01070002000100040037000E
:10A1F00081002000030078003E6B02000000000098
:10A20000000006009901070009003200E00F20005D
:10A2100002004000D1042B000800090031587800EA
:10A220009000B1006E010700020001000400370039
:10A2300081002000030078003E6B02000000000057
:10A24000000006008901070006003200E00F200030
:10A250000200400001F62A005E0107000200010032
:10A260000400370081002000030078003E6B0200EC
:10A270000000000000000600889FBE005D0107008E
:10A2800016FE07000004E0000C003200E00F200082
:10A290000800400061052B000400090031587800D7
:10A2A0005000B10011C0B30061EC9A001901900098
:10A2B00030042B0002000100040037008100200060
:10A2C000090078003E6B0200000000004F04BE0051
:10A2D000000006000000FA00889FBE008A1F780078
:10A2E0000005780082047800FCFD07000004E0000F
:10A2F0000C003200CF19B00040E62F000084470068
:10A30000CD000900391C7800C819B100C919B10085
:10A310000A0078001E3F0200000000008807780055
:10A3200004003700810020000A0078003E6B020024
:10A33000000000004F0578004F04BE000080FA00C6
:10A3400000000600889FBE002A010700E3FD070009
:10A350000004E0000600320011C0B30021EC9A00B6
:10A360001901900030042B000200010004003700A6
:10A3700081002000090078003E6B02000000000010
:10A380004F04BE00000006000000FA00881F78009D
:10A39000CF19B00041E62F000184470024010700D7
:10A3A000EE3F020000000000880778004F047800AC
:10A3B0000080FA00000006000000FA00881F780004
:10A3C000CF19B00041E62F000184470018010700B3
:10A3D0008E41020000000000880778004F047800DA
:10A3E0000080FA00000006000400FA00881F7800D0
:10A3F00003010700E68057007876020000000000A5
:10A400000000E0000800320000010700A27A02000C
:10A41000000000000004E00003003200E900070033
:10A420000200010003003700060107003E6B020036
:10A43000000000004F0478000080FA0000000600D1
:10A440000400FA00881F7800ED000700E68057003E
:10A4500078760200000000000000E00008003200F2
:10A46000EA000700B47A0200000000000004E000E7
:10A4700003003200D3000700020001000300370090
:10A48000F00007003E6B0200000000004F0478005F
:10A490000080FA00000006000400FA00881F78001F
:10A4A000D7000700E6805700787602000000000021
:10A4B0000000E00008003200D4000700BA7A020071
:10A4C000000000000004E00003003200BD000700AF
:10A4D0000200010003003700DA0007003E6B0200B3
:10A4E000000000004F0478000080FA000000060021
:10A4F0000200FA00881F7800000478000040EB009A
:10A50000C0FF9F0066804000E4805700B87D0200D5
:10A51000000000000000E00004003A004FF897003F
:10A52000C07A02000000000003003700C5000700E9
:10A530003E6B0200000000004F0478000080FA002B
:10A5400000000600881F780000047800C27A02002C
:10A55000000000000004E000030032009900070042
:10A560000200010003003700B60007003E6B020046
:10A57000000000004F04780000000600E87A0200A6
:10A5800000000000000006000400FA00881F7800A8
:10A590009B000700E680570078760200000000006C
:10A5A0000000E0000800320098000700AA7A0200CC
:10A5B000000000000004E0000300320081000700FA
:10A5C00002000100030037009E0007003E6B0200FE
:10A5D000000000004F0478000080FA000000060030
:10A5E0000400FA00881F780085000700E680570005
:10A5F00078760200000000000000E0000800320051
:10A6000082000700B87A0200000000000004E000A9
:10A61000030032006B000700020001000300370056
:10A62000880007003E6B0200000000004F04780025
:10A630000080FA00000006000400FA00881F78007D
:10A640006F000700E68057007876020000000000E7
:10A650000000E000080032006C000700BE7A020033
:10A66000000000000004E000030032005500070075
:10A670000200010003003700720007003E6B020079
:10A68000000000004F0478000080FA00000006007F
:10A690000200FA00889FBE00560007000040EB0051
:10A6A000A0FF9F0066804000E6805700B87D020052
:10A6B000000000000000E00003003A002FF89700BF
:10A6C000205C9B0004003700110020000900780086
:10A6D0003E6B0200000000004F04BE000080FA0044
:10A6E00000000600889FBE004200070052E892006A
:10A6F0000004E0001D003200728091008288910009
:10A70000AA7A0200000000000004E0000C00320001
:10A7100018889100A8889100B87A02000000000013
:10A720000004E0000600320038889100C8889100DB
:10A73000B87A0200000000000004E00005003A00C2
:10A7400091002000090078003E6B0200000000002C
:10A750000A00370011C0B30071EC9A001901900093
:10A7600030042B00020001000400370081002000AB
:10A77000090078003E6B0200000000004F04BE009C
:10A7800000000600000006000000FA00881F7800A4
:10A79000CF19B00041E62F000184470024000700D4
:10A7A0008644020000000000880778004F0478000B
:10A7B0000080FA0000000600DC7D020000000000BE
:10A7C000000006001801900011C0B30030042B00F7
:10A7D0000000060005000900315878006000B10053
:10A7E00011C0B30061E99A001301900030042B00FE
:10A7F00000000600800478000204780000000600D3
:10A800000004780066804000000006003FB8970012
:10A81000CFB8970000000600620020008800780092
:10A8200000000600420020008800780000000600BA
:10A83000CD000900321C7800C819B100C219B1005E
:10A84000000006001100200008007800000006004B
:10A8500082057800514090000080FB0001FD2F0030
:10A8600001004000E10F4000000006008001780078
:10A8700052E892000004E00000000600E03890007A
:10A88000E269020000000000000006000000FA007B
:10A89000889FBE008A9FBE008C1F7800000678004B
:10A8A00000F890000080FB0001002000F00F500035
:10A8B000E08F5800CA013E00006001001000370020
:10A8C000C600370011013700240137003901370075
:10A8D00055013700C20137005F013700B80137006A
:10A8E0006201370065013700760137008F013700BC
:10A8F0009C013700A4013700A8013700B0013700E0
:10A900006CF890000004E000B50132006CF8900093
:10A91000E34F500014003A009F020700EC3890000B
:10A920000C007800E2690200000000004C5090002A
:10A930000018A30003003A000C00780078650200BC
:10A94000000000004C5090000014A1000903070013
:10A950000004A100405698000040EB0040DE980043
:10A9600060FE98009E0137006CF89000E64F5000A2
:10A9700009003A00CE020700E26902000000000070
:10A98000EE020700B069020000000000EE020700BE
:10A99000F0C0B3000B0037006CF89000E54F50009A
:10A9A00010003A00C2020700E26902000000000045
:10A9B000E2020700B069020000000000CC020700BC
:10A9C000D0C0B30000FE98000040EB0060FE98008D
:10A9D00088770200000000004086980051869800A9
:10A9E0007F013700ECF89000E1CF500003003A00FF
:10A9F000D702070001FE9800790137006CF890003B
:10AA0000E24F500037003A00A9020700E269020055
:10AA100000000000C9020700B06902000000000049
:10AA2000CB0207006C4891000008A3000B00320025
:10AA30000C8090000000E000080032000C3990000B
:10AA40009C399000AC02070004003200AE020700FF
:10AA500002003600040EE20005003200AA020700E0
:10AA600001003E00042EEF00AD0207005C0137003C
:10AA70000C3890009C3890000C8190007C2A90004B
:10AA80008C32900002014000E0814800840F5100A8
:10AA9000858F59000400360088020700203E980088
:10AAA000313E9800070037000C3990009C39900027
:10AAB0000C80900000004100E0804900203E98009A
:10AAC000313E980010002000207088002C38900043
:10AAD000BC3890003102070070C0B30000FE98003F
:10AAE0003F0137006CF89000E44F50003C013A0001
:10AAF0004C5090000018A300030032000040EB000F
:10AB000060FE9800360137000C3890009C389000A9
:10AB10004C02070013003A0023020700260032000F
:10AB200023020700E2690200000000008302070020
:10AB3000B0690200000000007D02070061005000C3
:10AB4000E08058001502070090C0B30000FE980096
:10AB5000887702000000000070A6980001AE9800FF
:10AB60001F0137001C019000AC0190006202070039
:10AB7000110031000E020700E2690200000000002F
:10AB80006E020700B06902000000000068020700C2
:10AB900061004000E080480000020700A0C0B30050
:10ABA00000FE9800887702000000000070A6980060
:10ABB00001AE98000A0137004C5090000004A1003B
:10ABC000405698005D020700B069020000000000D6
:10ABD0000040EB0000FE9800010137005C02070016
:10ABE0001C809000E20F500003003A004C5090008F
:10ABF0000044B200070032001C809000E10F5000BA
:10AC000007003A004C5090000068A3000400320096
:10AC10000040EB0060FE980000FE9800F000370056
:10AC20004C5090000014A000520207000024A10024
:10AC3000500207000004A000405698001C689000D5
:10AC40000004E0000C003A00CF0FB00040F02F00ED
:10AC5000008447007D0009003C1C7800C80FB1004B
:10AC6000CC0FB1006C64020000000000880778007F
:10AC70003E640200000000000D020700E2690200CD
:10AC8000000000002D020700B06902000000000073
:10AC90001C819000E20F51000E003A000A020700EA
:10ACA00005003D000B020700C50107002602070052
:10ACB00002FE9800CA003700E5010700803EB000A0
:10ACC0000180B000E401070040C0B30000FE98001E
:10ACD000C30037001C809000E10F500005003A00CF
:10ACE000DB010700DC01070050C0B30000FE980044
:10ACF000BB0037004C5090000024A0004056980044
:10AD00000C007800BB000700B5003700EE0107001B
:10AD1000B3003D0009020700B06902000000000016
:10AD2000A7010700BC089000F0442400808F500069
:10AD300004003A006009200001002000970107008C
:10AD400003003700803E200001002000930107002F
:10AD500030C0B30000FE9800A1003700C00107001A
:10AD60009F003A00D801070032003500F3010700C8
:10AD7000B069020000000000BC089000F04424000C
:10AD8000808F500004003A00A00F20000100200036
:10AD90008C01070003003700C05D20000100200087
:10ADA00088010700D201070040C0B30000FE9800F0
:10ADB0008B003700C401070005003D00800107003B
:10ADC000E30107000C00780012010700840037003F
:10ADD000750107007F003A000040EB0060FE98001C
:10ADE000DB0107004C509000B3CFB300034060007C
:10ADF000E0010700D2CFB30002406000DD01070090
:10AE0000E1CFB30001406000DA01070003406000B9
:10AE1000D801070002406000D60107000140600031
:10AE2000405698006E0037004C5090000068A30018
:10AE3000030032000C0078007C0007006800370037
:10AE40008701070063003A005D0107000C007800ED
:10AE5000F000070062003700810107005D003A0042
:10AE6000AF010700BA0107005D0037006CA0900039
:10AE7000E10F500037003A00030037006CA090004B
:10AE8000E20F500033003A00887702000000000013
:10AE900079010700D212230013002000820F500016
:10AEA000838F58004E003600A4010700B0690200ED
:10AEB000000000008B010700B0C0B30000FE980046
:10AEC000470037007101070003003A006CA09000B2
:10AED000E10F50001F003A006C0107000300320030
:10AEE0006CA09000E20F50001A003A005C010700CD
:10AEF0003500320088770200000000005E01070084
:10AF0000E270220073002000820F5000838F5800EF
:10AF10003300360089010700B0690200000000001C
:10AF2000C0C0B30000FE98002D0037005701070095
:10AF300003003A006CA09000E10F500005003A00B9
:10AF4000520107001E0032006CA09000E20F50007A
:10AF50001B003200100107000C00780025000700DC
:10AF60001F0037008877020000000000180107006A
:10AF7000B0690200000000001A010700020036005C
:10AF8000E0C0B30000FE9800350107000E0032005B
:10AF90006C4891000054A000604E99008877020030
:10AFA000000000000A010700B06902000000000074
:10AFB0000C0107000200360000C1B30000FE98003B
:10AFC0002701070003003A000C0078000900070081
:10AFD000030037006C4891000054A000604E9900B7
:10AFE0004F0678004F05BE004F04BE000080FA00F7
:10AFF00000000600881F780000047800E038900008
:10B00000E269020000000000FD0007000040EB00C4
:10B0100060FC980000FC9800080078007865020049
:10B02000000000004F04780000000600881F780030
:10B0300000047800A00090001000900030049800F8
:10B0400041049800E838900008007800E2690200A6
:10B05000000000004830900088007800B0690200CD
:10B0600000000000E6000700485090000024A10006
:10B07000405498000040EB0060FC980000FC9800F1
:10B080004F0478000000060031C0B30061F898005A
:10B090008040EB0001F8980000000600E0489100B5
:10B0A0000154A100614899000002EB0064809800FF
:10B0B00011C0B30001D898006011B80002389800A0
:10B0C0001338980041C0B30061F8980004F8980064
:10B0D00000000600E04891000154A1006148990079
:10B0E0000001EB006280980011C0B30001D8980005
:10B0F000702A90008032900004389800153898002B
:10B1000041C0B30061F8980002F898000000060002
:10B1100000027800A000900010009000820F500004
:10B12000838F58000800320010C0B30000DA980086
:10B13000023A9800133A980020C0B30060FA9800D1
:10B140000040EB0000FA980000000600881F78001D
:10B1500000047800405090000068A3000500320011
:10B1600008007800607C0200000000000004E0009D
:10B1700008003200684891000038A3000500320042
:10B1800010C0B30000DC980060FC98000040EB00A9
:10B1900000FC98004F0478000000060000017800D1
:10B1A00010C0B30000D9980010032000808F500019
:10B1B00009003A0002F89000EF4F50000100320001
:10B1C00002F8900050C0B30060F998000040EB0016
:10B1D00000F998000800370002F89000ED4F500089
:10B1E0000100320002F8900060C0B30060F99800DE
:10B1F0000040EB0000F998000000060010019000EC
:10B20000A0019000320098004300980079FF0700E9
:10B21000000006000000FA00889FBE008A9FBE0062
:10B2200080047800501090000088A30003003200D2
:10B23000495090000048A30015003A00950007000F
:10B24000CF0FB00040F02F000084470073000700CC
:10B250006C64020000000000880778003E64020071
:10B260000000000069009000F900900075000700E0
:10B270003F003A0079299000893190008301D10084
:10B280000281D30009007800A1FF07003C003700CD
:10B2900079F890000004E0002B003A0019007800D3
:10B2A000A9C99000F2CBB30082C141008381FB00A9
:10B2B0000080FB000000EA0003814100C202B000F0
:10B2C00062817C000280B900A20020001100090008
:10B2D0000200D800CF80DE00C219DD006303B00099
:10B2E0008981410033054000A385480079289000FA
:10B2F00089309000800F5500818F5D00020036007C
:10B30000792D90008935900049000700CF0FB000DB
:10B3100040F02F0000844700400007006C640200EA
:10B3200000000000880778003E6402000000000072
:10B330000A01BE000900780075FF070010C0B300C5
:10B34000C0DC98000E00370039000700CF0FB000B6
:10B3500040F02F0000844700300007006C640200BA
:10B3600000000000880778003E6402000000000032
:10B3700069019000F90190000900780064FF07005E
:10B3800010C0B300F0FC98004F05BE004F04BE0093
:10B390000080FA00000006007300070030069800E5
:10B3A00041069800000006006F00070025003700E6
:10B3B0004C5090000004A000405698003C0037001C
:10B3C0006000B800100698002106980000000600F2
:10B3D0000004BE004C859000DC8590005C000700F6
:10B3E000560037000A0454008B845C00404B2C004C
:10B3F00041002000800F5400818F5C000000060097
:10B40000485090000004A10040549800485090001B
:10B410000014A10040549800000006007D000900BF
:10B42000391C7800C80FB100C90FB1000000060038
:10B4300018000700495090000004A100C054980073
:10B4400000000600E00F5000E08F580000000600EA
:10B450002000070019003700DAFF0700240037003A
:10B460001C019000AC01900031000700800F5100DA
:10B47000818F5900000006007CA190008CA99000EB
:10B4800002005000838058000000060028000700DA
:10B49000ECFF3700495090000024A000C0549800F1
:10B4A000495090000014A100C0549800000006000C
:10B4B000DC3890000C007800000006007C2890002A
:10B4C0008C309000000006004C5090000004E0001A
:10B4D000000006002400070060069800710698002E
:10B4E000000006000C3890009C389000ABFF37003D
:10B4F0006000B800A9FF3700F0FF0700800F51007F
:10B50000818F5900000006000C3990009C39900092
:10B5100015000700800F5100818F590000000600C0
:10B52000F0FF070080C0B30000FE98000000060096
:10B530003C009000CC009000000006004C309000D1
:10B540008C00780000000600DCFF070093FF370046
:10B550006C4891000054A100604E99000000EB007F
:10B5600060869800000006001C009000AC0090006F
:10B5700000000600405698004C5090000000060065
:10B58000020007001F00070000000600889FBE00A1
:10B590008A1F7800EA010700440B02000000000047
:10B5A000F83F27007A7929005942270008007800DF
:10B5B000807802000000000000757C00E4010700B4
:10B5C000FAFF3A009ACBBF000080FB00B1B920001F
:10B5D000E201070005003A0096CBBF000080FB00A7
:10B5E00071B92000E201070003003200D401070016
:10B5F000440B0200000000004F0578004F04BE001D
:10B6000000000600889FBE008A1F7800620B2000A1
:10B610008000EB00C0BB2000440B020000000000D3
:10B62000F85F2700DA5B2900596B270008007800D3
:10B63000807802000000000000757C00C401070053
:10B64000FAFF3A00C0CBBF000080FB0011BC200015
:10B65000C201070005003A00BCCBBF000080FB0020
:10B66000D1BB2000C201070005003200620B2000A0
:10B670008000EB00C0BB2000440B02000000000073
:10B680004F0578004F04BE000000060000000600D1
:10B69000AB010700440B020000000000010007009E
:10B6A00000000600889FBE008A1F7800E0C2B30039
:10B6B0009CEBB70010C0B3009DEBB700F83F27002C
:10B6C0007A79290059422700EA407C000800780076
:10B6D000A4780200000000009D010700FAFF3A0074
:10B6E0004F0578004F04BE0000000600889FBE0092
:10B6F00062BC2000A301070071BC2000BC01070050
:10B700000282700082BC20009E01070091BC2000D4
:10B71000B70107008282700022BC20009901070057
:10B7200031BC2000B20107000284700042BC20003E
:10B730009401070051BC2000AD0107008284700015
:10B740000804420089844A0002032B00330E2000C3
:10B75000821F4400839F4C0081732A00811F780060
:10B76000520B020000000000E68757004F04BE00A5
:10B7700000000600C800FA00881F78000004780066
:10B78000C0732A00C7000900305F78008E0CB1003A
:10B790000E01780030F42400E16424000099BE001A
:10B7A00090742400000978000040EB006047980086
:10B7B0007701070002000100E0B92000801F780037
:10B7C00040802A00801F78000E007800520B020093
:10B7D000000000006E01070002000100B0CBBF00B6
:10B7E0000000FB00801F7800AFCBBF000000FB0013
:10B7F000801F780020812A00801F78000E007800CA
:10B80000520B02000000000061010700020001006D
:10B81000C1B92000620107009DCBBF004800DD00D8
:10B82000811F700010822A00801F78000E007800AF
:10B83000520B020000000000550107000200010049
:10B8400051BB200056010700B6CBBF004800DD0009
:10B85000811F7000F0822A00801F78000E0078009F
:10B86000520B020000000000490107000200010025
:10B8700011BB20004A010700B2CBBF004800DD0029
:10B880000101700031BB200045010700B4CBBF00AF
:10B890004800DD0081017000829FBE00D0832A0035
:10B8A000801F78000E007800520B0200000000009C
:10B8B0003701070002000100A1B92000380107008C
:10B8C0009BCBBF004800DD00811F7000B0842A00C0
:10B8D000801F78000E007800520B0200000000006C
:10B8E0002B0107000200010061B920002C010700B4
:10B8F00097CBBF004800DD00811F700050852A00F3
:10B90000801F78000E007800520B0200000000003B
:10B9100000FE2F00808747001D0107000200010084
:10B920001801900011C0B30000862A000200010037
:10B930004F0478000080FA0000000600C800FA00FA
:10B94000881F78000004780040862A00C70009009C
:10B95000305F78008E0CB10060942400C154240044
:10B96000008FBE000040EB00404798000801070030
:10B970000200010021BC200009010700C3CBBF0069
:10B980004800DD000101700041BC200004010700F7
:10B99000C5CBBF004800DD0081017000829FBE0062
:10B9A000C0922A00801F78000E007800520B02001F
:10B9B00000000000F600070002000100FB00070085
:10B9C000A5BC200004010700B4BC2000050107004D
:10B9D00005017200C5BC2000FF000700D4BC200098
:10B9E0000001070085017200809FBE00829FBE009B
:10B9F00090932A00801F78000E007800520B0200FE
:10BA000000000000E20007000200010001BC20006D
:10BA1000E3000700C1CBBF004800DD00811F7000BC
:10BA2000B0842A00801F78000E007800520B0200BC
:10BA300000000000D600070002000100C1BB20008A
:10BA4000D7000700BDCBBF004800DD00811F70009C
:10BA500050852A00801F78000E007800520B0200EB
:10BA600000000000CA00070002000100E1BB200046
:10BA7000CB000700BFCBBF004800DD00811F700076
:10BA800050942A00801F78000E007800520B0200AC
:10BA900000000000BE00070002000100E1BC200021
:10BAA000BF000700CFCBBF004800DD00811F700042
:10BAB00020952A00801F78000E007800520B0200AB
:10BAC0000000000000FE2F0080874700B000070044
:10BAD0000200010020BD2000801F780010962A007F
:10BAE000801F78000E007800520B0200000000005A
:10BAF000A7000700020001001801900011C0B30068
:10BB000000862A0002000100E48757004F047800F5
:10BB10000080FA00000006005601FA00889FBE006F
:10BB20008A1F7800B0AA2A0011000900305F78004F
:10BB30002E01B1000E007800ECFE07000000EB00C3
:10BB4000100F98004057980075004700B1A62A00D2
:10BB50003F000900315878000004B1000E0478005D
:10BB6000F2044700700547003800FB00801F780092
:10BB7000D2AB2A00821F780009007800520B020025
:10BB8000000000008900780075004700800B02006B
:10BB900000000000E48757008A0F5400F2FF3A00CB
:10BBA000580520000E044400B09E2A007F000900C2
:10BBB000305C78000808B100590D20008E844400E4
:10BBC000B1962A007F000900B15C78000908B10035
:10BBD00076000700809FBE0022AC2A00821F7800FA
:10BBE00008007800520B0200000000008E1F780051
:10BBF000881F7800C0AD2A00801F780009007800F7
:10BC0000520B02000000000021BD20007E00090050
:10BC1000B9587800F907B100516CEF0040C5B30086
:10BC2000C0EBB70010CBB300C1EBB70010C1B3003D
:10BC3000BEEBB70076404000BFEBB700A0CAB30030
:10BC4000BCEBB700BDEBB700E0C2B300CEEBB70072
:10BC500010C0B300CFEBB700F85F2700EC875700A8
:10BC6000DA5B2900596B2700EA407C000800780065
:10BC7000A47802000000000035000700FAFF3A0037
:10BC80004F0578004F04BE000080FA000000060057
:10BC9000889FBE008A9FBE008C1F78000105780037
:10BCA0004606DD00F07F2700000446008004EB001C
:10BCB0000B04200069417D000204E00007003A0007
:10BCC00009004600F17F2700010040008240780013
:10BCD000A4780200000000000D00370082407800C8
:10BCE00008007800A4780200000000008904E80041
:10BCF0000804E8008B8F5400EEFF3A00F083270021
:10BD0000000046008040EB00A47802000000000024
:10BD10004F0678004F05BE004F04BE00000006002D
:10BD20004600DD0001004000F17F270001004000D7
:10BD300080780200000000000000FB000000060008
:10BD4000620220008000EB0060B9200000000600C5
:10BD50000804E800890F54000000060024000700D2
:10BD60008080700040152B00808F5000000006007E
:10BD70001F00070080807000A0AA2A00808F50005A
:10BD800000000600124178000281FB00000006005E
:10BD90001801900011C0B3000E00780000000600EA
:10BDA000914078008180FB000000060065BC200007
:10BDB0000900070074BC20000A000700050072009B
:10BDC00085BC20000400070094BC2000050007008B
:10BDD0008500720000000600954278008582FB0015
:10BDE00000000600144278004822DD000000060032
:10BDF00091407800C808DD0000000600881F780028
:10BE000065044000C001070000132B00980B0200DE
:10BE100000000000610026000000E0007800320011
:10BE2000B901070070132B00980B020000000000FE
:10BE3000C10026000000E000710032004200200036
:10BE400088007800E0132B00980B0200000000002F
:10BE5000010B26000000E0006900320042002000D3
:10BE60008800780030142B00980B020000000000BE
:10BE7000A10926000000E0006100320072002000ED
:10BE80008800780080142B00980B0200000000004E
:10BE9000E10026000000E000590032009A0107008E
:10BEA00000152B00980B0200000000006102260024
:10BEB0000000E000520032009301070070152B00D3
:10BEC000980B020000000000A10626000000E00020
:10BED0004B0032007200200088007800E0152B0033
:10BEE000980B020000000000C10D26000000E000D9
:10BEF00043003200520020008800780060162B00BA
:10BF0000980B020000000000010F26000000E00076
:10BF10003B0032007C010700C0162B00980B02008A
:10BF200000000000610F26000000E0003400320035
:10BF30007501070030172B00980B0200000000006D
:10BF4000E11126000000E0002D0032006E01070024
:10BF5000A0172B00980B02000000000061152600BE
:10BF60000000E000260032006701070010182B00D7
:10BF7000980B020000000000A11926000000E0005C
:10BF80001F003200720020008800780080182B000B
:10BF9000980B020000000000211B26000000E000BA
:10BFA00017003200820020008800780000192B0062
:10BFB000980B020000000000811B26000000E0003A
:10BFC0000F0032005001070090192B00980B02005F
:10BFD00000000000C11C26000000E0000800320044
:10BFE00049010700001A2B00980B02000000000016
:10BFF000412126000000E000010032008000EB003B
:10C00000010078004F04780000000600BA5B0200CF
:10C010000000000000000600000006000041EB00E8
:10C02000E1409000E1CF500001003A00014178006A
:10C030000001FD00B7EBB7000001FD00100190000A
:10C040002601070002000100000006000400FA00BB
:10C05000881F7800240107008E1F7800B11A2B007A
:10C06000811F7800BA0B020000000000E48757002F
:10C07000E10F500006003A001E01BE00F02324002C
:10C08000F1002000800F5100818F5900040036001C
:10C090001A0107003E6B0200000000000A00370092
:10C0A00002007800B1EBB7004810DE00B2EBB70039
:10C0B00003007800B3EBB7004818DE00B4EBB7001C
:10C0C00004010700020001004F0478000080FA001C
:10C0D000000006000400FA00881F78000201070033
:10C0E0008E1F7800B11A2B00811F7800BA0B020056
:10C0F00000000000E4875700E10F50000400320008
:10C10000FE0007003E6B0200000000000600370042
:10C110001E407800B5EBB7001E409000B6EBB700AC
:10C12000EC000700020001004F0478000080FA00D4
:10C1300000000600881F780000047800E4804000BA
:10C1400012012000E0B92000D60B02000000000020
:10C15000E0000700020001004F0478000000060024
:10C16000889FBE0080047800648440000800780046
:10C170008E740200000000000004E000080032009D
:10C1800018407800AFEBB70018409000B0EBB70054
:10C1900019019000D10007000200010004003700DF
:10C1A000A1002000090078003E6B020000000000A2
:10C1B0004F04BE0000000600881F780000047800CD
:10C1C000525B0200000000001801900011C0B30093
:10C1D000F01A2B00020001004F0478000000060056
:10C1E000485B02000000000000000600000178002B
:10C1F000E140900010C3B30080CF500008003A0027
:10C2000040C5B3009AEBB70010CBB3009BEBB7006F
:10C210006740500096EBB70097EBB700030037007C
:10C220000040EB0096EBB70097EBB70012019000CF
:10C23000AA00070002000100000006000400FA0046
:10C24000881F7800A80007008E1F7800B11A2B0005
:10C25000811F7800BA0B020000000000E48757003D
:10C26000E10F500004003200A40007003E6B020002
:10C27000000000000A0037001E407800C2EBB70043
:10C280001E409000C3EBB7001E009000C4EBB70047
:10C290004800DE00C5EBB7008E0007000200010079
:10C2A0004F0478000080FA00000006000400FA0045
:10C2B000881F78008C0007008E1F7800B11A2B00B1
:10C2C000811F7800BA0B020000000000E4875700CD
:10C2D000E10F500004003200880007003E6B0200AE
:10C2E00000000000100037001E00BE00C6EBB700C3
:10C2F0004802DE0004007800C7EBB70001007800B8
:10C30000C8EBB7004808DE00C9EBB7000000EB003F
:10C31000CAEBB700CBEBB700CCEBB700CDEBB70067
:10C320006C000700020001004F0478000080FA0052
:10C3300000000600881F780000047800E6804000B6
:10C34000F207200020BD2000D60B020000000000F4
:10C35000526CEF005F000700020001004F047800FC
:10C36000000006009E5C02000000000000000600C5
:10C37000881F7800000478008C5D02000000000037
:10C380001801900011C0B300F01A2B000200010048
:10C390004F047800000006000600FA00889FBE00E7
:10C3A0008004780001047800000FEB0061409000E9
:10C3B000004F780071409000104798006000B8006E
:10C3C00010079800210798008E9FE800B01A2B00F4
:10C3D000801F78000E007800BA0B020000000000F9
:10C3E000E4875700E10F50000500320011002000E3
:10C3F000090078003E6B02000000000007003700D3
:10C40000E80044001E009000485E020000000000AA
:10C410001901900031000700020001004F04BE0026
:10C420000080FA00000006004200FA00889FBE006B
:10C430008A9FBE00800578008004EB000A0420007B
:10C4400060FB2F000F004000511B2B004000090033
:10C45000315878001004B1000004EB008800780027
:10C4600009007800905E02000000000061FB2F00D0
:10C470008F80400080707C000004E00006003A00DD
:10C480001B01900011C0B30060FB2F000F004000A3
:10C49000020001000B0037000804E8008A0F540076
:10C4A000EEFF3A001B0190008040EB0060FB2F0084
:10C4B0000F004000020001008904E800F08F5400E2
:10C4C000DFFF3A004F05BE004F04BE000080FA00B7
:10C4D00000000600180190000000370011C0B300F2
:10C4E000701A2B000000060000047800000FEB001B
:10C4F0003E17780066804000000006001100200012
:10C500000800780000000600620020008800780023
:10C51000000006005050210001002000C4D020007F
:10C5200045D520004509DD00CB01DE008301710007
:10C530004501DD000001410081814900344078005F
:10C540000080FB00010020000200400083804800C2
:10C55000850F5200F3FF3A0000000600889FBE00DE
:10C560008A9FBE000005BE000278020000000000A5
:10C570002A6890008F000700C1D5200079010700CC
:10C580005DCDBF004800DD0001047000E1D5200052
:10C59000740107005FCDBF004800DD00810470001A
:10C5A000DCFF0700800F5400818F5C007D003A00A3
:10C5B000D0D0200011C0B30090CF100079003A0015
:10C5C00078004500E2D020001000090032587800C1
:10C5D0001001B100C00220000A0040000269800082
:10C5E000136980000298BE002269800033698000D0
:10C5F0000298BE00436980000308780060032000B1
:10C600000A00400052698000636980000298BE0001
:10C6100072698000836980000298BE00936980007F
:10C62000030878001FCDBF0020CD98004BCDBF0080
:10C630000140600040DD980001DD980021D4200019
:10C64000914078006155980032D420001241780062
:10C650007255980041D420004201070045CDBF002B
:10C660004800DD000100700000859800B1D4200072
:10C67000914078008100D100E18060006A4891001B
:10C680000004A10001407000604D990091D4200089
:10C69000340107004ACDBF004800DD0001007000F2
:10C6A0007035980063D4200093417800E34D9800E2
:10C6B00001D6200091407800214D98008180FB0038
:10C6C000C208DD0000D620008080400011429000AA
:10C6D0000482FB00214090004800DD00040170004E
:10C6E000314290000482FB00414090004800DD0090
:10C6F000840170006205980073059800B1D4200091
:10C7000091407800C608DD000110B2005A10900078
:10C710000080A10001007000501598004BCDBF00B3
:10C720004400DE0061006000106D9800E1D320003D
:10C730000C0107003FCDBF004800DD000101700083
:10C7400001D420000701070041CDBF004800DD00F3
:10C750008101700012359800233598004BCDBF0041
:10C760004300DE00610060004400DD00EA48910003
:10C770000144A10080C07000614D99004BCDBF0005
:10C780004500DE00610060004200DD00CA509000FC
:10C790000124A10080C07000415598000000EB000A
:10C7A00001003700100020004F05BE004F04BE00FE
:10C7B00000000600889FBE008A9FBE00EC000700B4
:10C7C00008C04400367802000000000000F47D003C
:10C7D0000804E8008A0F5400F9FF3A004F05BE0034
:10C7E0004F04BE00000006000400FA00889FBE004F
:10C7F0008A1F780080047800A1C0B300E1F79F0091
:10C800000040EB00F0F79F0081FF9F0090FF9F002A
:10C810000004EB00014578000840780036780200FB
:10C82000000000000004E00002003A008AFF9F00C0
:10C830000100370080FF9F00E88057000900780062
:10C84000800B0200000000000804E800F00F200048
:10C85000800F5400F0FF3A00EA805700090078008A
:10C86000800B0200000000004F0578004F04BE005E
:10C870000080FA000000060000000600881F780013
:10C8800018C0B3000004FD000DEDB7000004FD006A
:10C8900020FF07005CEDB7004801DE0002007800D1
:10C8A0005DEDB700010078005EEDB7004808DE00DE
:10C8B0005FEDB70008407800800007004F04780063
:10C8C000000006000000FA004FE8940046EDB700B3
:10C8D0000080FA00000006000000FA0000C0EB0033
:10C8E00061EDB70062EDB70063EDB70064EDB7002E
:10C8F00065EDB70066EDB70067EDB70068EDB7000E
:10C9000069EDB7006AEDB7006BEDB7006CEDB700ED
:10C910006DEDB7006EEDB7006FEDB70070EDB700CD
:10C9200071EDB70072EDB70073EDB70074EDB700AD
:10C930006683570044F02F0004024300E64A960045
:10C9400036019700C60197000580FB008C000700A8
:10C950000500780060EDB700C4D89000E1C0600029
:10C960004BCDBF000004A100014070004BEDB700AB
:10C9700014309000A43090003EEDB7004801DE0076
:10C98000020078003FEDB7000100780040EDB700ED
:10C990004808DE0041EDB70010C0B3000DEDB70050
:10C9A00078004200E1D0200010000900B058780063
:10C9B0001001B100C0022000040040003001BE00A0
:10C9C00002698800136988003001BE00226988006E
:10C9D00033698800100078004069880060032000F7
:10C9E000040040003001BE0052698800636988007D
:10C9F0003001BE00726988008369880010007800E9
:10CA00009069880024C890001FEDB7002658960052
:10CA100042EDB7003658960043EDB7000480900011
:10CA200044EDB7004800DE0045EDB70064489100D2
:10CA30006140600000404000B1D420009140780087
:10CA40000114A10058000700541090004800DE00B7
:10CA5000614060004200DD000124A1005200070097
:10CA60007430900049EDB7004800DE004AEDB70091
:10CA7000644891004400DE00610060004300DD0076
:10CA80000134A10048000700146890006140600074
:10CA90004400DD000144A100430007000658960051
:10CAA0004200DE00610060004500DD000154A1008D
:10CAB0003D0007000080FA0000000600889FBE00CD
:10CAC0008A9FBE002A000700E8C07D0008C044001D
:10CAD0005A780200000000000804E8008A0F5400A1
:10CAE000F9FF3A004F05BE004F04BE0000000600EB
:10CAF000889FBE008A1F7800800478001001900093
:10CB0000A0019000204890000080FB001C0007005E
:10CB10000004EB000AD62000E8407D002968900060
:10CB20004045B000084040005A7802000000000074
:10CB30000804E800E40F5400F7FF3A000040EB005F
:10CB4000A04C98004F0578004F04BE00000006007E
:10CB50000D6DEC0020689000D8FF07000000060073
:10CB600000000600914078008180FB000000060074
:10CB7000804478000004EB00CBD020009A0605002A
:10CB80004200DD0001D62000010040001240980064
:10CB9000C810DE002140980033409800C818DE001D
:10CBA000414098000000060080C07000010078003D
:10CBB0004BEDB700000006008000EB006118980004
:10CBC000110A880042E1A800211420009140780059
:10CBD00082CFB30082C060000104A0008000FD008D
:10CBE00042E1B7008000FD008420A9009420A80045
:10CBF000410A2000914078000144A1000146B300A1
:10CC00008000FD00A4E0B7008000FD00B06F880048
:10CC100000000600809FBE00821F780042C1BF0056
:10CC20000048A30002003A0005003700000A800017
:10CC300042C1BF000038A300FCFF3A001B003700D0
:10CC4000F80DEC00C06F8800E50F500018003A00A6
:10CC5000B26F8000624090000004E00010003200DB
:10CC6000CBC2BF000068A30003003A00E000070049
:10CC7000000A800002003700000A8000DC00070084
:10CC800011C0B300B06F8000714098008040EB008D
:10CC9000B06F80006140980004003700000A8000F7
:10CCA00042C1BF000038A300FCFF3A00F82DEF009E
:10CCB0008420A9004F0178004F00BE00004006000C
:10CCC0000800FA00889FBE008A9FBE008C9FBE00AD
:10CCD0000006780010007800E10F50001D003200BF
:10CCE000E20F50005C0032008000EB00110698005B
:10CCF0007C4090000004E0000E0032007146980075
:10CD0000CA00070040062000800F54000D003600C6
:10CD1000A00F2000808F50000A003600F0E12400B0
:10CD2000808F500007003E0010002000000E7800A9
:10CD3000040037006C409000E14F500001003200C9
:10CD4000DA0007000000EB0050069800400698004B
:10CD5000A20037007C4090000004E0009400320004
:10CD60008006EB004D0698007D469800AF00070056
:10CD700030062000800F540003003E002D0698006E
:10CD80001D0698001D003700900F2000808F500076
:10CD900004003E000000EB002006980010069800FA
:10CDA00016003700703E2000808F500005003E00C6
:10CDB0001C0090002006980020002000100698001B
:10CDC0000E00370070442F000080400061262400D0
:10CDD000810F500005003E001C00900020069800C6
:10CDE0001000200010069800040037001C0090007E
:10CDF000200698000000EB00100698009C009000B0
:10CE00002C009000808F5000020032000000EB00E8
:10CE1000500698001C0090000000E0000A0032005C
:10CE2000DC0090000100E80050069800F38F5000ED
:10CE30006A00360020002000000E7800A0002000CC
:10CE400050069800650037000000EB00500698007F
:10CE5000000E7800610037007C4090000004E00084
:10CE6000530032000000EB00400698007046980026
:10CE70008E0007000C0C90009C0C90006C00900041
:10CE8000FC0090000000540081805C008A000700D4
:10CE9000000578002C089000BC08900008005000A5
:10CEA000898058008400070000047800800645004F
:10CEB00030062000800F540036003600900F20000E
:10CEC000808F560033003600703E2000808F560061
:10CED00012003E001C009000E20F50002D003A00AE
:10CEE00066000700E0B79F00F1B79F000800E00070
:10CEF00003003D0064000700E0B79F00F1B79F000A
:10CF00006500070001003D005F0007000001BE0052
:10CF10006FB09700FFB097001600370070442F00E5
:10CF20000080460061262400810F500019003E0059
:10CF30001C009000E10F500016003A004F0007005F
:10CF400080BF9F0091BF9F000800E00003003D00EC
:10CF50004D00070080BF9F0091BF9F004E0007005B
:10CF600001003D00480007000001BE000FB8970017
:10CF70009FB8970068070200000000004026980054
:10CF8000512698006D269800A000200050069800B9
:10CF9000030037005C0090000000E9005006980094
:10CFA0005C009000E50F50000C003E000A003700C6
:10CFB0006C409000E14F5000010032003B00070040
:10CFC0004C0090008000E80041069800F1702200BB
:10CFD000810F500001003600000EEB004F06BE002E
:10CFE0004F05BE004F04BE000080FA00000006009E
:10CFF000000A800001002000600198007101980083
:10D00000000A800001002000B26F80000009980033
:10D0100011099800000A800001002000B26F800012
:10D020002009980031099800000006001F00070041
:10D030000C0D90009C0D90002C089000BC089000F6
:10D040000A0050008B8058001B0007000004BE003F
:10D050006C009000FC0090000005550081855D008B
:10D06000F2FF2F00030020000A00BE002E0802007D
:10D070000000000080004400000006006140B9008C
:10D08000560604000000000002002000037824007F
:10D09000AE060400000000006150B9005606020010
:10D0A000000000000A00E0000000060010C0B3000D
:10D0B0006046980000000600F2FF2F0003002000E9
:10D0C0002E08040000000000406F8800516F8800A7
:10D0D000411820009140780082CFB30082C06000E8
:10D0E0006140B3008000FD0084E1B7008000FD00D6
:10D0F0008461A800D022A900D002A900A1182000B4
:10D100009140780082C060006140B3008000FD0063
:10D110008AE1B7008000FD008A61A800A11120000B
:10D1200021809800C1112000506F8000218098005C
:10D1300001182000406F80003180980061182000A5
:10D14000506F800031809800406F80008000EB00BD
:10D150009C000700506F80008000EB0099000700E2
:10D160009760A8009780A80000000600436F800029
:10D17000634891000058A30009003200BA0007007C
:10D1800009003100BE000700416F8000413090006F
:10D19000618190000200400071000700020037002A
:10D1A0000000EB00E081980000000600536F800053
:10D1B000634891000058A30009003200AA0007004C
:10D1C00009003100AE000700516F8000413090002F
:10D1D00061819000020040006100070002003700FA
:10D1E0000000EB00E0819800000006003600F80027
:10D1F000809FBE00829FBE00849FBE00869FBE00AF
:10D20000446F8000A300070004003A0044509000DF
:10D210000004A10040529800470037009D0007001D
:10D220002000360041DF20009140780020C4B30088
:10D2300080CF50000C0032000040E80080CF50004A
:10D240000B00320000C0E90080CF50000E003A0011
:10D25000C422A800C402A9000000000063404000EE
:10D26000F4EDB70009003700910007000700370010
:10D27000C422A900C402A8000000000020C4B3001A
:10D28000F4EDB700010037008F000700426F800007
:10D2900012009000A200900061005000E080580051
:10D2A0001F00370041DF20009140780022C4B30006
:10D2B00082CF50000C00320030C4B30080CF500049
:10D2C0000B00320000C0E90080CF50000E003A0091
:10D2D000C422A900C402A8000000000002007800D7
:10D2E000F4EDB700090037007700070007003700AA
:10D2F000C422A800C402A9000000000040C4B3007A
:10D30000F4EDB7000100370069000700426F8000AC
:10D3100012009000A200900061004000E0804800F0
:10D320001001980021019800416F80004150900049
:10D330000004A000C05098008CFF07008760A9007F
:10D340004F03BE004F02BE004F01BE004F00BE00A3
:10D350003600F900004006008780A9000040060062
:10D36000889FBE0080047800010478000000E0007F
:10D370000D00320021F89100340007006149B80027
:10D3800000A02500212620009405020000000000D6
:10D390004809DD004800DE0000007100C808DE001A
:10D3A000800078000300370021F89100200007007A
:10D3B0008080EB0028809000010878004F04BE00B8
:10D3C000000006000002780081017800C0252000DE
:10D3D000808F500004003600B4809000500620007A
:10D3E0008008780011003700400620000088B9004E
:10D3F000D2252000110009000280D8008000FD0025
:10D400000300E0000300320034809000010878003F
:10D4100002003700348090000008EB00401F20001D
:10D42000000000000000E900FDFF3A0000000600D7
:10D4300011C3B300814F500002003A009760A90069
:10D44000010037009780A9000000060011C3B30057
:10D45000814F500002003A009760A8000100370099
:10D460009780A8000000060063809000C330900001
:10D470003331900001004000820F50000000060090
:10D4800063809000916F800001004000E08198006F
:10D490000000060014019000A401900034009000E8
:10D4A000C4009000800F5100818F590000000600D9
:10D4B000C422A800C402A8000000000010C4B300E9
:10D4C000F4EDB70000000600C422A900C402A900C0
:10D4D0000000000030C4B300F4EDB7000000060007
:10D4E000E10F50000D00320020D72A00801F780085
:10D4F00070042000801F780040D72A00801F780029
:10D5000090D82A00801F7800E0EE2000040C020072
:10D5100000000000500C0200000000009C7C020093
:10D5200000000000E1CA27001100980041CB27004D
:10D5300021009800C1CE27003100980000000600AD
:10D540000400FA00889FBE008A9FBE008004780015
:10D550000105780020009000000001000004E000B8
:10D560002D00320039009000000001000004780016
:10D570008A00780040740200000000000005780076
:10D580000000E00004003A00D1002000090078000B
:10D5900077000700200037000800780006740200BA
:10D5A00000000000800578000000E00004003A0060
:10D5B00031002000090078006D00070016003700D8
:10D5C0006C80570071DA2A00030009003158780096
:10D5D0004000B100B840900010C2B30080CF5000AE
:10D5E00005003200E3004400220020006C80570058
:10D5F000580C0200000000001901900011C0B30097
:10D600006C80570002000100E50044000A01780028
:10D61000090078000B0001004F05BE004F04BE005A
:10D620000080FA00000006000102780090019000DE
:10D630000300E0000D003A00B0DA2A00801F7800F5
:10D64000F0062000801F780040D72A00801F780055
:10D6500090D82A00801F7800E0EE2000040C020021
:10D6600000000000500C0200000000008240780022
:10D67000040078000300010000000600C000FA006A
:10D68000889FBE008A1F7800820007000D003A00C4
:10D69000B0DA2A00801F780061072000811F78001F
:10D6A00042D72A00821F780090D82A00801F780075
:10D6B000E0EE2000040C020000000000500C02000C
:10D6C00000000000A1F32F008F804000B2DF2A008D
:10D6D00075000700B1DB2A003F000900315C7800CB
:10D6E0000804B100891F7800B2E72A00821F780081
:10D6F00008007800520B020000000000880078004B
:10D7000060F32F000F004000800B020000000000BB
:10D7100009007800687B020000000000801F78008C
:10D7200020E82A00801F780008007800520B0200D1
:10D73000000000008800780020F32F000F00400058
:10D74000800B0200000000001A01900011C0B3001D
:10D7500020F32F000F00400002000100E88757006F
:10D760004F0578004F04BE000080FA00000006005C
:10D77000C000FA00889FBE008A1F7800450007009D
:10D780000D003A00B0DA2A00801F7800310820002E
:10D79000811F780042D72A00821F780090D82A0083
:10D7A000801F7800E0EE2000040C02000000000062
:10D7B000500C020000000000A1F32F008F804000F9
:10D7C00062EC2A003800070061E82A003F000900E7
:10D7D000315C78000804B100A0F32F000F00400076
:10D7E0007C0C020000000000A2F32F000F0141009A
:10D7F0000000410011C2B30001587800A1C0B3007D
:10D80000015878000048EB00891F7800B0E72A0033
:10D81000801F780008007800520B02000000000012
:10D820008800780060F32F000F004000800B02009A
:10D830000000000009007800687B02000000000082
:10D84000801F780021E82A00811F780008007800F6
:10D85000520B0200000000008800780020F32F0027
:10D860000F004000800B0200000000001A01900031
:10D8700011C0B30020F32F000F0040000200010090
:10D88000E88757004F0578004F04BE000080FA007B
:10D890000000060000057800810478001000900068
:10D8A0000000E000000006007F000900B258780088
:10D8B0000108B100010478000808B000000006006B
:10D8C00011C0B30001D898008000EB001128980027
:10D8D00000000600881F78008A9FBE0000047800C0
:10D8E00040D890000004E0000D003A001828900095
:10D8F0000000E000D40032000000EB00102C980083
:10D9000018009000A8009000D2000700E8389000AE
:10D9100008007800E269020000000000CA00370039
:10D92000485090000048A3000D003A0018289000CD
:10D930000000E000C40032000000EB00102C980052
:10D94000D10007003204980043049800E8389000A2
:10D9500008007800E269020000000000BA00370009
:10D96000485090000028A300B700320048509000B3
:10D970000068A3000500320008007800607C020007
:10D98000000000000004E000AF00320008D8900062
:10D99000E14F500002003A0010002000102C9800C7
:10D9A00018289000E20F50003300320005003E00BE
:10D9B0000000E00008003200E10F5000A2003A0031
:10D9C0000D003700E30F500043003200E40F500019
:10D9D0009D003A008C00370048D89000E14F50007D
:10D9E00099003A000000EB00502C98001000200035
:10D9F000102C980094003700A3000700980007003F
:10DA00009A00070019003A00582890000000E8002A
:10DA1000502C980041062000810F50008A003400ED
:10DA20000000EB00502C980098017800032C98001F
:10DA300095000700622498007324980000DC980089
:10DA40008877020000000000202C9800312C9800FC
:10DA50004830900088007800B069020000000000A3
:10DA600020002000102C9800770037000000EB0009
:10DA7000502C98007400370008007800D07B02001A
:10DA80000000000080000700020050008380580062
:10DA900033062000830F5000E08F580002003C0046
:10DAA000683090000100370058309000247C02005C
:10DAB0000000000028299000B829900000004100D3
:10DAC00081804900202C9800312C980030002000E3
:10DAD000102C98005C0037008877020000000000DE
:10DAE00028299000B8299000820F5000838F580099
:10DAF0005500390008007800D07B020000000000CB
:10DB00006100070002055000838558004240A900CB
:10DB10001900340058D890000004E00008003A00D2
:10DB20005500070051000700340032004C00070088
:10DB300061004000E0804800460007002F003700E9
:10DB40004D0007000A0050008B8058004700070076
:10DB50002A003100D838900008007800E2690200FD
:10DB6000000000003E0007000A0040008B804800D3
:10DB70003800070021003700E00F5500E08F5D00FE
:10DB80001E003D0058D890000004E0000A003A0052
:10DB900018009000A8009000E00F5000E08F58009F
:10DBA000160032002E00070061005000E08058008F
:10DBB000280007001100370018029000A80290000A
:10DBC0000081EB000250B8000A8150008B00510028
:10DBD000800F5200818F5A0008003600D83890001C
:10DBE00008007800E2690200000000001C00070045
:10DBF0000000450081804D00160007004000200015
:10DC0000102C98001000370038019000C8019000D7
:10DC100018009000A8009000140007000A003A00C5
:10DC2000E838900008007800E26902000000000077
:10DC300020002000102C98008877020000000000CF
:10DC4000202C9800312C98004F05BE004F0478001E
:10DC5000000006003004980041049800000006000F
:10DC600038009000C800900000000600800F5100AE
:10DC7000818F5900000006000300070078289000FB
:10DC8000883090000000060018019000A801900064
:10DC9000000006000400FA00889FBE008A9FBE00B4
:10DCA0008C9FBE0080067800891F2000808444007D
:10DCB00009007800283C0200000000000D067800F2
:10DCC0000D007800F831020000000000C00F2000B5
:10DCD0000080460010079800F831020000000000A4
:10DCE000000920000D004000DC650200000000007B
:10DCF0000D007800087E0200000000001E00900069
:10DD0000087E02000000000010C0B300A06E980062
:10DD100080CCB300E0669A00890078000D0078009E
:10DD2000AE6202000000000000047800C05A020049
:10DD3000000000008045EB00E10F54003A003A007B
:10DD40000D0078003A320200000000001E00900032
:10DD50003A32020000000000090078005A3C02003C
:10DD600000000000CF0FB00049F02F0009844700E9
:10DD7000920007006C640200000000008807780031
:10DD8000C00F200000804600000F7800CF0FB000C9
:10DD9000098447008E0007006C6402000000000048
:10DDA000880778008B1F20008D854500CF19B000B3
:10DDB0004AE62F000A8447008A00070062640200D6
:10DDC00000000000880778003E64020000000000A8
:10DDD000CF0FB00009844700780007006C64020090
:10DDE0000000000088077800CF0FB00009844700CA
:10DDF0001E007800760007006C640200000000003E
:10DE000088077800CF19B0000A8447007500070022
:10DE10006264020000000000880778003E6402008F
:10DE2000000000001BC0B30019C0B300A9FE990098
:10DE30002AC0B300EAF69B0009407800186A020085
:10DE4000000000000A407800186A0200000000008C
:10DE50000B04FB00880078000C0078002F000700FE
:10DE6000880078001E0090002C0007009E009000A3
:10DE70000C0078006468020000000000094078008F
:10DE8000266A0200000000000A407800266A0200AC
:10DE900000000000602020000D00400010407800CD
:10DEA000F67D0200000000006D4891000038A300DC
:10DEB000090032001D6890000004E00003003A00F1
:10DEC0004D5090000028A30003003A000C00780099
:10DED000A6580200000000002D4893000038A3005F
:10DEE000090032005D6092000004E00003003A0087
:10DEF0000D5092000028A30003003A001E0090007D
:10DF0000A6580200000000004F06BE004F05BE00EC
:10DF10004F04BE000080FA0000000600889FBE008B
:10DF20000004BE00187E0200000000006848910056
:10DF30000068A3000900320018309000A83090005B
:10DF4000E00F5000E08F58000400320018309000BD
:10DF5000A8309000702C9800013498000900E0006F
:10DF600008003A0068009000F80090001004980043
:10DF70002104980068009000F80090003004980098
:10DF800041049800080078003E54020000000000A0
:10DF900008007800606C02000000000068489100F2
:10DFA0000038A30003003A00485090000024A0006D
:10DFB000405498004F04BE00000006007D00090098
:10DFC0003D1C7800C80FB100CD0FB1000000060065
:10DFD0007D000900301C7800C80FB100C00FB100EF
:10DFE00000000600CD0009003B1C7800C819B100F4
:08DFF000CB19B100000006008E
:020000040000FA
:10DFF800000800009603000000000000FE0D00006D
:10E00800020000000200000000000000CC0D00002B
:10E018000E00000000000000000E000002000000DA
:10E028000200000000000000960B0000DC00000069
:10E0380000000000760D000036000000020000001D
:10E0480000000000000000000000000000000000C8
:10E0580000000000000000000000000000000000B8
:10E0680000000000000000000000000000000000A8
:10E078000000000000000000000000000000000098
:10E088000000000000000000F20D00000400000085
:10E09800020000000100410000000000E40D000043
:10E0A8000800000000000000F60D00000400000059
:10E0B80000000000FA0D000004000000000000004D
:10E0C800EC0D00000600000000000000720C0000CB
:10E0D8009A00000000000000AC0D000020000000C5
:10E0E80002000000E4AA1200AB3DAB005BAB740079
:10E0F800ABA2AB00CFABFF00AB33AC005AAC8F0088
:10E10800ACAEAC00CCAC0000AD36AD005AAD0000F2
:10E11800020E0000020000000200000000000000E3
:10E12800040E0000020000000200000000000000D1
:10E13800060E00000200000000000000DA0D0000DA
:10E148000A000000020000000000000000000000BB
:10E158000000020000000000080E0000020000009D
:10E16800020000004B0000000C0D00006A000000D7
:10E1780000000000D40E000026000000020000008D
:10E18800D60E08000F000000080F0900000000006C
:10E19800020006000F000000060F06000201000042
:10E1A800000000000000000000000600020200005D
:10E1B80000000000060F000006000000000000003C
:10E1C800FA0E00000C000000000000000A0E00001B
:10E1D800A000000002000000010000000000000094
:10E1E80000000A00000000000000000000640000B9
:10E1F8000000000000000000E8030000000000002C
:10E2080000001000270000000000000000A08600A9
:10E21800010000000000000040420F000000000064
:10E228000000800096980000000000000000E10057
:10E23800F50500000000000000CA9A003B0000003D
:10E2480000000000E40B5400020000000000E80099
:10E2580076481700000000000010A500D4E8000070
:10E2680000000000A0724E001809000000004000E5
:10E278007A10F3005A0000000080C600A47E8D00CA
:10E288000300000000C16F00F286230000000000B8
:10E298008A5D78004563010000006400A7B3B600FA
:10E2A800E00D000000E889000423C7008A00000090
:10E2B800AA0E00002A00000002000000286E750067
:10E2C8006C6C2900003031003233340035363700A9
:10E2D800383941004243440045460000303132009D
:10E2E80033343500363738003961620063646500BD
:10E2F800660000000C0F0000020000000000000093
:10E308000E0F00000200000000000000100F0000C7
:10E318000200000000000000120F000002000000D0
:10E3280000000000140F00000200000000000000C0
:10E33800160F0000020000000200000001000000AB
:10E34800180F00000200000000000000000000009C
:020000040000FA
:10E35800000000000000000000400600000000006F
:10E3680000000000004006003400FA001D0007000D
:10E378002C77020000000000207E02000000000050
:10E38800C1FC2F008F804000008020004A6E0200F0
:10E398000000000010002000706A02000000000069
:10E3A800A05C8800E87D020000000000A05C8000FE
:10E3B80001802000A06A0200000000000080200008
:10E3C8006E33020000000000C08F20006E33020090
:10E3D80000000000809F2000603C02000000000058
:10E3E800F0FF37000001EB00223A8800800220008D
:10E3F800303A880044C7BF0003CEB3000340600032
:10E4080044E7B70044C7BF00F043B20044E7B70091
:10E41800820888001021A90010C1BF00F1CCB30008
:10E42800014060000054A00010E1B70011A1A8004D
:10E438008082EB006508880011E1A8009208880036
:10E448001221A90012C1BF000140600012E1B7000B
:10E4580013A1A800400620007008880013E1A80056
:10E46800F20888001E21A9001FA1A80004C3B30058
:10E47800044078001E61B7001FE1A800B1C0BF00CA
:10E48800F1C8B300014060000045B300B1E0B70037
:10E498008760A900020988002021A90021A1A800FD
:10E4A800044078002061B700C208880030B72C000B
:10E4B800E0088800B2C0BF0081CFB300014060000F
:10E4C8005040B300B2E0B7008780A90021E1A8005E
:10E4D8002216880062168800A21688000216880094
:10E4E800421688008216880065198800C9C2A800EB
:10E4F800C942A8008EC6BF0003406000E040B300D8
:10E508008EE6B7008FC6BF0003406000A040B3008E
:10E518008FE6B700C0E2A800C962A800C022A9001F
:10E52800C002A900C142A900C9A2A900C9E2A90064
:10E53800C982A900CFC6BF00034060002041B300D4
:10E54800CFE6B700CCC6BF00034060003041B3003F
:10E55800CCE6B700C3C6BF00034060004041B3002B
:10E56800C3E6B700D122A800D0C2A800A4C6BF0045
:10E57800034060009041B300A4E6B700A6C6BF0000
:10E58800034060006041B300A6E6B700D8C6BF00EC
:10E59800034060003040B300D8E6B700D7C6BF00DC
:10E5A800034060005040B300D7E6B700C522A8007A
:10E5B800C122A900C482A800C082A900CD22A80057
:10E5C800C922A900C8C2A800A8C6BF0003406000AD
:10E5D8006040B300A8E6B700ACC6BF0003406000C7
:10E5E8005041B300ACE6B700C902A900C8C6BF00D5
:10E5F800034060000034A000C8E6B700C8E2A900E4
:10E60800C7C6BF00034060007040B300C7E6B7004C
:10E61800D4C6BF0003406000B040B300D4E6B700E2
:10E62800D3C6BF0003406000A040B300D3E6B700E4
:10E638000000060001087800220098008000EB0026
:10E648001100980000000600FCFF3700889FBE00FC
:10E658008004780081417800100490000800E000F0
:10E6680007003A00C0C3B30080CF50002400320036
:10E6780009007800F4FF070008007800460037001A
:10E68800C0C3B30080CF500019003200E40F54001B
:10E6980008003E00E0C3B30080CF500018003A00E5
:10E6A8008000EB0019007800B86B02000000000041
:10E6B8000F003700B0082000800F540010003A0007
:10E6C8008100FB000001EB00E0C3B30080CF5100E4
:10E6D80001003A0012002000828F5000080032002A
:10E6E8002100200019007800B86B0200000000002B
:10E6F80009007800D4FF07000000EB00260037006F
:10E7080063005400E10F500014003E0000CDB30038
:10E7180000C04100E94F5000100036002900900069
:10E7280012C2B3000274780029009000990090008A
:10E7380001004000124098002900900099009000C4
:10E748000100400023409800190090006300400039
:10E7580090049800100020000F0037002900900056
:10E7680003747800E0C3B30080CF510006003A007C
:10E7780019019000A90090000040EB0000F178001A
:10E788002000200004003700190090000000E80075
:10E7980090049800100020004F04BE0000000600FE
:10E7A8000001780054000700090032006C40400066
:10E7B80080CF5000060032006A40500080CF5000E1
:10E7C800030032006640500080CF500009003A0034
:10E7D800A24090004C00070008003200774050002B
:10E7E80080CF5000050032000040E80080CF500084
:10E7F800020032000000EB0001003700100020008A
:10E8080000000600800178003B00070009003A007C
:10E81800A340900000C0E80080CF500007003200FD
:10E828000300780054460200000000000001780050
:10E838000F0037003400070005003A000300780095
:10E84800724D020000000000000178000800370047
:10E858000001EB0020C4B30080CF500004003A0050
:10E8680003007800FE5E020000000000000178004E
:10E8780002007800000006000001BE001E0007002C
:10E888000D003A00A24090007540500080CF500023
:10E898001000320020C3B30080CF500003003A00BC
:10E8A800C00F2000030040001200370016000700C8
:10E8B8000F003A000B00370020C4B30080CF50008F
:10E8C80006003A00A24090007140500080CF5000EE
:10E8D80007003A0003007800060037000A00070026
:10E8E80003003A00801F20000300400001003700A9
:10E8F8000000EB00000006009040900060C4B300E8
:10E9080080CF50000000060080C4B30080CF5000C4
:10E91800000006000001780090407800F0C4B300C1
:10E9280080CF500008003A00924090006E4050009E
:10E9380080CF50000A0032000040E80080CF50002D
:10E9480009003A0006003700A0C5B30080CF500088
:10E9580005003A0012409000814F500002003A0032
:10E9680010002000010037000000EB000000060046
:10E9780000027800814178000040EB0050DA9800EE
:10E98800B4089000F0142400808F500007003A006B
:10E998002F00070080B52100320007002A0032004E
:10E9A800C0DA20004300070028003700F0242400C4
:10E9B800808F500007003A002500070000712200F0
:10E9C80028000700200032008038210039000700A5
:10E9D8001E0037000040EB0040DA980064489100C0
:10E9E8000004A100604A9900541090000080A10022
:10E9F800501298008000EB003132980041329800A4
:10EA08006011B800722A980003329800513A9800B1
:10EA1800613A9800118298002B0007000034A10089
:10EA2800604A990051329800613298006448910018
:10EA38000064A100604A990062029800730298007D
:10EA480001007800010037001000200000000600D7
:10EA5800421F200032329800E01520004032980012
:10EA68000000060001002000702A9800013298007A
:10EA7800523A98000000EB00603A9800120020001B
:10EA880012829800100007000034A000604A990024
:10EA9800800C200050329800400620006032980018
:10EAA800644891000064A100604A99000304E000F2
:10EAB8000000060001002000600298007102980022
:10EAC8000200780000000600644891000014A100CC
:10EAD800604A9900644891000000060021E2A800FD
:10EAE80021A2A9002182A9002162A90021C2BF0098
:10EAF800C1CFB3000140600021E2B70020E2A900C5
:10EB080020C2A90020A2A9002082A9002062A90091
:10EB180020C2BF0091CFB3000140600020E2B700DF
:10EB28002002A9005001200040118800B03EB0002A
:10EB380010118800A9C0BF000044A1000046B3001E
:10EB4800A9E0B7008560A9009560A800000006004C
:10EB5800416D8000506D8000808068000100EA00EF
:10EB6800010070004F00DE0000000600416D8000CB
:10EB780060D72000614078008100E800416D88007E
:10EB8800416D800022032000801F780011000900D9
:10EB98008200D800010178004F007800426D88009B
:10EBA8000000FB00000006008040780023C2BF0080
:10EBB8000018A300FDFF3A000100FB0020118800A7
:10EBC80000000600889FBE00000478008144780099
:10EBD800104078000004E00004003200F2FF070053
:10EBE800584078000004E000FCFF3A000904E00007
:10EBF80002003200A0C0B300EBFF070010002000A5
:10EC08004F04BE0000000600000006003600F800B1
:10EC1800809FBE00829FBE00841F780022C2BF0072
:10EC28000008A3001400320064D72000230320004A
:10EC380031118000506D800001707A00506D8000A5
:10EC4800426D80000000E800110009000300D800B0
:10EC5800828F500001003200AA2DEC00506D800018
:10EC6800110009000300D800516D880022C2BF00BE
:10EC78000008A300EEFF3A0022C2BF000008A3006C
:10EC880001003A008560A9004F0278004F01BE00DC
:10EC98004F00BE003600F900004006000080FB006F
:10ECA8004400DE00E94F5000030036007043B00016
:10ECB8000080FB00020037000043B0000080FB002A
:10ECC800000006006F406000E94F50000300360066
:10ECD8007043B0000080FB00020037000043B00022
:10ECE8000080FB0000000600889FBE008A9FBE00CF
:10ECF8008C9FBE0080047800010578006033B8005E
:10ED08000041EB00024478005C5020002D002000F8
:10ED18004B06200027003700E34F540029003E002F
:10ED280000CDB30000C040000204E000160032002D
:10ED3800E34F510003003A00E24F40003F003A0021
:10ED480002003700E24F40000F003A008C0F5300DA
:10ED58008D8F5B0039003E000880FB000781FB00B7
:10ED68000B91B9004832DE006A22B9000441410023
:10ED78000641410002707D000844E8006033B80095
:10ED88000041EB000B003700E94F50002B003E001C
:10ED98000241E800C83BDD000680FD00864378009C
:10EDA8000043EB008080FB0000F02F0000036300AD
:10EDB80001037300B94078000104E000D6FF3A006F
:10EDC8000F003700F0C2B30080CF50000C003200B3
:10EDD800EDCF50000A003200EACF500008003200A0
:10EDE8006F40500080CF500005003200E9CF50003E
:10EDF800030032007A40400080CF50000F003A00F4
:10EE08005050200021002000800F5300818F5B00AC
:10EE18000A003E000780FB00420620000280B9007D
:10EE28004831DE006A11B900024040000640400047
:10EE38003045980010002000010037000000EB006A
:10EE48004F06BE004F05BE004F04BE00000006007E
:10EE580000C3B3000461B70002A1EF000021EF0076
:10EE6800A5C0BF00F1C8B300014060000054A00075
:10EE7800A5E0B7008460A9009460A80005E1A80097
:10EE8800000006000400FA009460A80000000000DA
:10EE98009460A9000108800001007800ECEDB7003B
:10EEA8004808DE00EDEDB700D26F8000E36F800008
:10EEB800E2BF9F00F3BF9F00E18F400004003A00CB
:10EEC80061015100E0815900E2BF9F00F3BF9F003C
:10EED8004FF89700EEEDB7005FF89700EFEDB70039
:10EEE8006FF89700F0EDB7007FF89700F1EDB700E5
:10EEF80084C0BF000038A300E3FF3A009460A80074
:10EF08000080FA00000006000400FA00DDFF070098
:10EF1800ECCDBF00C0FF9F00EDCDBF00D0FF9F002C
:10EF2800EECDBF00E0FF9F00EFCDBF002F00070030
:10EF38000080FA00000006000400FA00D1FF070074
:10EF4800EDCDBF00C0FF9F00EECDBF00D0FF9F00FA
:10EF5800EFCDBF00E0FF9F00F0CDBF00230007000A
:10EF68000080FA00000006000400FA00C5FF070050
:10EF7800EECDBF00C0FF9F00EFCDBF00D0FF9F00C8
:10EF8800F0CDBF00E0FF9F00F1CDBF0017000700E4
:10EF98000080FA00000006006011B800E004B0002C
:10EFA8000180B0000280B0000380B000C4092000D6
:10EFB800050020006033B8002809020000000000A6
:10EFC80000000600809FBE00D06F8000E16F8000C7
:10EFD80061004000E0804800D06F8800E16F880041
:10EFE8008460A9004F00BE0000400600B0FF9F00EB
:10EFF8004FB89700DFB8970000000600C522A800A8
:10F008002012200010138800000028000013880038
:10F01800000006000080FB004013880060C2BF00AB
:10F028000008A300FDFF3200401380000080FB00B1
:10F0380000000600C522A90050C0B300F5FF070074
:10F048000040EB00F3FF0700C522A800F7FF3700D8
:10F05800C522A90060C0B300EEFF0700C522A800C2
:10F0680000000600889FBE008084FB00F1FF0700B7
:10F0780063046000FDFF3A00C522A90030C0B30058
:10F08800E4FF07004848DE00E2FF07000940780077
:10F09800E0FF070008407800DEFF0700C522A8004F
:10F0A8000080FB004F04BE0000000600889FBE00E1
:10F0B800814478000084FB00DEFF070063006000E5
:10F0C800FDFF3A00E2FF0700C522A90020C0B300F7
:10F0D800D0FF07004840DE00CEFF07000840780058
:10F0E800CCFF070009407800CAFF0700C522A80026
:10F0F8004F04BE0000000600889FBE008004780010
:10F10800CCFF070063046000FDFF3A00C522A90098
:10F1180030C0B300BFFF07004848DE00BDFF07004E
:10F1280009407800BBFF070008407800B9FF0700D6
:10F13800C522A8000080FB004F04BE0000000600A6
:10F14800889FBE000004780081447800B9FF07005A
:10F1580063006000FDFF3A00BDFF0700C522A9005B
:10F1680020C0B300ABFF07004840DE00A9FF07003E
:10F1780008407800A7FF070009407800A5FF0700AE
:10F18800C522A8004F04BE000000060000000600CB
:10F19800889FBE008A9FBE008C9FBE0080047800B6
:10F1A80000889000E20F500006003200495090009D
:10F1B8000044A100540007000000EB00B0A4980030
:10F1C8004D00370019889000E10F500047003A00C1
:10F1D80039A69000EE0F560018003E0049AD900089
:10F1E800D9AD900029A99000B9A990000A00BE00E5
:10F1F800B4050200000000000000E0003E003200FC
:10F20800AAAC9800BBAC98000C044600880AB00071
:10F2180002002400C36124000A00BE00B8050200F1
:10F2280000000000200602000000000000B47C007E
:10F238000C00E800B0A498002F0037008A0A2000CC
:10F24800090545006066B8008005EB001A047800DF
:10F258006140B90056060200000000000800E00006
:10F2680004003D000200200003782400AE060200DE
:10F27800000000000001BE000C00BE00AE06020047
:10F28800000000000006BE008B05E8000A85E800C3
:10F29800EF8F5500EDFF3A000000EB00B0A4980096
:10F2A80002002000031724000C00BE0068070200BB
:10F2B80000000000EC070200000000004200DD0032
:10F2C800A2002000110009000280D800E29220006C
:10F2D80000015100D2A49800820C78004950900097
:10F2E8000044A000080007000300370049509000C0
:10F2F8000044A100C05498004F06BE004F05BE0050
:10F308004F04BE0000000600C05498004950900009
:10F318000054A100C0549800000006000000FA0044
:10F32800889FBE008A9FBE008C9FBE000606BE0056
:10F3380002055000838558005FB39700EFB397002C
:10F348000C0353008D835B000A30B80007D4B90062
:10F35800010444000BB3B9008600440002015200C6
:10F3680083815A004A0A0200000000000C0640008F
:10F378008D8648000C00BE004F06BE004F05BE003B
:10F388004F04BE000080FA0000000600889FBE00FF
:10F398008A1F780080047800010578000100780051
:10F3A8000001EB008900E900130037000204E800BF
:10F3B800888F54000E003600000378000081E800B2
:10F3C8008002EB00888354001202780096017800CE
:10F3D800830F520002003100040B78000309780003
:10F3E8008502E8000281E800858F5300F6FF3A00A5
:10F3F8000080E80008017800810F5100EBFF390018
:10F408000908A3000D003A00090078000000A100D7
:10F418000000450070BC970010044400100007006D
:10F4280001003D00130007000200200003F0230044
:10F43800B805020000000000060037000900780047
:10F448000000A10060047D000500070001003D00E8
:10F45800080007004F0578004F04BE0000000600B2
:10F468006140B90056060200000000000800E000F4
:10F47800000006000200200003782400AE06040005
:10F4880000000000C1DC20000600090031187800E7
:10F49800E000B10000000600405290000482FB002A
:10F4A800D0509000C808DD000481700060529000C0
:10F4B8000482FB00F0509000C808DD0084817000D1
:10F4C800626E8800736E8800404290000482FB00E0
:10F4D800D0409000C808DD000481700060429000B0
:10F4E8000482FB00F0409000C808DD0084817000B1
:10F4F800826E8800936E8800004A90000482FB00A8
:10F5080090489000C808DD0004817000204A9000EF
:10F518000482FB00B0489000C808DD0084817000B8
:10F52800A26E8800B36E8800406890004600DE0036
:10F5380061006000D8EDB700000006000300070076
:10F548000080FB000000EA000300370001007000A3
:10F558008000EA00008070004F00DE000000060016
:10F5680001000700F6FF3700F8FF37000100070029
:10F57800F3FF3700F5FF3700EEFF3700606E8000BD
:10F58800716E8000F1FF07000004E0000B003200FC
:10F59800806E8000916E8000F3FF07000004E00099
:10F5A80006003200A06E8000B16E8000F1FF0700F7
:10F5B800110020000004E00001003A008000EB0088
:10F5C800010078000000060000000600889FBE00C9
:10F5D8008A9FBE008C9FBE008E1F780000057800B1
:10F5E8000107780070162000808F500003003E004D
:10F5F8006044B8000806BE00100037008A0578008D
:10F608006044B8000806BE000B057800811620008B
:10F618001C0007008100E900FDFF3A001F000700F9
:10F628000006BE0080E92F00000747000B2DB00040
:10F6380070162000800F5700F3FF3E000E00E00018
:10F64800050032008000EB000E0007008100E80092
:10F65800810F5700FCFF3A0010000700C000DD00D2
:10F668000000200000047400818474000800BE00BB
:10F678004F0778004F06BE004F05BE004F04BE007E
:10F68800000006003A00780000044400E0844C00C2
:10F698000C0644008D864C0000000600F2FF2F0087
:10F6A800030020000800BE002E0802000000000031
:10F6B8000004BE00F2FF2F00030020000C00BE0073
:10F6C8002E08040000000000CF80DE00EE0F50007E
:10F6D800E08F58002E003E00006001000E00370049
:10F6E800130037000E0037001300370020003700E2
:10F6F8001D003700200037001500370016003700BE
:10F7080017003700080037001D0037000E003700CB
:10F718000B0037001C003700606D80001D003700AB
:10F72800806D80001B003700006E800019003700D4
:10F73800706D800017003700906D8000150037004D
:10F74800306E800013003700206E800011003700F3
:10F75800D06D80000F003700E06D80000D0037008D
:10F76800F06D80000B003700B06D80000900370095
:10F77800A06D800007003700C06D800005003700CD
:10F78800106E800003003700406E800001003700D3
:10F79800506E800000000600881F78000004780082
:10F7A800002890001800500028C99000F3CBB3003F
:10F7B800034141000281FB0002014100C202B00086
:10F7C80062017C000280B900A20020000300200032
:10F7D8004A0A0200000000000002BE00E00F5000CC
:10F7E800E08F580008003D0060011000E08118001B
:10F7F80068209000F82090006033B800800F510016
:10F80800818F590004003E0068209000F820900085
:10F8180004034000858348007828900088309000D1
:10F82800800F5300818F5B0002003600782B900018
:10F83800883390000600BE004F04780000000600E0
:10F84800000178006000B8000200E0000500320006
:10F858000300200080B22600E10E2000940502007B
:10F868000000000000000600000006006000B8006C
:10F8780000000600000006000000EB000000060083
:10F88800FDFF37008001780040B89000810F5000DC
:10F898000400360043B8900011002000820F500089
:10F8A8000300390043B89000D0B198008000EB0005
:10F8B800010078000000060080017800E050900008
:10F8C800F0C4B30080CF500016003A00F350900007
:10F8D8006B40500080CF500006003A00828920001B
:10F8E800810C200003007800E6FF07000080FB0081
:10F8F8000D00370090C4B30080CF500003003200E1
:10F90800A0C4B30080CF500006003A00C2C1200056
:10F9180001AF200003007800DAFF07000080FB0039
:10F92800010037000000EB000000060000000600A0
:10F938007275020000000000A2C7200021C7200045
:10F9480060D020001E7302000000000020C72000C5
:10F9580000000600E6750200000000000000060036
:10F96800881F78000004EB000B003700BA7502000E
:10F97800000000008040780060D020002A73020058
:10F9880000000000000478000000E0000D003200D4
:10F99800E20F500006003200AC75020000000000C3
:10F9A8000004E000F1FF3A00E20F540005003A00BD
:10F9B80060D0200028730200000000001000200022
:10F9C800010037000000EB004F047800000006003B
:10F9D800A0C7200000000600889FBE008A1F78008C
:10F9E800000578008004EB000800370038C0B30039
:10F9F8009001200001002000090007000844E900E8
:10FA0800E14F4400FAFF3A008904E800890F5500E5
:10FA1800F6FF3A004F0578004F04BE0000000600CC
:10FA28000400FA00820220000202B8000289B9002C
:10FA380085024100E4BF9F00F5BF9F000080EB00F6
:10FA48008080EB006FB99700FFB997006101510002
:10FA5800E0815900E2BF9F00F3BF9F006FB9970094
:10FA6800FFB99700800F5100818F5900F5FF3A00C8
:10FA78000080FA0000000600CF80DE00F20F2000B0
:10FA880003002000829FBE006033B80034062000C7
:10FA9800050020000601BE00927902000000000067
:10FAA8000070880002000700E48757000000060085
:10FAB800011920009140780082CFB30082C0600015
:10FAC8006140B3008000FD0090E1B7008000FD00B8
:10FAD8009061A800600C880000000600F00F20006C
:10FAE800F3FF0700000006000000EB00F0FF07002E
:10FAF8000000060000708000EDFF0700000006000F
:10FB0800889FBE0080047800010478007C0C020005
:10FB180000000000880F50000F003E000000E000C9
:10FB28000D003200C103200009007800980C020083
:10FB3800000000000000E00007003A00E103200098
:10FB480009007800980C0200000000001100200055
:10FB58000000E000010032008000EB0001007800A6
:10FB68004F04BE00000006001041780000C3B30037
:10FB7800804F510003003A008048EB008001EB0001
:10FB8800070037001300200010C3B300804F510056
:10FB980003003A0010C0B300804878008001EB00F1
:10FBA80003007800000006000000FE0000000600C8
:10FBB8000000FE0000000600100020000000060003
:10FBC800FDFF3700FCFF370000000600F07C020054
:10FBD800000000000000060008CEBF000080FB0007
:10FBE8000000060031C6B300814F50000100360006
:10FBF8000140780008EEB7000080FB00407D02005D
:10FC080000000000000006008000EB0061A09800E2
:10FC1800CA7802000000000000000600CC7802004C
:10FC28000000000000000600BC7402000000000094
:0CFC38000080FB00000006000000060039
:00000001FF
